:10000000D6C700000C9408080C9408080C94080843
:100010000C940808FDC70000FBC70000F9C70000EA
:10002000F7C70000F5C70000F3C70000F1C70000E4
:10003000EFC700000C947365EBC70000E9C7000030
:10004000E7C70000E5C70000E3C70000E1C7000004
:10005000DFC70000DDC70000DBC700000C94FF898C
:10006000D7C700000C94E88D0C941E8ED1C70000F9
:10007000CFC70000CDC70000CBC70000C9C7000034
:10008000C7C70000C5C70000C3C70000C1C7000044
:100090000C94938E0C94C98EBBC700000C940A7804
:1000A000B7C70000B5C70000B3C70000B1C7000064
:1000B000AFC70000ADC70000ABC70000A9C7000074
:1000C000A7C70000A5C70000A3C700000C943E8F7F
:1000D0000C94748F9DC700000C94E98F0C941F90B2
:1000E00097C70000364D164D3F4D3F4D3F4D3F4D9C
:1000F0003F4D3F4D3F4D3F4D3F4D3F4D6D4B7F4B36
:10010000864B8C4B934B994B9E4BA74BAE4BC54BA1
:10011000C84B3F4DDA4BDD4BE04BE34BFD4BFF4B08
:10012000064C0D4C204C274C2E4C3F4D3F4D3F4D27
:100130003F4D3F4D3F4D3F4D3F4D3F4D3F4D694C36
:100140003F4D3F4D3F4D3F4D3F4D3F4D6D4D4C8BD6
:100150004F8B3E8B428B488B868B538B578B5D8BA3
:10016000618B658B6B8B6F8B738B868B798B7D8BA8
:10017000818B084AD73B3BCE016E84BCBFFDC12FAB
:100180003D6C74319ABD56833DDA3D00C77F11BE88
:10019000D9E4BB4C3E916BAAAABE000000803F0789
:1001A000634236B79BD8A71A39685618AEBAAB5512
:1001B0008C1D3CB7CC5763BD6DEDFD753EF61772D7
:1001C00031BF000000803F08000000BE92244912A9
:1001D0003EABAAAA2ABECDCCCC4C3E00000080BECD
:1001E000ABAAAAAA3E00000000BF000000803F00AA
:1001F00000000000084178D3BB4387D1133D190E9E
:100200003CC3BD4282AD2B3E68EC8276BED98FE105
:10021000A93E4C80EFFFBE01C4FF7F3F00000000FD
:1002200000004D6F74696F6E004D6F74696F6E00E2
:10023000696E7075742044535463616C69627261B5
:1002400074653A004E6F2053656E736F7221004ED5
:100250006F20445320546865726D6F6D65746572CC
:100260002100445320546865726D2E005556204974
:100270006E742E00555620496E74656E73697479DC
:1002800000234E6F2073656E736F722100536F757C
:100290006E64204C6576656C004D6561737572699E
:1002A0006E672E2E00234E6F2073656E736F722162
:1002B00000536F756E64204C6576656C00234E6F3D
:1002C0002073656E736F7220666F7220504D21002F
:1002D0004E6F2073656E736F722100206E672F4C16
:1002E00000504D313A322E353A3130004D65617350
:1002F0007572696E672E2E004F3220436F6E630059
:10030000434F3220436F6E630053656E736F7220EC
:100310006572726F722100234E6F2073656E736F6A
:10032000722100434F3220436F6E63004D6561734D
:100330007572696E6700234E6F2070482073656E7A
:10034000736F72210070482076616C756500234ED2
:100350006F2054422073656E736F723F004E6F20A2
:1003600073656E736F72210049522054656D70651C
:10037000726174757265004D6561737572696E673F
:100380002E2E004E6F2073656E736F723F004952C0
:100390002054656D7065726174757265004D65619C
:1003A000737572696E672E2E004C696768742049F8
:1003B0006E74656E7369747900416E676C65732F36
:1003C000003E6128782C792C7A292F673A006765DE
:1003D0007453656C665465737442697428293A20B5
:1003E000006973496E74657272757074456E6162EE
:1003F0006C65642831293A2000676574496E74651C
:1004000072727570744D617070696E672831293A27
:100410002000676574496E74657272757074536FED
:10042000757263652831293A2000676574496E74D6
:10043000657272757074536F7572636528293A20FE
:10044000006765745261746528293A20332E31346F
:100450003135393F00616363656C2E69734C6F778A
:10046000506F77657228293A2000616363656C2EAE
:10047000697341736C65657028293A200061636374
:10048000656C2E6973546170536F757263654F6E3E
:100490005A28293A2000616363656C2E69735461A0
:1004A00070536F757263654F6E5928293A20006149
:1004B0006363656C2E6973546170536F7572636505
:1004C0004F6E5828293A2000616363656C2E69736A
:1004D0004163746976697479536F757263654F6EA1
:1004E0005A28293A2000616363656C2E6973416361
:1004F000746976697479536F757263654F6E5928A4
:10050000293A200069734163746976697479536F7D
:10051000757263654F6E5828293A200069735461DB
:1005200070446574656374696F6E4F6E5A28293B19
:100530002066616C73653F20006973546170446587
:1005400074656374696F6E4F6E5A28293B2074720C
:1005500075653F2000697354617044657465637408
:10056000696F6E4F6E5928293B2066616C73653F39
:1005700020006973546170446574656374696F6EBB
:100580004F6E5928293B20747275653F20006973AE
:10059000546170446574656374696F6E4F6E58285A
:1005A000293B2066616C73653F200069735461705C
:1005B000446574656374696F6E4F6E5828293B20DB
:1005C000747275653F20006765745375707072654D
:1005D000737342697428293B2066616C73653F2000
:1005E000006765745375707072657373426974281F
:1005F000293B20747275653F2000697341637469FB
:1006000076697479416328293A20006973496E61DB
:10061000637469766974795A456E61626C656428A1
:10062000293A20006973496E616374697669747947
:1006300059456E61626C656428293A2000697349E6
:100640006E616374697669747958456E61626C6530
:100650006428293A20006973416374697669747962
:100660005A456E61626C656428293A2000697341BD
:100670006374697669747959456E61626C65642842
:10068000293A200069734163746976697479584521
:100690006E61626C656428293A2000676574467251
:1006A000656546616C6C4475726174696F6E28296A
:1006B0003A20006765744672656546616C6C5468E3
:1006C000726573686F6C6428293A200067657454FA
:1006D000696D65496E616374697669747928293A30
:1006E0002000676574496E61637469766974795432
:1006F00068726573686F6C642829200067657441AF
:10070000637469766974795468726573686F6C6430
:1007100028292000676574446F75626C65546170A8
:1007200057696E646F7728292000676574446F7578
:10073000626C655461704C6174656E637928293A06
:1007400020006765745461704475726174696F6EDE
:1007500028293A2000676574417869734F6666738B
:1007600065742826782C2026792C20267A293A2090
:10077000006765745461705468726573686F6C6467
:1007800028293A200058595A2047733A20005859CE
:100790005A20434F554E54533A20007365742067D6
:1007A00061696E735B5D3A006761696E735F6F725A
:1007B00069675B5D3A00466C616D65204952004F88
:1007C0006666206169722D636F6E6421004974272B
:1007D0007320746F6F20636F6F6C210054656D70B0
:1007E0002069732066696E65210049732061697212
:1007F0002D636F6E64206F6E3F0049742773207104
:100800007569746520686F742100497427732076B8
:1008100065727920686F74210054656D7020487589
:100820006D696469747900234E6F2073656E736F10
:100830007220666F722074656D7020262068756D59
:10084000696469747921004E6F2053656E736F720D
:10085000210054656D702048756D69646974790074
:100860004F6666206169722D636F6E642100497462
:10087000277320746F6F20636F6F6C210054656D58
:10088000702069732066696E652100497320616973
:10089000722D636F6E64206F6E3F00497427732062
:1008A000717569746520686F74210049742773201D
:1008B0007665727920686F7421200023616E6F74F1
:1008C00068657220495220696E7075743D00496EEA
:1008D00076616C6964206B65792100233A53686FF7
:1008E000772F48696465204C4344002A3A5468696C
:1008F000732048656C700044433A436C6561722014
:100900004C43440044423A5265736574204C6F670F
:100910006765720044373A4D6F74696F6E004436F4
:100920003A44532054656D700044353A5556204979
:100930006E74656E736974790044343A4F32206383
:100940006F6E632E0044333A434F3220636F6E6301
:100950002E0044323A504D28313A322E353A313059
:10096000290044323A504D28313A322E353A31304E
:10097000292A0044313A54757262696469747900B5
:1009800044303A566F6C7461676500393A6F722073
:10099000334420616363656C2E00393A496E636CA1
:1009A0002E20616E672E00383A70482076616C7593
:1009B0006500373A49522054656D7000373A495204
:1009C0002054656D702A00363A4D61676E65746912
:1009D00063206669656C6400353A476173204C6535
:1009E00076656C00343A495220466C616D6500337F
:1009F0003A4C6967687420496E742E00323A616E11
:100A0000642048656967687400323A54656D7020E7
:100A1000507265737375726500313A54656D70205C
:100A200048756D696469747900303A536F756E6406
:100A3000204C6576656C00303A536F756E64204CBF
:100A40006576656C2A002020202020202020202090
:100A500020202020200020202020202020202020B6
:100A600020202020200020202020202020202020A6
:100A70002020202020200020202020202020202096
:100A80002020202020202000202020202020202086
:100A90002020202020202020002020202020202076
:100AA00020202020202020202000482D6669656C11
:100AB000643A2028004C6F6767657220446972654C
:100AC0006374696F6E00482D6669656C64005365D8
:100AD0006172636820446972656374696F6E002394
:100AE0002D2D2D2D2D2D2D2D2D2D2D2D2D2D2D2D36
:100AF0002D2D2D2D2D2D2D2D2D2D2D2D2D2D2D2D26
:100B00002D2D2D2D00235265736F6C7574696F6EDA
:100B10003A20202000234D696E2056616C75653A9D
:100B20002020202000234D61782056616C75653AA5
:100B3000202020200023556E697175652049443AB4
:100B40002020202000234472697665722056657249
:100B50003A202020002353656E736F723A202020C4
:100B60002020202000232D2D2D2D204D61676E6526
:100B70007469632053656E736F72202D2D2D2D2D9A
:100B80002D2D2D2D2D2D2D2D2D2D2D2D2D2D2D00C2
:100B90006E6F20484D4335383833206D61676E6580
:100BA0007469632073656E736F72202E2E2E20433E
:100BB0006865636B20776972696E672100236B65D6
:100BC000793D0020766F6C746167653D0023547534
:100BD00072626964697479205570706572204C691D
:100BE0006D69743A200020766F6C746167653D0012
:100BF00023547572626964697479204C6F776572E9
:100C0000204C696D69743A200023547572626964DE
:100C1000697479204C6F776572204C696D69742016
:100C200056696E663A200023434F32204D415820CA
:100C3000766F6C7420280023434F32207A65726FE0
:100C400020766F6C74202800234F322063616C691A
:100C500062726174696F6E3A200023547572626922
:100C600064697479204C6F776572204C696D697482
:100C70002056313A200043616C6962726174696F79
:100C80006E2050726573737572653D005365612007
:100C90006C6576656C20502863616C63293D002388
:100CA0004572726F723A7072657373757265204225
:100CB0004D503038352C20636865636B207769723E
:100CC000696E67210049522054656D702073656E0E
:100CD000736F7220666F756E6400504D322E352032
:100CE00073656E736F72206C696B656C7920666FCB
:100CF000756E6400456455484B205345534C6F67EF
:100D00006765720053656E736F7220736C6F742029
:100D1000616E6420747970653A0057656C636F6D1D
:100D20006520746F20456455484B00005EBCE2614D
:100D30003FDD83C29C7E20A3FD1F41009D23BE4654
:100D4000DB65F88C11AF32CA57E97400000A0B0258
:100D5000090C0D0E0807030401000000000000004C
:100D60000000000000000000000000000000000083
:100D70000000000000000012111000000000000040
:100D80000000000000000000000000000000000063
:100D9000000102102020080810204010204080028E
:100DA00001020108040201010204081020408080B1
:100DB0004020100804020180040201804020100835
:100DC000040201080402010102040810204080010D
:100DD00002040810204080050505050705080808DD
:100DE00008020202020A0A080804040404010101BC
:100DF00001010101010303030303030303040707C4
:100E0000070C0C0C0C0C0C0C0C0202020206060661
:100E100006060606060B0B0B0B0B0B0B0B0000203C
:100E2000002300260029002C002F003200000100C2
:100E30000003010601090100002200250028002B03
:100E4000002E003100340002010000050108010BF2
:100E50000100002100240027002A002D003000336B
:100E60000001010000040107010A014E414E494EF4
:100E7000495459494E46CDCCCC3D0AD7233C17B7EF
:100E8000D13877CC2B329595E6241FB14F0A00005C
:100E900020410000C84200401C4620BCBE4CCA1B7A
:100EA0000E5AAEC59D7400407A10F35A00A0724EDF
:100EB00018090010A5D4E80000E87648170000E4FF
:100EC0000B54020000CA9A3B000000E1F505000047
:100ED00080969800000040420F000000A0860100AC
:100EE0000000102700000000E8030000000064007C
:100EF000000000000A0000000000010000000000E7
:100F00002C76D888DC674F0823DFC1DFAE59E1B10A
:100F1000B796E5E3E453C63AE651997696E8E6C219
:100F20008426EB898C9B62ED407C6FFCEFBC9C9F20
:100F300040F2BAA56FA5F490055A2AF75C936B6C42
:100F4000F9676DC11BFCE0E40D47FEF520E6B50036
:100F5000D0ED902E0300943577050080841E0800A4
:100F600000204E0A000000C80C333333330F986E54
:100F700012831141EF8D2114893BE65516CFFEE611
:100F8000DB18D1844B381BF77C1D901DA4BBE424D7
:100F9000203284725E228100C9F124ECA1E53D2754
:100FA00059372177508EFB8EA68F5190F23711243E
:100FB0001FBECFEFD1E2DEBFCDBF00E00CBF1BE014
:100FC000A0E0B2E0E8E6F9E401E00BBF02C0079060
:100FD0000D92A032B107D9F721E1A0E2BBE001C038
:100FE0001D92A53BB207E1F71FE0CCEADFE000E08D
:100FF00006C022970109FE010BBF0E94269DC03A40
:10100000D10780E00807A9F70E9454980C94A3A484
:101010000C940000CF92DF92EF92FF920F931F93F8
:10102000E82FF92F05C0015011092109310961F19B
:10103000908196239417B9F305C001501109210935
:10104000310911F1908196239413F7CFC12CD12C43
:10105000E12CF12C0AC08FEFC81AD80AE80AF80A66
:101060000C151D052E053F0579F080818623841718
:1010700091F36C2D7D2D8E2D9F2D1F910F91FF9043
:10108000EF90DF90CF90089560E070E080E090E016
:101090001F910F91FF90EF90DF90CF90089527E37D
:1010A0003AE0FC01318320830895089527E33AE074
:1010B000FC01318320830C9462982F923F924F92CF
:1010C0005F926F927F928F929F92AF92BF92CF92D8
:1010D000DF92EF92FF920F931F93CF93DF93CDB7E1
:1010E000DEB72E970FB6F894DEBF0FBECDBF8C01D2
:1010F0007E876D87DC014D915C91119712962D9141
:101100003C911397421753072CF4942F852FA90174
:10111000292F382FD801149660E070E0CB01E2E06F
:10112000F0E0ED84FE84EE15FF0544F5CD90DD90F2
:10113000C216D3065CF44901AA2497FCA094BA2CE9
:10114000680D791D8A1D9B1D960116C04C155D0505
:101150005CF44A01AA2497FCA094BA2C680D791D6E
:101160008A1D9B1DA60108C0EE24D7FCE094FE2C2E
:101170006C0D7D1D8E1D9F1D3196D3CF0E94FB9956
:101180006B017C016D857E8562507109882777FD32
:101190008095982F0E94FB999B01AC01C701B60175
:1011A0000E942F996B017C012D853E8524313105EC
:1011B0000CF4BFC04801412C512C3201A12CB12CA0
:1011C000D4016D917D914D01882777FD8095982FF1
:1011D0000E94FB99A70196010E9464989B01AC01B3
:1011E0000E948F9B9B01AC01C301B2010E946598D4
:1011F0002B013C01BFEFAB1ABB0AED85FE85AE1695
:10120000BF06F1F6BF0161507109882777FD80950F
:10121000982F0E94FB999B01AC01C301B2010E946F
:101220002F990E94429C4B015C0120E030E040E895
:101230005FE30E94D09A18160CF07BC018870F83CA
:10124000212C312C1B821C821D821E821A82198243
:10125000AF81B8858D919D91B887AF839C0144275C
:1012600037FD4095542F29873A874B875C87CA0101
:10127000B9010E94FB99A70196010E9464982B0175
:101280003C0120E030E0A9010E94D09A181624F019
:10129000C301B201905802C0C301B201A50194017B
:1012A0000E942B9987FF13C08B819C81AD81BE81E9
:1012B00029853A854B855C85820F931FA41FB51F36
:1012C0008B839C83AD83BE833FEF231A330A49810E
:1012D0005A814F5F5F4F5A8349838D859E8548179A
:1012E000590709F0B5CF20E030E040EC5FE3C501DD
:1012F000B4010E948F9B4B015C0195E029163104DB
:101300000CF49CCF6B817C818D819E810E94FB9926
:101310006B017C01B101882777FD8095982F0E9491
:10132000FB999B01AC01C701B6010E942F996B018B
:101330007C01C701B6012E960FB6F894DEBF0FBE32
:10134000CDBFDF91CF911F910F91FF90EF90DF9074
:10135000CF90BF90AF909F908F907F906F905F9055
:101360004F903F902F900895CF93DF93EC01FB01B6
:10137000248135810E949F97CE01DF91CF910895FE
:1013800026E00C94558DDC01ED91FC910190F081EB
:10139000E02D1994EF92FF920F931F93CF93DF9359
:1013A0001F92CDB7DEB77C01FC0100811181C8011D
:1013B00069830E94A2A06981681719F0C8010E9480
:1013C000AAA0C7010F90DF91CF911F910F91FF90BD
:1013D000EF900895EF92FF920F931F93CF93DF93B7
:1013E0001F921F92CDB7DEB703E61BE083569B40EA
:1013F0007C01C701800F911FF80161918F019A83D1
:101400008983CE010196C6DFFBE00B3D1F0789F7FC
:1014100083E69BE00F900F90DF91CF911F910F918A
:10142000FF90EF9008950F931F93CF93DF931F9238
:101430001F92CDB7DEB70FE91DE0F80160818EED98
:1014400093E09A838983CE010196A4DFF80161813C
:101450008FED93E09A838983CE0101969BDFC801CB
:101460000F900F90DF91CF911F910F9108950F93DF
:101470001F93CF93DF9300D000D0CDB7DEB78C01A0
:101480008091790C8823A1F065EA76E0CE0101967F
:101490000E94B894B801CE0101960E94B196BC0199
:1014A0008BE39FE00E941E91CE0101960E944D9415
:1014B00026960FB6F894DEBF0FBECDBFDF91CF9159
:1014C0001F910F910895BF92CF92DF92EF92FF92FA
:1014D0000F931F93CF93DF93CDB7DEB762970FB60D
:1014E000F894DEBF0FBECDBF6C017B018A018091F5
:1014F000F704882309F480C08091F604882309F456
:101500007BC077FF09C0E094F09440E06E2D8FE837
:101510009DE00E94DC7F4CC040E060E08FE89DE0F1
:101520000E94DC7F0E94498A28EE33E040E050E0D0
:101530000E94F49CBA01A9012AE0CE0101960E9402
:10154000AE95BE016F5F7F4FCE0107960E94379523
:1015500060E578E0CE0107960E94C296BC01CE01FC
:101560000D960E943795CE0107960E944D94CE01AC
:1015700001960E944D94BE01635F7F4F8FE89DE00E
:101580000E94F590B98840E06B2D8FE89DE00E94A5
:10159000DC7FE114F10411F4EB2C06C040E06E2D69
:1015A0008FE89DE00E94DC7FCE010D960E944D9455
:1015B000B6018FE89DE00E94F59069E97AE08FE836
:1015C0009DE00E94D290F60164816E0D40E08FE8AC
:1015D0009DE00E94DC7F0E94498A60938B0D70938E
:1015E0008C0D80938D0D90938E0DB801882777FD1B
:1015F0008095982F0E94788A62960FB6F894DEBF85
:101600000FBECDBFDF91CF911F910F91FF90EF9053
:10161000DF90CF90BF9008954F925F926F927F922C
:10162000AF92BF92CF92DF92EF92FF920F931F93F0
:10163000CF93DF93CDB7DEB762970FB6F894DEBFD6
:101640000FBECDBF6C017B015A018091F704882346
:1016500009F498C08091F604882309F493C00E948D
:10166000498A00918B0D10918C0D20918D0D309138
:101670008E0D4090EA045090EB046090EC04709062
:10168000ED04040D151D261D371D06171707280725
:10169000390708F077C0F7FE0AC08701009510955A
:1016A00040E0602F8FE89DE00E94DC7F47C040E073
:1016B00060E08FE89DE00E94DC7F0E94498A28EE6E
:1016C00033E040E050E00E94F49CBA01A9012AE016
:1016D000CE0101960E94AE95BE016F5F7F4FCE0195
:1016E00007960E94379560E578E0CE0107960E9444
:1016F000C296BC01CE010D960E943795CE01079689
:101700000E944D94CE0101960E944D94BE01635FEC
:101710007F4F8FE89DE00E94F59009891A89E114B6
:10172000F10441F00E0D1F1D40E0602F8FE89DE099
:101730000E94DC7FCE010D960E944D94B6018FE889
:101740009DE00E94F59068E87AE08FE89DE00E94B5
:10175000D290F6016481600F40E08FE89DE00E9426
:10176000DC7F0E94498A60938B0D70938C0D80936F
:101770008D0D90938E0DB501882777FD8095982F5C
:101780000E94788A62960FB6F894DEBF0FBECDBF76
:10179000DF91CF911F910F91FF90EF90DF90CF904D
:1017A000BF90AF907F906F905F904F9008958F9211
:1017B0009F92AF92BF92CF92DF92EF92FF920F93E0
:1017C0001F93CF93DF937C016B01EA018091F704B3
:1017D000882309F474C08091F604882309F46FC04B
:1017E00077FF1CC0C094D09441E06C2D8FE89DE041
:1017F0000E94DC7FB7018FE89DE00E94F59067E7CB
:101800007AE08FE89DE00E94D290F70164816C0D30
:1018100041E08FE89DE00E94DC7F3EC00E94498A43
:101820000091EA041091EB042091EC043091ED0456
:101830008090870D9090880DA090890DB0908A0DB2
:10184000080D191D2A1D3B1D061717072807390704
:10185000B0F541E06C2D8FE89DE00E94DC7FB70180
:101860008FE89DE00E94F59066E67AE08FE89DE0C3
:101870000E94D290F70164816C0D41E08FE89DE0F9
:101880000E94DC7F0E94498A6093870D7093880DC7
:101890008093890D90938A0DBE01882777FD8095EE
:1018A000982FDF91CF911F910F91FF90EF90DF90D4
:1018B000CF90BF90AF909F908F900C94788ADF91DB
:1018C000CF911F910F91FF90EF90DF90CF90BF903D
:1018D000AF909F908F9008958091F704882379F0BE
:1018E0008091F604882359F06FED8FE89DE00E9407
:1018F000049169E775E08FE89DE00C9403910895E9
:10190000CF93DF93EC018091F7048823A1F08091BD
:10191000F604882381F06FED8FE89DE00E9404912A
:101920008C819D81892B39F0BE018FE89DE0DF918C
:10193000CF910C94F590DF91CF9108958091F704A9
:10194000882301F18091F6048823E1F08FE89DE07F
:101950000E94D07F40E060E08FE89DE00E94DC7F45
:1019600066E57AE08FE89DE00E94D29041E060E079
:101970008FE89DE00E94DC7F66E47AE08FE89DE0DE
:101980000C94D2900895CF93DF93CDB7DEB72C9708
:101990000FB6F894DEBF0FBECDBF8091D90B9091EA
:1019A000DA0B892B01F56CE075E0CE0107960E94F9
:1019B000B89461E87DE0CE0107960E94B196BC0123
:1019C000CE0101960E94379548EC50E06FEF7FEF13
:1019D000CE01019678DDCE0101960E944D94CE0194
:1019E00007960E944D948091D90B9091DA0B019744
:1019F00001F560E175E0CE0107960E94B89461E8B8
:101A00007DE0CE0107960E94B196BC01CE01019601
:101A10000E94379548EC50E06FEF7FEFCE010196C2
:101A200052DDCE0101960E944D94CE0107960E9490
:101A30004D9466E175E0CE0107960E94B8946BE77D
:101A40007DE0CE0107960E94B196BC01CE010196C1
:101A50000E94379540ED57E06FEF7FEFCE01019682
:101A6000A6DECE0101960E944D94CE0107960E94FB
:101A70004D9480919D0D90919E0D019719F467E30F
:101A80007AE002C069E27AE0CE0101960E945696A1
:101A900048EC50E06FEF7FEFCE010196BDDDCE0147
:101AA00001960E944D9469E17AE0CE0101960E9470
:101AB000569640ED57E06FEF7FEFCE01019677DE4F
:101AC000CE0101960E944D9469E07AE0CE01019624
:101AD0000E94569648EC50E06FEF7FEFCE010196E2
:101AE0009BDDCE0101960E944D946CEF79E0CE0112
:101AF00001960E94569640ED57E06FEF7FEFCE01C2
:101B0000019655DECE0101960E944D946FEE79E06C
:101B1000CE0101960E94569648EC50E06FEF7FEFA1
:101B2000CE01019679DDCE0101960E944D9464EEBE
:101B300079E0CE0101960E94569640ED57E06FEF96
:101B40007FEFCE01019633DECE0101960E944D94C7
:101B500068ED79E0CE0101960E94569648EC50E07F
:101B60006FEF7FEFCE01019657DDCE0101960E9407
:101B70004D9467EC79E0CE0101960E94569640EDB7
:101B800057E06FEF7FEFCE01019611DECE01019697
:101B90000E944D9480919D0D90919E0D039719F494
:101BA0006CEB79E002C062EB79E0CE0101960E9415
:101BB000569648EC50E06FEF7FEFCE0101962CDD9A
:101BC000CE0101960E944D9467EA79E0CE0101961C
:101BD0000E94569640ED57E06FEF7FEFCE010196E1
:101BE000E6DDCE0101960E944D946AE979E0CE01CE
:101BF00001960E94569648EC50E06FEF7FEFCE01C1
:101C000001960ADDCE0101960E944D946BE879E0C1
:101C1000CE0101960E94569640ED57E06FEF7FEFA0
:101C2000CE010196C4DDCE0101960E944D9460E87C
:101C300079E0CE0101960E94569648EC50E06FEF95
:101C40007FEFCE010196E8DCCE0101960E944D9413
:101C500063E779E0CE0101960E94569640ED57E089
:101C60006FEF7FEFCE010196A2DDCE0101960E94BB
:101C70004D9480919D0D90919E0D029719F462E60E
:101C800079E002C062E579E0CE0101960E945696A5
:101C900048EC50E06FEF7FEFCE010196BDDCCE0146
:101CA00001960E944D9465E479E0CE0101960E9470
:101CB000569640ED57E06FEF7FEFCE01019677DD4E
:101CC000CE0101960E944D9469E379E0CE01019620
:101CD0000E94569648EC50E06FEF7FEFCE010196E0
:101CE0009BDCCE0101960E944D9469E279E0CE0121
:101CF00001960E94569640ED57E06FEF7FEFCE01C0
:101D0000019655DDCE0101960E944D946EE179E079
:101D1000CE0101960E94569648EC50E06FEF7FEF9F
:101D2000CE01019679DCCE0101960E944D9464E1CA
:101D300079E0CE0101960E94569640ED57E06FEF94
:101D40007FEFCE01019633DDCE0101960E944D94C6
:101D500064E079E0CE0101960E94569648EC50E08E
:101D60006FEF7FEFCE01019657DCCE0101960E9406
:101D70004D9467EF78E0CE0101960E94569640EDB3
:101D800057E06FEF7FEFCE01019611DDCE01019696
:101D90000E944D946BEE78E0CE0101960E9456961B
:101DA00048EC50E06FEF7FEFCE01019635DCCE01BD
:101DB00001960E944D946BED78E0CE0101960E9451
:101DC000569640ED57E06FEF7FEFCE010196EFDCC6
:101DD000CE0101960E944D942C960FB6F894DEBF6A
:101DE0000FBECDBFDF91CF9108954F925F926F925A
:101DF0007F928F929F92AF92BF92CF92DF92EF929B
:101E0000FF92CF93DF93CDB7DEB72C970FB6F89440
:101E1000DEBF0FBECDBF92DD8CEA9CE00E9435850F
:101E20002B013C018CEA9CE00E94C7844B015C01C1
:101E3000609138027091390280913A0290913B0290
:101E40000E94FB99AB01BC018CEA9CE00E94D28607
:101E50006B017C01C301B2010E94FB9920E030E0DC
:101E600048EC52E40E942F99AB01BC0122E0CE0164
:101E700001960E94DA95BE016F5F7F4F8EE79CE06E
:101E80000E943F95CE0101960E944D9463EC78E04C
:101E90008EE79CE00E948F966EE77CE084E89CE0F1
:101EA0000E9422956FEB78E0CE0101960E94B894D3
:101EB0006EE77CE0CE0101960E94B196BC018EE7F0
:101EC0009CE00E942295CE0101960E944D9463E30E
:101ED00076E08AE89CE00E94559521E0B501A401D6
:101EE000CE0101960E94DA95BE016F5F7F4F8AE8AE
:101EF0009CE00E948996CE0101960E944D946BE170
:101F000075E08AE89CE00E948F9621E0B701A60167
:101F1000CE0107960E94DA95BE01695F7F4FCE0120
:101F200001960E94379564EF76E0CE0101960E94FB
:101F3000C296BC018AE89CE00E948996CE01019677
:101F40000E944D94CE0107960E944D946EE77CE06E
:101F5000CE0101960E94379562E375E0CE010196AD
:101F60000E94C2966AE87CE00E94B196BC018AE8B1
:101F70009CE00E942295CE0101960E944D9464E857
:101F80007CE0CE0101960E9437954AE050E060E087
:101F900070E0CE01019697DACE0101960E944D9431
:101FA00021E0B501A401CE0101960E94DA95BE019F
:101FB0006F5F7F4F80E99CE00E943F95CE010196C4
:101FC0000E944D9460E97CE0CE0101960E94379515
:101FD0004AE050E06FEF7FEFCE010196E8DBCE01E3
:101FE00001960E944D9465E070E080E090E00E94D0
:101FF000788A61E275E0CE0101960E94B894CE0124
:1020000001967EDCCE0101960E944D9421E0B7013D
:10201000A601CE0107960E94DA95BE01695F7F4F47
:10202000CE0101960E94379564EF76E0CE010196CD
:102030000E94C296BC0180E99CE00E942295CE01DC
:1020400001960E944D94CE0107960E944D9460E93E
:102050007CE0CE0101960E9437954AE050E068EF9F
:102060007FEFCE010196A3DBCE0101960E944D9435
:1020700065E070E080E090E00E94788A80917B0CBF
:10208000882331F068E572E080E090E00E94788A71
:102090002C960FB6F894DEBF0FBECDBFDF91CF9167
:1020A000FF90EF90DF90CF90BF90AF909F908F9078
:1020B0007F906F905F904F900895CF93DF93EC01E6
:1020C0008C819D81892B61F0BE018BE39FE00E9492
:1020D0001E91BE0182E191E1DF91CF910C941E919E
:1020E000DF91CF9108951F93CF93DF93CDB7DEB7E4
:1020F000A8970FB6F894DEBF0FBECDBF182F83ECA4
:102100009CE00E94F27481110EC060E97BE0CE0178
:1021100001960E945696CE010196CFDFCE01019620
:102120000E944D94A3C0BE016F5F7F4F83EC9CE083
:102130000E94D473112309F493C065E67BE08BE31E
:102140009FE00E940E9165E57BE08BE39FE00E949B
:10215000D290BE016F5F7F4F8BE39FE00E942E9174
:1021600065E47BE08BE39FE00E94D2904D855E8525
:102170006F8578892AE030E08BE39FE00E940A9225
:1021800065E37BE08BE39FE00E94D29049895A8906
:102190006B897C892AE030E08BE39FE00E940A9201
:1021A00065E27BE08BE39FE00E94D29020E030E08C
:1021B00040E251E4698D7A8D8B8D9C8D0E948F9BBE
:1021C000AB01BC0122E030E08BE39FE00E9426934C
:1021D00064E375E08BE39FE00E942E9165E17BE074
:1021E0008BE39FE00E94D29020E030E040E251E497
:1021F0006D8D7E8D8F8D98A10E948F9BAB01BC0150
:1022000022E030E08BE39FE00E94269364E375E0D8
:102210008BE39FE00E942E9165E07BE08BE39FE0E3
:102220000E94D29020E030E040E251E469A17AA11E
:102230008BA19CA10E948F9BAB01BC0122E030E0EE
:102240008BE39FE00E94269364E375E08BE39FE0BD
:102250000E942E916FED7AE08BE39FE00E940E9139
:1022600064EF71E080E090E00E94788AA8960FB653
:10227000F894DEBF0FBECDBFDF91CF911F910895BF
:102280004F925F926F927F928F929F92AF92BF9286
:10229000CF92DF92EF92FF920F931F93CF93DF9332
:1022A000CDB7DEB7CA54D1090FB6F894DEBF0FBE62
:1022B000CDBF8C0162E17BE0CE01CD960E94B89447
:1022C00062E17BE0CE01C7960E94B894BE016F5FC9
:1022D0007F4F83EC9CE00E9485754D885E886F88F7
:1022E000788CC98CDA8CEB8CFC8C8D8D9E8DAF8DAF
:1022F000B8A12B968CAF9DAFAEAFBFAF2B97C801E7
:102300000197039708F0E2C1A7019601C301B2014A
:1023100090580E94D8982BED3FE049EC5FE30E9473
:1023200065982091340230913502409136025091E7
:1023300037020E9465984B015C0120E030E0A90162
:102340000E942B9987FD09C08092670C9092680CBF
:10235000A092690CB0926A0C10C02BED3FE049ECE2
:1023600050E4C501B4010E9465986093670C7093B6
:10237000680C8093690C90936A0C8090670C909025
:10238000680CA090690CB0906A0C2BED3FE049EC12
:1023900050E4C501B4010E94D09A181684F42BEDC4
:1023A0003FE049EC50E4C501B4010E946498609399
:1023B000670C7093680C8093690C90936A0C20E012
:1023C00030E044E353E46091670C7091680C8091B5
:1023D000690C90916A0C0E948F9B2BED3FE049E4C1
:1023E00050E40E942F996093630C7093640C809367
:1023F000650C9093660C0E94C8994AE0CE018B96BA
:102400000E94839568E375E0CE0185960E94B8949A
:10241000BE01655D7F4FCE0185960E94B19662E454
:1024200075E00E94C296BC0180E99CE00E94229562
:10243000CE0185960E944D94CE018B960E944D94BC
:102440008090630C9090640CA090650CB090660C2A
:1024500020E030E044EB52E4C501B4010E942B9926
:10246000181694F020E030E040E05FE3C501B401CD
:102470000E9465980E94C8994AE0CE018B960E94FE
:10248000839569E475E023C020E030E044E353E441
:10249000C501B4010E942B991816A4F1A50194015D
:1024A00060E070E884E393E40E9464986093630CB6
:1024B0007093640C8093650C9093660C0E94C8998D
:1024C0004AE0CE018B960E9483956CE475E0CE01C4
:1024D00085960E94B894BE01655D7F4FCE018596BA
:1024E0000E94B196BC01CE01CD960E942295CE01EC
:1024F00085960E944D94CE018B960E944D946DEA74
:1025000076E063C020E030E047E853E4C501B40161
:102510000E942B99181604F120E030E044E353E4C4
:10252000C501B4010E94649820E030E040E05FE320
:102530000E9465986093630C7093640C8093650CA3
:102540009093660C0E94C8994AE0CE018B960E9437
:1025500083956CE475E01FC0A501940160E070E014
:1025600084EB93E40E94649820E030E040E05FE375
:102570000E9465986093630C7093640C8093650C63
:102580009093660C0E94C8994AE0CE018B960E94F7
:10259000839569E475E0CE0185960E94B894BE01EA
:1025A000655D7F4FCE0185960E94B196BC01CE013C
:1025B000CD960E942295CE0185960E944D94CE0123
:1025C0008B960E944D946FE475E0CE01C7960E94F1
:1025D0005595BE01635C7F4FCE0185960E9437956D
:1025E0004AE050E060E070E0CE0185960E94630A08
:1025F000CE0185960E944D940E94498A2091EA045A
:102600003091EB044091EC045091ED0480908B0DDF
:1026100090908C0DA0908D0DB0908E0D280D391DD1
:102620004A1D5B1D261737074807590708F441C2A2
:102630000E94498A0E94F9994B015C016091EA0469
:102640007091EB048091EC049091ED040E94FB9951
:1026500020E030E040E85EE30E948F9B27966CAF5D
:102660007DAF8EAF9FAF279760918B0D70918C0DD2
:1026700080918D0D90918E0D0E94FB999B01AC0174
:1026800027966CAD7DAD8EAD9FAD27970E94659866
:102690009B01AC01C501B4010E942B9987FD09C2C1
:1026A00062E375E0CE0185960E94B894BE01695C34
:1026B0007F4FCE0185960E94B196BC01CE01CD968A
:1026C0000E948996CE0185960E944D94C80102977A
:1026D000029708F0C8C120E030E040E251E4C301B5
:1026E000B2010E948F9B4B015C0120E030E040E290
:1026F00051E4C701B6010E948F9B6B017C0120E071
:1027000030E040E251E42B966CAD7DAD8EAD9FADD7
:102710002B970E948F9B2B013C010E94498A20919C
:10272000DB0B3091DC0B4091DD0B5091DE0B621B1B
:10273000730B840B950B0E94F99920E030E04AE777
:1027400054E40E942F99AB01BC0123E0CE018B968B
:102750000E94DA956AE575E0CE0185960E94B894EC
:10276000BE01655D7F4FCE0185960E94B19660E502
:1027700078E00E94C296BC018EE79CE00E94229500
:10278000CE0185960E944D94CE018B960E944D9469
:102790006EE77CE0CE0185960E94379560E97CE08B
:1027A000CE0185960E94B196BE01635C7F4F0E9468
:1027B000B196BC01CE01CD960E942295CE018596A0
:1027C0000E944D946AEA7AE08AE89CE00E9436967C
:1027D00021E0B501A401CE0185960E94DA95BE01E3
:1027E0006B5D7F4F8AE89CE00E948996CE018596BA
:1027F0000E944D9421E0B301A201CE0185960E9472
:10280000DA9521E0B701A601CE01C1960E94DA95C2
:1028100062E375E0CE018B960E94B894BE016F5CB6
:102820007F4FCE018B960E94B19662E375E00E94C5
:10283000C296BE016B5D7F4F0E94B19661E575E067
:102840000E94C296BC018AE89CE00E948996CE0153
:102850008B960E944D94CE01C1960E944D94CE015C
:1028600085960E944D94A5019401C501B4010E9472
:102870008F9B4B015C01A7019601C701B6010E9425
:102880008F9B9B01AC01C501B4010E9465986B014F
:102890007C01A3019201C301B2010E948F9B9B01A5
:1028A000AC01C701B6010E9465980E94429C6093EA
:1028B0005F0C7093600C8093610C9093620C65E5E3
:1028C00075E08AE89CE00E948F9640915F0C5091E1
:1028D000600C6091610C7091620C21E0CE018B96CE
:1028E0000E94DA95BE01655D7F4FCE0185960E94FC
:1028F000379565E375E0CE0185960E94C296BC01CE
:1029000080E99CE00E942295CE0185960E944D941C
:10291000CE018B960E944D9460E97CE08AE89CE0B1
:102920000E948996C0905F0CD090600CE090610C82
:10293000F090620C20E030E04AE754E4C701B601B1
:102940000E94D09A87FD29C020E030E04AE754E495
:10295000C701B6010E942F99AB01BC0123E0CE0153
:102960008B960E940896BE01655D7F4FCE018596CD
:102970000E94379566E375E0CE0185960E94C29667
:10298000BC0180E99CE00E942295CE0185960E94C0
:102990004D94CE018B960E944D9420E030E64AE69D
:1029A00056E460915F0C7091600C8091610C909185
:1029B000620C0E942B99BE01635C7F4F87FF4FC062
:1029C000CE0185960E94379569E575E0CE01859622
:1029D0000E94C2966AE87CE00E94B196BC018AE837
:1029E0009CE00E942295CE0185960E944D94033072
:1029F000110599F46AE87CE0CE0185960E9437952E
:102A0000CE0185965ADBCE0185960E944D9462E1F7
:102A10007BE08AE89CE00E9455956CE575E0CE016C
:102A20008B960E94B89460E97CE0CE018B960E9460
:102A3000B196BC01CE0185960E9437954AE050E0E0
:102A40006FEF7FEFCE0185960E94D70BCE01859662
:102A50000E944D94CE018B960E944D9404C08AE84A
:102A60009CE00E9422956AE070E080E090E00E9485
:102A7000788ACE01C7960E944D94CE01CD960E94D1
:102A80004D94C65BDF4F0FB6F894DEBF0FBECDBFCF
:102A9000DF91CF911F910F91FF90EF90DF90CF903A
:102AA000BF90AF909F908F907F906F905F904F906E
:102AB000089562E17BE0CE0185960E94B894CE0134
:102AC00085960E94800CCE0185960E944D94BE0191
:102AD000695C7F4F8FE89DE00E94F590E1CD8F9279
:102AE0009F92AF92BF92CF92DF92EF92FF920F939D
:102AF0001F93CF93DF9300D000D0CDB7DEB78C010A
:102B0000C0900A02D0900B02E0900C02F0900D02EF
:102B100020E030E040E450E4C701B6010E94D09AC2
:102B200018166CF420E030E04AEF54E4C701B60117
:102B30000E948F9B0E94C8996B017C0106C080E3B4
:102B4000C82E85E7D82EE12CF12C0E949E0C40E087
:102B500060E08FE89DE00E94DC7F6EEC7AE08FE819
:102B60009DE00E94D29041E060E08FE89DE00E94ED
:102B7000DC7F66EC7AE08FE89DE00E94D29064E60C
:102B800070E080E090E00E94788A0E94498A609319
:102B9000DB0B7093DC0B8093DD0B9093DE0B0E94BC
:102BA000498A8090DB0B9090DC0BA090DD0BB090FD
:102BB000DE0BDC01CB0188199909AA09BB098C1528
:102BC0009D05AE05BF055CF4C8015ADB0E94498A29
:102BD00064E170E080E090E00E94788AE0CF01300C
:102BE000110509F041C06AE87CE084E89CE00E949D
:102BF00022950E949E0C64E87CE0CE0101960E9422
:102C000037954AE050E060E070E0CE0101960E9406
:102C1000630ACE0101960E944D9465EB7AE0CE01E5
:102C200001960E9456964AE050E06FEF7FEFCE018A
:102C300001960E94D70BCE0101960E944D9465E645
:102C400075E0CE0101960E94B8946AE87CE0CE015E
:102C500001960E94B196BC018AE89CE00E942295F0
:102C6000CE0101960E944D9426960FB6F894DEBFD1
:102C70000FBECDBFDF91CF911F910F91FF90EF90CD
:102C8000DF90CF90BF90AF909F908F900895CF929C
:102C9000DF92EF92FF92CF93DF9300D000D0CDB7B9
:102CA000DEB70E949E0C6EE170E080E090E00E9432
:102CB000788A8CEA9CE00E94C7846B017C0164E600
:102CC00070E080E090E00E94788A63E376E08AE832
:102CD0009CE00E94559521E0B701A601CE01019626
:102CE0000E94DA95BE016F5F7F4F8AE89CE00E94E8
:102CF0008996CE0101960E944D946AE87CE0CE014F
:102D000001960E9437954AE050E060E070E0CE0105
:102D100001960E94630ACE0101960E944D940E9482
:102D20006C0C68E775E08AE89CE00E948F96C09280
:102D30006F0CD092700CE092710CF092720C20E04B
:102D400030E040EF51E4C701B6010E94D09A87FD00
:102D500003C06BEA78E054C020E030E040ED51E47D
:102D6000C701B6010E94D09A87FD1FC06BE978E0C9
:102D7000CE0101960E9456964AE050E06FEF7FEF39
:102D8000CE0101960E94D70BCE0101960E944D9470
:102D90008091FA04882331F06CED75E080E090E0DA
:102DA0000E94788A6BE878E02BC020E030E040EBAE
:102DB00051E4C701B6010E94D09A87FD03C06DE7B8
:102DC00078E01EC06EE678E0CE0101960E9456962D
:102DD0004AE050E06FEF7FEFCE0101960E94D70BE3
:102DE000CE0101960E944D948091FA04882331F01F
:102DF0006CED75E080E090E00E94788A60E678E013
:102E0000CE0101960E9456964AE050E06FEF7FEFA8
:102E1000CE0101960E94D70BCE0101960E944D94DF
:102E20006CE271E080E090E00E94788A8091FA0480
:102E3000882331F068EE73E080E090E00E94788AA9
:102E400026960FB6F894DEBF0FBECDBFDF91CF91AF
:102E5000FF90EF90DF90CF900895CF92DF92EF92A6
:102E6000FF92CF93DF93CDB7DEB72C970FB6F894D0
:102E7000DEBF0FBECDBF62E578E0CE0101960E94B5
:102E800056964AE050E06FEF7FEFCE0101960E9428
:102E9000D70BCE0101960E944D946091C6047091AB
:102EA000C70488EE9CE00E940287E12CF12C64E6C6
:102EB00070E080E090E00E94788A6091C604709192
:102EC000C70488EE9CE00E9402872FEFE21AF20A04
:102ED00023E0E216F1045CF32AE0E216F1041CF4AC
:102EE000892B29F703C0892B09F0D4C06091EA0C23
:102EF0007091EB0C882777FD8095982F0E94FB99A5
:102F00006B017C0160936F0C7093700C8093710C5B
:102F10009093720C6091E80C7091E90C882777FD12
:102F20008095982F0E94FB9960936B0C70936C0CAA
:102F300080936D0C90936E0C21E0B701A601CE0139
:102F400007960E94DA9563E376E0CE0101960E942F
:102F5000B894BE01695F7F4FCE0101960E94B19681
:102F6000BC018AE89CE00E942295CE0101960E9455
:102F70004D94CE0107960E944D9440916B0C509158
:102F80006C0C60916D0C70916E0C21E0CE01079677
:102F90000E94DA956BE775E0CE0101960E94B89425
:102FA000BE01695F7F4FCE0101960E94B196BC01C0
:102FB0008AE89CE00E948996CE0101960E944D9479
:102FC000CE0107960E944D9462E276E08AE89CE08A
:102FD0000E948F9662E17BE0CE0101960E94B89438
:102FE00044E150E060E070E0CE0101960E94630A87
:102FF000CE0101960E944D9460916F0C7091700CFF
:103000008091710C9091720C0E94C8994AE0CE0197
:1030100001960E948395BE016F5F7F4F84E89CE01C
:103020000E943F95CE0101960E944D9440E066E0DB
:103030008FE89DE00E94DC7F64E87CE08FE89DE003
:103040000E94F5906FED8FE89DE00E94049161E28F
:1030500075E08FE89DE00E94039160916B0C709188
:103060006C0C80916D0C90916E0C0E94C8994AE096
:1030700050E08FE89DE00E94ED9162E276E08FE8FB
:103080009DE00E94039164E670E080E090E00E9481
:10309000788A18C067E478E0CE0101960E945696BF
:1030A0004AE050E060E070E0CE0101960E94630AC1
:1030B000CE0101960E944D9467E278E08AE89CE098
:1030C0000E9436962C960FB6F894DEBF0FBECDBF89
:1030D000DF91CF91FF90EF90DF90CF900895CF9246
:1030E000DF92EF92FF92CF93DF93CDB7DEB72C97AD
:1030F0000FB6F894DEBF0FBECDBF69E178E0CE0118
:1031000001960E9456964CE251E06FEF7FEFCE01A0
:1031100001960E94D70BCE0101960E944D946091BA
:10312000C6047091C70488EE9CE00E940287E12CDF
:10313000F12C64E670E080E090E00E94788A609173
:10314000C6047091C70488EE9CE00E9402872FEFAE
:10315000E21AF20A23E0E216F1045CF32AE0E21636
:10316000F1041CF4892B29F703C0892B09F057C1FE
:103170006091EA0C7091EB0C882777FD8095982F71
:103180000E94FB996B017C0160936F0C7093700C33
:103190008093710C9093720C6091E80C7091E90C23
:1031A000882777FD8095982F0E94FB9960936B0C80
:1031B00070936C0C80936D0C90936E0C21E0B701B2
:1031C000A601CE0107960E94DA9563E376E0CE0170
:1031D00001960E94B894BE01695F7F4FCE010196AF
:1031E0000E94B196BC018AE89CE00E942295CE0123
:1031F00001960E944D94CE0107960E944D944091F5
:103200006B0C50916C0C60916D0C70916E0C21E008
:10321000CE0107960E94DA956BE775E0CE01019624
:103220000E94B894BE01695F7F4FCE0101960E9453
:10323000B196BC018AE89CE00E948996CE01019675
:103240000E944D94CE0107960E944D9462E276E072
:103250008AE89CE00E948F9662E17BE0CE010196B5
:103260000E94B89444E150E060E070E0CE01019625
:103270000E94630ACE0101960E944D9460916F0CEA
:103280007091700C8091710C9091720C0E94C89991
:103290004AE0CE0101960E948395BE016F5F7F4F89
:1032A00084E89CE00E943F95CE0101960E944D94D7
:1032B00040E066E08FE89DE00E94DC7F64E87CE00F
:1032C0008FE89DE00E94F5906FED8FE89DE00E94F1
:1032D000049161E275E08FE89DE00E9403916091A6
:1032E0006B0C70916C0C80916D0C90916E0C0E9427
:1032F000C8994AE050E08FE89DE00E94ED9162E2BB
:1033000076E08FE89DE00E94039164E670E080E043
:1033100090E00E94788A86E99CE00E943E98C090E6
:103320006F0CD090700CE090710CF090720C20E05B
:1033300030E040EF51E4C701B6010E94D09A87FD0A
:1033400003C06AE078E054C020E030E040ED51E492
:10335000C701B6010E94D09A87FD1FC06AEF77E0CF
:10336000CE0101960E9456964AE050E06FEF7FEF43
:10337000CE0101960E94D70BCE0101960E944D947A
:103380008091FA04882331F06CED75E080E090E0E4
:103390000E94788A6AEE77E02BC020E030E040EBB4
:1033A00051E4C701B6010E94D09A87FD03C06CEDBD
:1033B00077E01EC06DEC77E0CE0101960E94569634
:1033C0004AE050E06FEF7FEFCE0101960E94D70BED
:1033D000CE0101960E944D948091FA04882331F029
:1033E0006CED75E080E090E00E94788A6FEB77E00A
:1033F000CE0101960E9456964AE050E06FEF7FEFB3
:10340000CE0101960E94D70BCE0101960E944D94E9
:1034100062E370E080E090E00E94788A01C037DCCF
:103420002C960FB6F894DEBF0FBECDBFDF91CF91C3
:10343000FF90EF90DF90CF900895CF92DF92EF92C0
:10344000FF921F93CF93DF93CDB7DEB7AA970FB646
:10345000F894DEBF0FBECDBF182F882351F08091A6
:10346000790C882331F062E17BE08BE39FE00E94DE
:103470002E918CEE9CE00E94D579BE016F5F7F4F4C
:103480008CEE9CE00E947579CE010D967C01112393
:1034900091F18091790C882371F168EA77E0C70196
:1034A0000E945696C7010E94370AC7010E944D9498
:1034B000FE0131966F01F601419151916191719137
:1034C0006F0126E030E08BE39FE00E94269362E3E9
:1034D00075E08BE39FE00E940391CE14DF0459F75F
:1034E00062E17BE0C7010E94B894C7010E94370ADD
:1034F000C7010E944D9423E938E144E85FE3698104
:103500007A818B819C810E948F9B6D877E878F87BC
:10351000988B22E430E645E85FE36D817E818F8100
:1035200098850E948F9B698B7A8B8B8B9C8B25E86F
:103530003BEE41E95FE369857A858B859C850E9436
:103540008F9B6D8B7E8B8F8B988FB7018CEE9CE061
:103550000E945579112309F49EC08091790C88232B
:1035600009F499C0B7018CEE9CE00E9475796E0158
:10357000F9E1CF0ED11C6BE977E0C6010E945696A7
:10358000C6010E94370AC6010E944D94F70141917D
:103590005191619171917F0122E030E08BE39FE0D6
:1035A0000E94269362E375E08BE39FE00E94039103
:1035B000EC14FD0459F762E17BE0C7010E94B89466
:1035C000C7010E94370AC7010E944D946E01F5E2BF
:1035D000CF0ED11C9601AE01495D5F4FBE01675D04
:1035E0007F4F8CEE9CE00E94B87A6EE877E08BE328
:1035F0009FE00E94D29069A57AA54AE050E08BE353
:103600009FE00E94ED9162E375E08BE39FE00E94F2
:1036100003916FA178A54AE050E08BE39FE00E9400
:10362000ED9162E375E08BE39FE00E9403916DA151
:103630007EA14AE050E08BE39FE00E94ED9162E1C1
:103640007BE08BE39FE00E942E91B7018CEE9CE023
:103650000E94F67A65E877E08BE39FE00E94D290C3
:10366000F70141915191619171917F012AE030E020
:103670008BE39FE00E94269362E375E08BE39FE07B
:103680000E940391EC14FD0459F762E17BE08BE3A7
:103690009FE00E942E9161E070E08CEE9CE00E9421
:1036A000E9791123A9F08091790C882389F061E7E9
:1036B00077E08BE39FE00E94D2908CEE9CE00E942A
:1036C000407B4AE050E0BC018BE39FE00E94F49114
:1036D00024E030E043E050E062E070E08CEE9CE0FB
:1036E0000E94F679112309F441C08091790C882356
:1036F000E9F165E577E08BE39FE00E94D2909E01BF
:103700002B5D3F4FAE01495D5F4FBE01675D7F4F4F
:103710008CEE9CE00E94527B69A57AA54AE050E0BD
:103720008BE39FE00E94ED9162E375E08BE39FE005
:103730000E9403916FA178A54AE050E08BE39FE0DF
:103740000E94ED9162E375E08BE39FE00E9403919C
:103750006DA17EA14AE050E08BE39FE00E94ED91D5
:1037600062E17BE08BE39FE00E942E9165E070E0D8
:103770008CEE9CE00E94137A1123A9F08091790CC1
:10378000882389F062E477E08BE39FE00E94D29087
:103790008CEE9CE00E94957B4AE050E0BC018BE3FC
:1037A0009FE00E94F49166E070E08CEE9CE00E9445
:1037B000207A1123A9F08091790C882389F06AE29C
:1037C00077E08BE39FE00E94D2908CEE9CE00E9419
:1037D000A77B4AE050E0BC018BE39FE00E94F4919C
:1037E00067E070E08CEE9CE00E94237A1123A9F040
:1037F0008091790C882389F064E177E08BE39FE086
:103800000E94D2908CEE9CE00E94B97B4AE050E08E
:10381000BC018BE39FE00E94F49168E070E08CEEC5
:103820009CE00E94307A1123A9F08091790C8823C2
:1038300089F06CEF76E08BE39FE00E94D2908CEEF3
:103840009CE00E94CB7B4AE050E0BC018BE39FE010
:103850000E94F49169E070E08CEE9CE00E943D7A59
:103860001123A9F08091790C882389F062EE76E02B
:103870008BE39FE00E94D2908CEE9CE00E94DD7B67
:103880004AE050E0BC018BE39FE00E94F4916AE0C3
:1038900070E08CEE9CE00E944A7A1123A9F080919E
:1038A000790C882389F06CEC76E08BE39FE00E9432
:1038B000D2908CEE9CE00E94EF7B4AE050E0BC018D
:1038C0008BE39FE00E94F4916BE070E08CEE9CE053
:1038D0000E94577A1123A9F08091790C882389F0EE
:1038E00063EB76E08BE39FE00E94D2908CEE9CE04D
:1038F0000E94017C4AE050E0BC018BE39FE00E9403
:10390000F4916CE070E08CEE9CE00E94647A1123EC
:1039100009F494C08091790C882309F48FC06BE975
:1039200076E08BE39FE00E94D2908CEE9CE00E94B8
:10393000137C4AE050E0BC018BE39FE00E94F491CD
:1039400064E876E08BE39FE00E94D2908CEE9CE0EE
:103950000E94387D682F70E04AE050E08BE39FE0E2
:103960000E94F4916DE676E08BE39FE00E94D29096
:103970008CEE9CE00E943C7D682F70E04AE050E0B5
:103980008BE39FE00E94F49166E576E08BE39FE095
:103990000E94D2908CEE9CE00E94407D682F70E0E7
:1039A0004AE050E08BE39FE00E94F4916DE376E003
:1039B0008BE39FE00E94D2908CEE9CE00E94447DBD
:1039C000682F70E04AE050E08BE39FE00E94F491A2
:1039D00064E276E08BE39FE00E94D2908CEE9CE064
:1039E0000E94487D682F70E04AE050E08BE39FE042
:1039F0000E94F4916BE076E08BE39FE00E94D2900E
:103A00008CEE9CE00E944C7D682F70E04AE050E014
:103A10008BE39FE00E94F4916AEF75E08BE39FE0F7
:103A20000E94D2908CEE9CE00E94507D682F70E046
:103A30004AE050E08BE39FE00E94F49161E08CEE5D
:103A40009CE00E94ED7C61E08CEE9CE00E94F27CA8
:103A500061E08CEE9CE00E94F77C1123B1F0809134
:103A6000790C882391F061EE75E08BE39FE00E9472
:103A7000D2908CEE9CE00E94547D682F70E04AE06A
:103A800050E08BE39FE00E94F49160E08CEE9CE0BC
:103A90000E94F77C1123B1F08091790C882391F07A
:103AA00067EC75E08BE39FE00E94D2908CEE9CE087
:103AB0000E94547D682F70E04AE050E08BE39FE065
:103AC0000E94F49161E08CEE9CE00E94FC7C11234A
:103AD000B1F08091790C882391F06BEA75E08BE36B
:103AE0009FE00E94D2908CEE9CE00E94587D682F4F
:103AF00070E04AE050E08BE39FE00E94F49160E0C8
:103B00008CEE9CE00E94FC7C1123B1F08091790C3A
:103B1000882391F06EE875E08BE39FE00E94D290DD
:103B20008CEE9CE00E94587D682F70E04AE050E0E7
:103B30008BE39FE00E94F49161E08CEE9CE00E9498
:103B4000017D1123B1F08091790C882391F062E717
:103B500075E08BE39FE00E94D2908CEE9CE00E9487
:103B60005C7D682F70E04AE050E08BE39FE00E94AC
:103B7000F49160E08CEE9CE00E94017D1123B1F095
:103B80008091790C882391F065E575E08BE39FE0E7
:103B90000E94D2908CEE9CE00E945C7D682F70E0C9
:103BA0004AE050E08BE39FE00E94F49161E08CEEEC
:103BB0009CE00E94067D1123B1F08091790C88234E
:103BC00091F069E375E08BE39FE00E94D2908CEE68
:103BD0009CE00E94607D682F70E04AE050E08BE33B
:103BE0009FE00E94F49160E08CEE9CE00E94067DD4
:103BF0001123B1F08091790C882391F06CE175E08C
:103C00008BE39FE00E94D2908CEE9CE00E94607D4E
:103C1000682F70E04AE050E08BE39FE00E94F4914F
:103C200061E08CEE9CE00E94CF7C61E08CEE9CE039
:103C30000E94D47C61E08CEE9CE00E94D97C60E024
:103C40008CEE9CE00E94DE7C60E08CEE9CE00E94AA
:103C5000E37C60E08CEE9CE00E94E87C112309F498
:103C600095C08091790C882309F490C064E075E0D8
:103C70008BE39FE00E94D2908CEE9CE00E94647DDA
:103C8000682F70E04AE050E08BE39FE00E94F491DF
:103C900066EE74E08BE39FE00E94D2908CEE9CE095
:103CA0000E94687D682F70E04AE050E08BE39FE05F
:103CB0000E94F49168EC74E08BE39FE00E94D29044
:103CC0008CEE9CE00E946C7D682F70E04AE050E032
:103CD0008BE39FE00E94F4916FEA74E08BE39FE036
:103CE0000E94D2908CEE9CE00E94707D682F70E064
:103CF0004AE050E08BE39FE00E94F49166E974E0B3
:103D00008BE39FE00E94D2908CEE9CE00E94747D39
:103D1000682F70E04AE050E08BE39FE00E94F4914E
:103D20006DE774E08BE39FE00E94D2908CEE9CE004
:103D30000E94787D682F70E04AE050E08BE39FE0BE
:103D40000E94F4916AE674E08BE39FE00E94D290B7
:103D50008CEE9CE00E947C7D682F70E04AE050E091
:103D60008BE39FE00E94F49165E574E08BE39FE0B4
:103D70000E94D2908CEE9CE00E94807D682F70E0C3
:103D80004AE050E08BE39FE00E94F49160E08CEE0B
:103D90009CE00E940B7D40ED5FE069E470E48CEEF6
:103DA0009CE00E944E7C112309F44EC08091790C56
:103DB000882309F449C061E474E08BE39FE00E942A
:103DC000D2908CEE9CE00E94257CAB01BC0122E0ED
:103DD00030E08BE39FE00E9427936AE274E08BE37C
:103DE0009FE00E94D2908CEE9CE00E94897C4AE089
:103DF00050E0682F8BE39FE00E94269262E174E01E
:103E00008BE39FE00E94D29061E08CEE9CE00E94E8
:103E1000847D682F70E04AE050E08BE39FE00E94D1
:103E2000F49169EF73E08BE39FE00E94D29061E030
:103E30008CEE9CE00E94887D682F70E04AE050E0A4
:103E40008BE39FE00E94F49141E061E08CEE9CE006
:103E50000E94107D1123B9F08091790C882399F08C
:103E600061EE73E08BE39FE00E94D29061E08CEE04
:103E70009CE00E948C7D682F70E04AE050E08BE36C
:103E80009FE00E94F49141E061E08CEE9CE00E9492
:103E9000157D60E08CEE9CE00E94CA7C1123D1F07D
:103EA0008091790C8823B1F06EEC73E08BE39FE096
:103EB0000E94D2908CEE9CE00E94347D682F70E0CE
:103EC0004AE050E08BE39FE00E94F4918CEE9CE08E
:103ED0000E94907DAA960FB6F894DEBF0FBECDBFAC
:103EE000DF91CF911F91FF90EF90DF90CF900895D9
:103EF0002F923F924F925F926F927F928F929F92FA
:103F0000AF92BF92CF92DF92EF92FF920F931F93E7
:103F1000CF93DF93CDB7DEB7C554D1090FB6F89470
:103F2000DEBF0FBECDBF2B013C012DA33EA34FA38F
:103F300058A70E94498A22966CAF7DAF8EAF9FAF83
:103F4000229720E9421621E052066104710434F000
:103F500020E9422E55245394612C712C8DA19EA1F1
:103F6000AFA1B8A580319742A105B1052CF030E191
:103F700027E290E080E004C03DA12EA19FA188A58A
:103F800040917B0C411104C03DA32EA39FA388A7A1
:103F900022966CAD7DAD8EAD9FAD229728EE33E0BD
:103FA00040E050E00E94F49C26962CAF3DAF4EAF0F
:103FB0005FAF2697F1E0FDAB19A61AA61BA61CA6BB
:103FC0008E01035F1F4F22273327A90124193509CA
:103FD0004609570929AB3AAB4BAB5CAB29A53AA5CF
:103FE0004BA55CA58DA19EA1AFA1B8A52817390747
:103FF0004A075B070CF035C369A57AA58BA59CA57C
:104000000E94FB9920E030E04AE754E40E942F9997
:10401000AB01BC0123E0C8010E94DA95B80184E835
:104020009CE00E943F95C8010E944D948DA19EA1E5
:10403000AFA1B8A50A97A105B10594F42AE0269688
:104040004CAD5DAD6EAD7FAD2697C8010E94AE95BB
:10405000B80184E89CE00E943F95C8010E944D94FD
:10406000BE016F5F7F4F8CEE9CE00E94F67A61ECA0
:1040700073E08AE89CE00E943696DE0111961D01ED
:10408000C12CD12C7601F10181909190A190B19039
:104090001F01A5019401C501B4010E948F9B9B01E2
:1040A000AC01C701B6010E9465986B017C0123E059
:1040B000B501A401CE0143960E940896BE016D5E33
:1040C0007F4FC8010E94379562E375E0C8010E94E6
:1040D000C296BC018AE89CE00E948996C8010E94B1
:1040E0004D94CE0143960E944D942016310659F608
:1040F000C701B6010E94429C6B017C01FDE24F1694
:10410000F1E05F066104710444F00E949E0C40E0FF
:1041100060E08FE89DE00E94DC7F23E0B701A6010C
:10412000C8010E94DA9569E575E0CE0143960E94C8
:10413000B89464E87CE0CE0143960E94B19661E8B1
:1041400075E00E94C296B8010E94B19666E875E0DB
:104150000E94C296BC018AE89CE00E948996CE012A
:1041600043960E944D94C8010E944D942DEC3CEC66
:104170004CE45FE3C701B6010E94D09A29813A81DD
:104180004B815C812DA73EA74FA758AB18160CF0AA
:10419000ACC12AE939E949E95FE3C701B6010E94E8
:1041A0002B9987FFA2C13DA9332309F49EC18984BD
:1041B0009A84AB84BC8420E030E0A901C501B4013D
:1041C0000E942B99CD80DE80EF80F884882309F14E
:1041D0002DA53EA54FA558A9CA01B9010E948F9BE4
:1041E0006EAB7FAB88AF99AFA7019601C701B6014F
:1041F0000E948F9B9B01AC016EA97FA988AD99ADF0
:104200000E9465980E94429CA50194010E94D89842
:1042100004C06BED7FE089EC9FE320EE3EE245E6D3
:1042200052E40E948F9B6EAB7FAB88AF99AF20E0CA
:1042300030E0A901C701B6010E942B99882309F13A
:104240002DA53EA54FA558A9CA01B9010E948F9B73
:104250006AAF7BAF8CAF9DAFA5019401C501B401DE
:104260000E948F9B9B01AC016AAD7BAD8CAD9DAD77
:104270000E9465980E94429CA70196010E94D898CE
:1042800004C06BED7FE089EC9FE320EE3EE245E663
:1042900052E40E948F9B6AAF7BAF8CAF9DAF20E052
:1042A00030E0A9016DA57EA58FA598A90E942B9944
:1042B0008823F9F0A5019401C501B4010E948F9BE8
:1042C0004B015C01A7019601C701B6010E948F9BBB
:1042D0009B01AC01C501B4010E9465980E94429CFB
:1042E0002DA53EA54FA558A90E94D8986B017C0129
:1042F00008C09BEDC92E9FE0D92E99ECE92E9FE3D3
:10430000F92E6AE575E0C8010E94B89464E87CE083
:10431000C8010E94B19669E875E00E94C296BC018E
:104320008AE89CE00E942295C8010E944D946AE5AB
:1043300075E0C8010E94B89464E87CE0C8010E945E
:10434000B19663EA75E00E94C296BC0184E89CE0E5
:104350000E942295C8010E944D9421E04EA95FA9B8
:1043600068AD79ADC8010E94DA9521E04AAD5BAD38
:104370006CAD7DADCE0143960E94DA9520EE3EE213
:1043800045E652E4C701B6010E948F9BAB01BC0118
:1043900021E0CE014F960E94DA95BE01615E7F4F0B
:1043A000CE0149960E94379562E375E0CE014996A9
:1043B0000E94C296BE016D5E7F4F0E94B19662E37D
:1043C00075E00E94C296B8010E94B196BC018EE7CA
:1043D0009CE00E942295CE0149960E944D94CE0108
:1043E0004F960E944D94CE0143960E944D94C80171
:1043F0000E944D944DE2441641E05406610471045C
:1044000074F469A57AA58BA59CA525E030E040E071
:1044100050E00E94F49C672B682B692BC1F564E87F
:104420007CE0C8010E94379545E050E06FEF7FEFD8
:10443000C8010E940C0BC8010E944D946CEA75E003
:10444000C8010E94B89445E050E061EF7FEFC801D9
:104450000E94630AC8010E944D9462E17BE0C8019A
:104460000E94B894C8010E94800CC8010E944D941B
:104470006EE77CE0C8010E94379545E050E060E0BF
:1044800070E0C8010E94D70BC8010E944D946EE7EE
:104490007CE08AE89CE00E9489965FE14516510421
:1044A0006104710434F489A59AA5ABA5BCA5B7FD38
:1044B00011C06AE87CE0C8010E943795C8010E94DB
:1044C0005D10C8010E944D9462E17BE08AE89CE0A7
:1044D0000E945595B201C30177FE04C069A97AA96B
:1044E0008BA99CA90E94788AA9C023E04DA55EA54E
:1044F0006FA578A9C8010E94DA956AE575E0CE013A
:1045000043960E94B89464E87CE0CE0143960E94F2
:10451000B1966EEA75E00E94C296B8010E94B1960B
:1045200067E875E00E94C296BC0184E89CE00E94A6
:104530002295CE0143960E944D94C8010E944D944D
:1045400049855A856B857C8523E0C8010E940896C1
:104550004D815E816F81788523E0CE0149960E946E
:104560000896BE01675E7F4FCE0143960E94379545
:1045700063EB75E0CE0143960E94C296B8010E949B
:10458000B19667E875E00E94C296BC018EE79CE098
:104590000E942295CE0143960E944D94CE014996E9
:1045A0000E944D94C8010E944D949DE2491691E0ED
:1045B00059066104710474F469A57AA58BA59CA5BC
:1045C00025E030E040E050E00E94F49C672B682B2F
:1045D000692BF1F464E87CE0C8010E9437954AE059
:1045E00050E06FEF7FEFC8010E940C0BC8010E94E2
:1045F0004D946EE77CE0C8010E9437954AE050E098
:1046000060E070E0C8010E94D70BC8010E944D9481
:104610006AE87CE0C8010E943795C8010E945D10DD
:10462000C8010E944D9462E17BE08AE89CE00E9410
:104630005595C301B2010E94788A1DAA0E94498A39
:104640009B01AC0122968CAD9DADAEADBFAD229766
:10465000281B390B4A0B5B0B29A73AA74BA75CA772
:10466000BDCC64E87CE0CE010D960E9437954AE00F
:1046700050E06FEF7FEFCE010D960E94630ACE01EE
:104680000D960E944D949DA99923B1F16CEA75E0B5
:10469000CE010D960E94B89445E050E061EF7FEFA7
:1046A000CE010D960E94630ACE010D960E944D9494
:1046B00080917B0C882391F069EB73E0CE010D961D
:1046C0000E94569645E050E060E070E0CE010D9605
:1046D0000E94630ACE010D960E944D9462E17BE038
:1046E000CE010D960E94B894CE010D960E94800CCA
:1046F000CE010D960E944D946EE77CE0CE010D96A2
:104700000E9437954AE050E06FEF7FEFCE010D96A3
:104710000E94D70BCE010D960E944D94CB5BDF4FCC
:104720000FB6F894DEBF0FBECDBFDF91CF911F91C2
:104730000F91FF90EF90DF90CF90BF90AF909F9040
:104740008F907F906F905F904F903F902F90089543
:104750008F929F92AF92BF92CF92DF92EF92FF9291
:104760000F931F93CF93DF93CDB7DEB72C970FB680
:10477000F894DEBF0FBECDBF67E773E084E89CE02E
:104780000E94369664E87CE0CE0101960E9437953F
:1047900044E150E060E070E0CE0101960E94630ABF
:1047A000CE0101960E944D9468E673E084E89CE097
:1047B0000E94369664E87CE0CE0101960E9437950F
:1047C00044E150E06FEF7FEFCE0101960E94D70BDE
:1047D000CE0101960E944D9482E79DE00E94FB89E4
:1047E0004B015C0182E79DE00E94FD896B017C0129
:1047F00004E010E020E030E048EC52E4C701B601EC
:104800000E94D09A18168CF40150110909F4D7C0EF
:1048100064E670E080E090E00E94788A82E79DE0A4
:104820000E94FD896B017C01E5CF21E0B501A40167
:10483000CE0107960E94DA9568EC75E0CE010196EC
:104840000E94B894BE01695F7F4FCE0101960E941D
:10485000B196BC018AE89CE00E942295CE010196A7
:104860000E944D94CE0107960E944D946AE87CE028
:10487000CE0101960E94379542E350E06FEF7FEF43
:10488000CE0101960E94D70BCE0101960E944D9455
:1048900069E775E0CE0101960E94B894CE010196B9
:1048A0000E94800CCE0101960E944D9468E775E04D
:1048B0008AE89CE00E948F9621E0B701A601CE0114
:1048C00007960E94DA9563E376E0CE0101960E9496
:1048D000B894BE01695F7F4FCE0101960E94B196E8
:1048E000BC0180E99CE00E942295CE0101960E94C5
:1048F0004D94CE0107960E944D9462E375E0CE017F
:1049000001960E94B89460E97CE0CE0101960E9475
:10491000B196BC0184E89CE00E942295CE010196EC
:104920000E944D9464E87CE0CE0101960E94379588
:104930004AE050E060E070E0CE0101960E940C0B6E
:10494000CE0101960E944D9469E775E0CE01019673
:104950000E94B894CE0101960E94800CCE0101966F
:104960000E944D9468E775E080E99CE00E948F9674
:1049700060E97CE0CE0101960E94379562E375E024
:10498000CE0101960E94C2966AE87CE00E94B19630
:10499000BC018AE89CE00E942295CE0101960E940B
:1049A0004D9480919D0D90919E0D039709F044C008
:1049B00084E090E090939E0D80939D0D3DC06DE549
:1049C00073E084E89CE00E94369664E87CE0CE01C7
:1049D00001960E9437954AE050E060E070E0CE0119
:1049E00001960E94630ACE0101960E944D9466EBE7
:1049F00075E0CE0101960E94B89464E87CE0CE0197
:104A000001960E94B196BC018AE89CE00E94229522
:104A1000CE0101960E944D9480919D0D90919E0D26
:104A2000049721F410929E0D10929D0D81E090E06C
:104A30009093E3048093E20464E670E080E090E009
:104A40000E94788A80917B0C882331F060E273E0C9
:104A500080E090E00E94788A2C960FB6F894DEBF32
:104A60000FBECDBFDF91CF911F910F91FF90EF90BF
:104A7000DF90CF90BF90AF909F908F900895CF928E
:104A8000DF92EF92FF920F931F93CF93DF93CDB7F7
:104A9000DEB72C970FB6F894DEBF0FBECDBF809166
:104AA0007B0C811102C00E949E0C8091E2049091C7
:104AB000E304029741F080919D0D90919E0D009727
:104AC00021F0039711F044DE9DC185E790E10E943B
:104AD000B78D64E670E080E090E00E94788A6DE92E
:104AE00073E084E89CE00E94369664E87CE0CE01A6
:104AF00001960E94379544E150E060E070E0CE01FD
:104B000001960E94630ACE0101960E944D946EE8C0
:104B100073E084E89CE00E94369664E87CE0CE0175
:104B200001960E94379544E150E06FEF7FEFCE0190
:104B300001960E94D70BCE0101960E944D9460E031
:104B400070E08FE69DE00E94FA7E6B017C0104E03C
:104B500010E0A7019601C701B6010E94839C88233B
:104B600009F442C00150110909F02EC163E873E055
:104B700084E89CE00E94369664E87CE0CE010196D1
:104B80000E9437954AE050E060E070E0CE01019667
:104B90000E94630ACE0101960E944D9466EB75E077
:104BA000CE0101960E94B89464E87CE0CE010196A3
:104BB0000E94B196BC018AE89CE00E942295CE0139
:104BC00001960E944D9480919D0D90919E0D0397AA
:104BD00021F410929E0D10929D0D82E090E0909332
:104BE000E3048093E204DFC021E0B701A601CE0117
:104BF00007960E94DA9568EC75E0CE0101960E9456
:104C0000B894BE01695F7F4FCE0101960E94B196B4
:104C1000BC018AE89CE00E942295CE0101960E9488
:104C20004D94CE0107960E944D946AE87CE0CE0137
:104C300001960E94379542E350E06FEF7FEFCE017F
:104C400001960E94D70BCE0101960E944D9469E710
:104C500075E0CE0101960E94B894CE0101960E94A3
:104C6000800CCE0101960E944D9468E775E08AE8B9
:104C70009CE00E948F9660E070E08FE69DE00E94CD
:104C8000F87E6B017C0104E010E0A7019601C701EA
:104C9000B6010E94839C882359F00150110909F044
:104CA000A2C062E17BE080E99CE00E9455955CC077
:104CB00021E0B701A601CE0107960E94DA9563E3D1
:104CC00076E0CE0101960E94B894BE01695F7F4FE5
:104CD000CE0101960E94B196BC0180E99CE00E9441
:104CE0002295CE0101960E944D94CE0107960E9416
:104CF0004D9462E375E0CE0101960E94B89460E99C
:104D00007CE0CE0101960E94B196BC0184E89CE053
:104D10000E942295CE0101960E944D9464E87CE0A9
:104D2000CE0101960E9437954AE050E06FEF7FEF89
:104D3000CE0101960E940C0BCE0101960E944D946B
:104D400069E775E0CE0101960E94B894CE01019604
:104D50000E94800CCE0101960E944D9468E775E098
:104D600080E99CE00E948F9660E97CE0CE0101968C
:104D70000E94379562E375E0CE0101960E94C296CB
:104D80006AE87CE00E94B196BC018AE89CE00E943F
:104D90002295CE0101960E944D9483E090E090937D
:104DA0009E0D80939D0D64E670E080E090E00E948F
:104DB000788A80917B0C882329F160E273E080E09F
:104DC00090E00E94788A1EC068EC70E080E090E07D
:104DD0000E94788A60E070E08FE69DE00E94FA7E93
:104DE0006B017C01B6CE68EC70E080E090E00E9440
:104DF000788A60E070E08FE69DE00E94F87E6B01AB
:104E00007C0143CF2C960FB6F894DEBF0FBECDBF0A
:104E1000DF91CF911F910F91FF90EF90DF90CF9096
:104E200008951F93CF93DF93182FCFE0DCE0812FFD
:104E30000E940E8B899399936CE370E080E090E080
:104E40000E94788A8CE0CF35D80789F768E270E055
:104E50008FE09CE00E945D0820E030E040EA50E4F2
:104E60000E948F9B20E030E040E85AE30E948F9B35
:104E7000DF91CF911F9108954F925F926F927F9231
:104E80008F929F92AF92BF92CF92DF92EF92FF925A
:104E90000F931F93CF93DF93CDB7DEB764970FB611
:104EA000F894DEBF0FBECDBF7C018B0161ED75E0D4
:104EB00084E89CE00E9455950E949E0C64E87CE08A
:104EC000CE0101960E9437954AE050E06FEF7FEFE8
:104ED000CE0101960E94630ACE0101960E944D9474
:104EE000C7019FDF698B7A8B8B8B9C8B40901A025A
:104EF00050901B0260901C0270901D02A301920151
:104F00006091160270911702809118029091190217
:104F10000E9464984B015C0120E030E0A9010E94EE
:104F20002B99882309F451C0C0902202D09023020B
:104F3000E0902402F090250220E030E0A901C701B2
:104F4000B6010E942B9918160CF03FC080911E02EA
:104F500090911F02A0912002B09121028D879E871F
:104F6000AF87B88B9C01AD01C701B6010E942B9998
:104F7000882359F1A70196016D857E858F859889D3
:104F80000E942F990E941C9B6D877E878F87988B2C
:104F9000A301920169897A898B899C890E9464980E
:104FA000A50194010E942F992D853E854F85588932
:104FB0000E948F9B0E949C999B01AC01C701B60186
:104FC0000E948F9B6B017C0103C0C12CD12C760108
:104FD00064E87CE0CE0101960E9437954AE050E0FB
:104FE00060E070E0CE0101960E94630ACE01019656
:104FF0000E944D9420E030E64AEE56E4C701B60127
:105000000E94D09A18163CF46EE473E08AE89CE0A3
:105010000E94369644C001151105B9F421E0B7018C
:10502000A601CE0107960E94DA956BED75E0CE01E0
:1050300001960E94B894BE01695F7F4FCE01019630
:105040000E94B1966FED75E01BC00230110539F575
:1050500022E049895A896B897C89CE0107960E9492
:10506000DA956BED75E0CE0101960E94B894BE0111
:10507000695F7F4FCE0101960E94B19663EE75E0A5
:105080000E94C296BC018AE89CE00E942295CE0153
:1050900001960E944D94CE0107960E944D946AE8B5
:1050A0007CE0CE0101960E9437954AE050E06FEF18
:1050B0007FEFCE0101960E94D70BCE0101960E9490
:1050C0004D9464E670E080E090E00E94788A8091E0
:1050D0007B0C882331F060E273E080E090E00E9476
:1050E000788A64960FB6F894DEBF0FBECDBFDF910D
:1050F000CF911F910F91FF90EF90DF90CF90BF90D5
:10510000AF909F908F907F906F905F904F90089599
:105110004F925F926F927F928F929F92AF92BF92C7
:10512000CF92DF92EF92FF92CF93C82F8091380BEE
:1051300081110DC00E94498A60932C0B70932D0B36
:1051400080932E0B90932F0B81E08093380B8091EE
:10515000300B81110DC00E94498A6093280B709317
:10516000290B80932A0B90932B0B81E08093300BBB
:1051700010920E0C10920D0CE0900D0CF0900E0C95
:1051800088E2E816F1040CF08AC08C2F0E940E8B86
:10519000F701EE0FFF1FE15FF34F9183808368E219
:1051A00070E08FE09CE00E945D0820E030E040EA83
:1051B00050E40E948F9B20E030E040E85AE30E94D8
:1051C0008F9B6B017C016093240B7093250B809364
:1051D000260B9093270B40902A0250902B02609050
:1051E0002C0270902D02A301920160912602709111
:1051F000270280912802909129020E9464989B01C5
:10520000AC0160E070E080EC90E40E9464984B0197
:105210005C0120E030E0A9010E942B9920E030E001
:1052200040E650E4811105C0C701B6010E948F9B82
:105230001EC0C701B6010E948F9BA30192010E946C
:10524000659820E030E040E850E40E946498A501B1
:1052500094010E942F9920E030E040EC50E40E943D
:105260008F9B20E030E040E850E40E946598609316
:10527000200B7093210B8093220B9093230B64E1FE
:1052800070E080E090E00E94788A80910D0C90910F
:105290000E0C019690930E0C80930D0C6DCF6091C7
:1052A000200B7091210B8091220B9091230BCF91B9
:1052B000FF90EF90DF90CF90BF90AF909F908F9036
:1052C0007F906F905F904F900895CF92DF92EF9212
:1052D000FF92CF93DF93CDB7DEB72C970FB6F8943C
:1052E000DEBF0FBECDBF65E473E084E89CE00E94A2
:1052F000369664E87CE0CE0101960E9437954AE03C
:1053000050E060E070E0CE0101960E94630ACE0199
:1053100001960E944D948091810290918202F8DE64
:105320006B017C0120E030E0A9010E94D09A87FD4A
:1053300022C022E0B701A601CE0107960E94DA95AD
:1053400065EE75E0CE0101960E94B894BE01695FDA
:105350007F4FCE0101960E94B196BC018AE89CE085
:105360000E942295CE0101960E944D94CE0107968F
:105370000E944D9406C066E373E08AE89CE00E94B8
:1053800036966AE87CE0CE0101960E9437954AE0A5
:1053900050E06FEF7FEFCE0101960E94D70BCE0158
:1053A00001960E944D942C960FB6F894DEBF0FBE66
:1053B000CDBFDF91CF91FF90EF90DF90CF90089518
:1053C0002F923F924F925F926F927F928F929F9215
:1053D000AF92BF92CF92DF92EF92FF920F931F9303
:1053E000CF93DF9300D01F92CDB7DEB76B017C0166
:1053F0005A8349835901FA012081318142815381C5
:105400000E942B99181614F0F50183C010E001508A
:10541000104C000F111F000F111FE981FA81E00FDE
:10542000F11F2081318142815381C701B6010E9461
:10543000D09A87FF6BC011E0612E712C4301880C5C
:10544000991C880C991CE981FA81E80DF91D2080CE
:10545000318042805380A2019101C701B6010E94B0
:10546000D09A181614F41F5FE7CFA2019101C7016B
:10547000B6010E942B998501080D191D811102C0EA
:10548000F80147C0C3018150904C880F991F880FC5
:10549000991FA981BA81A80FB91F2D913D914D91F6
:1054A0005C9129833A834B835C83F501E80FF91FF4
:1054B00080809180A280B380C701B6010E94649869
:1054C0006B017C01A5019401F801608171818281E9
:1054D00093810E9464989B01AC01C701B6010E94B0
:1054E0008F9B6B017C0129813A814B815C81C201D8
:1054F000B1010E9464989B01AC01C701B6010E94F2
:105500002F99A50194010E94659807C0F501E00F4D
:10551000F11F60817181828193810F900F900F90B4
:105520000F90DF91CF911F910F91FF90EF90DF903F
:10553000CF90BF90AF909F908F907F906F905F9033
:105540004F903F902F900895CF92DF92EF92FF926D
:105550001F93CF93DF93182FCAE0D0E0C12CD12C3A
:105560007601812F0E940E8BBC01882777FD8095E4
:10557000982F0E94FB999B01AC01C701B6010E94C4
:1055800065986B017C0162E370E080E090E00E942E
:10559000788A219731F720E030E040E251E4C701FA
:1055A000B6010E942F9920E030E040EA50E40E94CA
:1055B0008F9B20E030E040E85AE30E948F9BDF9110
:1055C000CF911F91FF90EF90DF90CF900895FC0155
:1055D00020E030E0772767FD7095AB01425051091C
:1055E000DF01A81BB90BA417B50724F4A1912A0F5A
:1055F000311DF6CFA9014E5B5F4F860F971FFC014F
:105600003297208130E0322F222731968081280F77
:10561000311D81E04217530709F080E00895FF92A1
:105620000F931F93CF93DF93F82E0AE010E0C0E0B2
:10563000D0E08F2D0E940E8BC80FD91F65E070E05F
:1056400080E090E00E94788A0150110991F7CE0124
:105650006AE070E00E94AB9CCB01DF91CF911F917B
:105660000F91FF9008950F931F93CF93DF93CDB7C2
:10567000DEB72E970FB6F894DEBF0FBECDBF8D8775
:105680009E870E949E0C8D859E85C9DF8C0162E3FA
:1056900070E080E090E00E94788AB801882777FD6A
:1056A0008095982F0E94FB9920E030E040EA50E47A
:1056B0000E948F9B20E030EC4FE754E40E942F992A
:1056C000AB01BC0123E0CE0107960E94DA9567EF9B
:1056D00076E0CE0101960E94B894BE01695F7F4FCB
:1056E000CE0101960E94B19664EF75E00E94C296C9
:1056F000BC018AE89CE00E942295CE0101960E949E
:105700004D94CE0107960E944D9467EF75E084E8B2
:105710009CE00E94559564E87CE0CE0101960E94D1
:1057200037954AE050E068E070E0CE0101960E94B3
:10573000630ACE0101960E944D946AE87CE0CE0196
:1057400001960E9437954AE050E06FEF7FEFCE015F
:1057500001960E94D70BCE0101960E944D9464E8F9
:105760007CE08AE89CE00E94899680917B0C8823EB
:1057700031F060E273E080E090E00E94788A2E963B
:105780000FB6F894DEBF0FBECDBFDF91CF911F9152
:105790000F910895CF93DF93CDB7DEB72C970FB657
:1057A000F894DEBF0FBECDBF3ADF9093740C8093A8
:1057B000730C62E370E080E090E00E94788A609170
:1057C000730C7091740C4AE0CE0101960E9483958F
:1057D000BE016F5F7F4F8AE89CE00E943F95CE013B
:1057E00001960E944D948091E60C9091E70C892BD4
:1057F00009F45FC062EE7CE0CE0107960E94379507
:10580000BE01695F7F4FCE0101960E94379544E14A
:1058100050E060E070E0CE0101960E94630ACE0184
:1058200001960E944D946FEF75E0CE0101960E94A3
:10583000B8946AE87CE0CE0101960E94B196BC0162
:1058400084E89CE00E942295CE0101960E944D942E
:1058500064E87CE0CE0101960E94379544E150E077
:105860006FEF7FEFCE0101960E94D70BCE0101961C
:105870000E944D94BE01695F7F4FCE0101960E9448
:10588000379562E375E0CE0101960E94C29664E806
:105890007CE00E94B196BC018AE89CE00E942295BF
:1058A000CE0101960E944D94CE0107960E944D9420
:1058B00054C06AE076E084E89CE00E94559564E874
:1058C0007CE0CE0101960E94379544E150E060E013
:1058D00070E0CE0101960E94630ACE0101960E94FB
:1058E0004D946EE076E0CE0101960E94B8946AE88D
:1058F0007CE0CE0101960E94B196BC0184E89CE058
:105900000E942295CE0101960E944D9464E87CE0AD
:10591000CE0101960E94379544E150E06FEF7FEF92
:10592000CE0101960E94D70BCE0101960E944D94A4
:105930006FEF75E0CE0101960E94B8946AE87CE0B2
:10594000CE0101960E94B196BC018AE89CE00E94BB
:105950002295CE0101960E944D9480917B0C882364
:1059600031F060E273E080E090E00E94788A2C964B
:105970000FB6F894DEBF0FBECDBFDF91CF91089573
:105980000F931F93CF93DF93CDB7DEB72C970FB64E
:10599000F894DEBF0FBECDBF8C0181E00E940B8B5F
:1059A00064E670E080E090E00E94788A0E949E0C9D
:1059B000C80135DE60E074E0681B790B4AE0CE0177
:1059C00007960E9483956EE076E0CE0101960E94D4
:1059D000B894BE01695F7F4FCE0101960E94B196D7
:1059E000BC018AE89CE00E942295CE0101960E94AB
:1059F0004D94CE0107960E944D9440E066E08FE8FA
:105A00009DE00E94DC7F66EB77E0CE0101960E946C
:105A1000569642E350E068E070E0CE0101960E94A5
:105A2000630ACE0101960E944D946AE87CE0CE01A3
:105A300001960E94379542E350E06FEF7FEFCE0171
:105A400001960E94D70BCE0101960E944D9465E10C
:105A500076E0CE0101960E94B8946AE87CE0CE011F
:105A600001960E94B196BC018AE89CE00E942295B2
:105A7000CE0101960E944D9480917B0C882331F0D9
:105A800060E273E080E090E00E94788A2C960FB686
:105A9000F894DEBF0FBECDBFDF91CF911F910F9164
:105AA00008950F9390E0BBDDBC01882777FD8095BA
:105AB000982F0E94FB992DE038E643E55BE30E94B6
:105AC0008F9B06E021E532E049E652E079DC20E0F8
:105AD00030E048EC52E40E948F9B20E030E048EA3E
:105AE00051E40E948F9B20914D0230914E024091D3
:105AF0004F02509150020E942F990F910895CF921A
:105B0000DF92EF92FF92CF93DF93CDB7DEB72C9762
:105B10000FB6F894DEBF0FBECDBFC3DF6B017C01B3
:105B200068EF72E084E89CE00E94369664E87CE0CE
:105B3000CE0101960E94379542E350E060E070E0AC
:105B4000CE0101960E94630ACE0101960E944D94F7
:105B500022E0B701A601CE0107960E94DA956AEE0F
:105B600075E0CE0101960E94B894BE01695F7F4F37
:105B7000CE0101960E94B1966FE176E00E94C29636
:105B8000BC018AE89CE00E942295CE0101960E9409
:105B90004D94CE0107960E944D946AE87CE0CE01B8
:105BA00001960E94379542E350E06FEF7FEFCE0100
:105BB00001960E94D70BCE0101960E944D948091D0
:105BC0007B0C882331F060E273E080E090E00E947B
:105BD000788A2C960FB6F894DEBF0FBECDBFDF914A
:105BE000CF91FF90EF90DF90CF900895CF92DF920A
:105BF000EF92FF920F9390E012DDBC01882777FDB2
:105C00008095982F0E94FB992DE038E643E55BE3F1
:105C10000E948F9B06E021E532E049E652E0D0DBAE
:105C200020E030E048EC52E40E948F9B6B017C0145
:105C300020E030E0A9010E942B99181634F0C12C05
:105C4000D12C48EAE42E41E4F42EC0924D02D092C9
:105C50004E02E0924F02F09250020F91FF90EF90AF
:105C6000DF90CF9008952F923F924F925F926F9264
:105C70007F928F929F92AF92BF92CF92DF92EF92DC
:105C8000FF920F931F93CF93DF9300D01F92CDB756
:105C9000DEB76C0148EA54E086E994E09A83898390
:105CA0000DE91BE0EE24E394F12C66246394712C3F
:105CB000E2E12E2E312CF3E14F2E512CA0E1AA2E41
:105CC000B12CB1E18B2E912C80919404909195048C
:105CD0008E159F050CF4EDC091E0C916D10431F486
:105CE000F80180819181E981FA8109C0F2E0CF1643
:105CF000D10439F4E981FA8180819181F80191839D
:105D00008083E981FA8180819181009741F4FA01D1
:105D1000808191819093B9048093B80429C0813027
:105D2000910541F4FA01808191819093C704809399
:105D3000C6041EC08230910541F4FA018081918130
:105D40009093C5048093C40413C0039789F4FA01A7
:105D5000808191819093BB048093BA0462E17BE0DF
:105D600082EE9CE04B835C830E9455955C814B8165
:105D7000E981FA8181919191FA83E98384309105D7
:105D800041F4FA0120813181309382022093810213
:105D90002CC08530910541F4FA0120813181309386
:105DA000C3042093C20421C08630910541F4FA0156
:105DB000208131813093BF042093BE0421C08730FD
:105DC000910541F4FA01208131813093BD04209383
:105DD000BC044AC08A30910541F4FA012081318126
:105DE0003093C1042093C0043FC08531910541F434
:105DF000FA01208131813093C9042093C80434C052
:105E00008631910541F4FA01208131813093E50416
:105E10002093E40429C08731910531F5FA012081EE
:105E200031812830310549F4B092E904A092E804A8
:105E30009092E7048092E60417C02730310549F4B8
:105E40003092E9042092E8045092E7044092E6047C
:105E50000BC02630310541F47092E9046092E804E9
:105E60001092E7041092E6049C012B5031092A306D
:105E70003105B8F4FA01208131813093BB042093BD
:105E8000BA04F7E1F89FB001F99F700D11246D5726
:105E90007D4F82EE9CE04B835C830E9455955C8134
:105EA0004B812FEFE21AF20A4E5F5F4F0E5F1F4FDA
:105EB0000BCF0F900F900F900F90DF91CF911F910C
:105EC0000F91FF90EF90DF90CF90BF90AF909F9099
:105ED0008F907F906F905F904F903F902F9008959C
:105EE00081E08093F6048091F704882321F08FE805
:105EF0009DE00C948B7F08958FE89DE00E94877F42
:105F00001092F60408958091F70481110AC081E08F
:105F10008093F7048093F6048FE89DE00E940E8042
:105F20000CC08091F604882341F0E6DF8FE89DE005
:105F30000E9408801092F7040895D2CF4F925F928A
:105F40006F927F92AF92BF92CF92DF92EF92FF92C9
:105F50000F931F93CF93DF93CDB7DEB7EA970FB6BA
:105F6000F894DEBF0FBECDBF182F62E17BE0CE01FB
:105F7000C5960E94B894612FCE0145960E94E9888B
:105F8000BE016B5E7F4FCE0101960E941E70CE0156
:105F900001960E947D71CE0101960E9411736CE002
:105FA000CE0101960E946D72CE0101960E9427706B
:105FB000082F10E00330110509F46FC162E672E0AA
:105FC000CE01C5960E94369662E17BE08AE89CE0AD
:105FD0000E945595BE016B5C7F4FCE0183960E9457
:105FE00037954AE050E060E070E0CE0183960E9471
:105FF000630ACE0183960E944D9441E060E08FE8F1
:106000009DE00E94DC7F63E376E0CE01C5960E94AE
:10601000559583EEA82E8BE0B82ECC24C394D12CBA
:10602000E12CF12CE016F1060CF0EDC06E2DCE0146
:1060300001960E949E73F5012191319141915191F8
:106040005F010E9465982B013C0120E030E04CEF9D
:1060500052EC0E942B9987FF25C04AE0B601CE0181
:1060600089960E94839560E777E0CE0183960E942F
:10607000B894BE01675D7F4FCE0183960E94B196B2
:1060800064E276E00E94C296BC018AE89CE00E942D
:106090008996CE0183960E944D94CE0189960E94E6
:1060A0004D9449C022E0B301A201CE0183960E9423
:1060B000DA954AE0B601CE018F960E94839560E79B
:1060C00077E0CE0189960E94B894BE01615D7F4F52
:1060D000CE0189960E94B19669E278E00E94C2964C
:1060E000BE016D5D7F4F0E94B196BC018EE79CE0C2
:1060F0000E942295CE0189960E944D94CE018F96E2
:106100000E944D94CE0183960E944D946EE77CE0F0
:10611000CE0183960E94379562E375E0CE018396A7
:106120000E94C296BC018AE89CE00E948996CE013A
:1061300083960E944D940130110559F4E114F10445
:1061400009F05AC06AE87CE0CE01C5960E9422950B
:1061500053C00230110511F522E0B301A201CE01B6
:1061600089960E94DA95BE01675D7F4FCE018396C6
:106170000E94379562E375E0CE0183960E94C29635
:10618000BC01CE01C5960E948996CE0183960E94DD
:106190004D94CE0189960E944D942EC06EE77CE00E
:1061A000CE0183960E94379544E150E06FEF7FEF78
:1061B000CE0183960E94D70BCE0183960E944D9408
:1061C00069E775E0CE0183960E94B894CE0183966C
:1061D0000E94800CCE0183960E944D948091F7041A
:1061E000882351F08091F604882331F060ED77E048
:1061F00080E090E00E94788AFFEFEF1AFF0A8FEFAD
:10620000C81AD80A0FCFCE01C5960E94E2978AE835
:106210009CE00E94E29701151105C9F46FE472E059
:106220008AE89CE00E94369664E472E0CE01839690
:106230000E9456964AE050E06FEF7FEFCE018396C2
:106240000E94D70BCE0183960E944D94EEC004307D
:1062500011050CF003C1BE016B5C7F4FCE0183962C
:106260000E9437954AE050E06FEF7FEFCE018396B2
:106270000E94D70BCE0183960E944D9469E775E08A
:10628000CE0183960E94B894CE0183960E94800C22
:10629000CE0183960E944D94E1C060E376E0CE018A
:1062A000C5960E945595BE016B5C7F4FCE018396CB
:1062B0000E9437954AE050E060E070E0CE0183969E
:1062C0000E94630ACE0183960E944D9462E17BE0B6
:1062D0008AE89CE00E9455956AE87CE0CE01C5966C
:1062E0000E94229500E010E0602FCE0101960E94EE
:1062F0009E736B017C0122E0AB01BC01CE01011554
:10630000110569F483960E94DA95BE016D5D7F4F99
:106310008FE89DE00E94F590CE0183961BC0899680
:106320000E94DA95BE01675D7F4FCE0183960E9481
:10633000379562E375E0CE0183960E94C296BC0158
:10634000CE01C5960E948996CE0183960E944D94F7
:10635000CE0189960E944D9422E0B701A601CE019C
:1063600089960E94DA95BE01675D7F4FCE018396C4
:106370000E94379562E375E0CE0183960E94C29633
:10638000BC018AE89CE00E948996CE0183960E9417
:106390004D94CE0189960E944D940F5F1F4F03309C
:1063A000110509F0A1CFCE01C5960E94E297BE016A
:1063B0006B5C7F4FCE0183960E9437954AE050E098
:1063C0006FEF7FEFCE0183960E94D70BCE018396AD
:1063D0000E944D9469E775E0CE0183960E94B894BF
:1063E000CE0183960E94800CCE0183960E944D942C
:1063F0008AE89CE00E94E29766E376E0CE0183960D
:106400000E94B8946AE87CE0CE0183960E94B1961F
:1064100060E476E00E94C296BC018AE89CE00E949B
:106420002295CE0183960E944D94CE01C5960E947E
:106430004D94EA960FB6F894DEBF0FBECDBFDF9144
:10644000CF911F910F91FF90EF90DF90CF90BF9071
:10645000AF907F906F905F904F90089560E476E0EA
:106460008AE89CE00E948F96E0CF8F929F92AF9235
:10647000BF92CF92DF92EF92FF920F931F93CF9331
:10648000DF93CDB7DEB7A2970FB6F894DEBF0FBE8D
:10649000CDBF5C016A017B01122F8091790C8823AA
:1064A000D9F060E372E08BE39FE00E94D2904AE073
:1064B00050E0B5018BE39FE00E94ED9162E375E04F
:1064C0008BE39FE00E94039122E030E0B701A60138
:1064D0008BE39FE00E942793612FCE0145960E9497
:1064E000E988BE016B5E7F4FCE0101960E941E704F
:1064F000CE0101960E947D71CE0101960E9411731A
:106500006CE0CE0101960E946D72CE0101960E9450
:106510002770082F10E00B30110514F00AE010E08E
:106520008BE5A816B10408F44FC0F3EE8F2EFBE004
:106530009F2EC12CD12C7601A12CB12CA016B10616
:10654000BCF46A2DCE0101960E949E739B01AC01A2
:10655000F40161937193819391934F01C701B60147
:106560000E9465986B017C01FFEFAF1ABF0AE6CF6E
:10657000B801882777FD8095982F0E94FB999B0191
:10658000AC01C701B6010E942F996B017C01E3EEBB
:106590008E2EEBE09E2EA12CB12CA016B1060CF095
:1065A00052C0F4012081318142815381C701B6017B
:1065B0000E946498F40161937193819391934F01C8
:1065C000FFEFAF1ABF0AE9CFA114B10439F473EE9B
:1065D000872E7BE0972EA12CB12C1DC00A151B0520
:1065E0000CF0850101501109602FCE0101960E9427
:1065F0009E739B01AC01000F111F000F111F0D5165
:10660000144FC701B6010E946498F801608371833A
:106610008283938318C0A016B106ACF46A2DCE0114
:1066200001960E949E739B01AC01C701B6010E94B6
:106630006498F40161937193819391934F01FFEFFB
:10664000AF1ABF0AE8CFA2960FB6F894DEBF0FBE0E
:10665000CDBFDF91CF911F910F91FF90EF90DF9011
:10666000CF90BF90AF909F908F900895CF93DF937E
:10667000C8EED4E060E088810E94C08B82E090E0A8
:106680000E949E8A61E088810E94C08B8AE090E02F
:106690000E949E8A60E088810E94C08B20E432E4E0
:1066A0004FE050E061E08091E6040E941D8C0E9462
:1066B000F99920E030E048EC52E40E942F992091B3
:1066C000770D3091780D4091790D50917A0D0E949F
:1066D0008F9B20E030E44CE156E40E942F9920E0AB
:1066E00030E040E05FE30E948F9BDF91CF910895FF
:1066F000CF92DF92EF92FF92B9DF6B017C0120E035
:1067000030E040E050E40E94D09A18161CF4AEDF4E
:106710006B017C0120E030E040E050E4C701B601AD
:106720000E94D09A18161CF4A1DF6B017C0120E0B6
:1067300030E040E050E4C701B6010E94D09A18163C
:106740001CF494DF6B017C0120E030E040E050E479
:10675000C701B6010E94D09A18162CF4FF90EF9052
:10676000DF90CF9083CFC701B601FF90EF90DF900D
:10677000CF9008954F925F926F927F928F929F92E7
:10678000AF92BF92CF92DF92EF92FF92CF93DF93BF
:1067900000D01F92CDB7DEB7ABDF9B01AC016983A0
:1067A0003A834B835C830E94558A2B013C016EE146
:1067B00070E080E090E00E94788A9ADF6B017C01B3
:1067C0000E94558A4B015C0184189508A608B708F9
:1067D00029813A814B815C8181ED881687E098069A
:1067E000A104B1040CF43DC0C701B6010E94649835
:1067F0006B017C0120E030E0A9010E94D09A1816BC
:106800005CF426EA3BE944EC5BE3C701B6010E9475
:106810002B9987FF0BC025C026EA3BE944EC5BEBD4
:10682000C701B6010E94D09A1816DCF0C501B40168
:1068300028EE33E040E050E00E94F49CCA01B90128
:106840000E94FB994B015C0120E030E04AE754E4F0
:10685000C701B6010E948F9BA50194010E942F9948
:1068600003C060E070E0CB010F900F900F900F908D
:10687000DF91CF91FF90EF90DF90CF90BF90AF90DE
:106880009F908F907F906F905F904F90089523E33B
:1068900033E948E853E40E942F9920E030E040E8D3
:1068A0005FE30E9465980E94429C26E636EA45EA2C
:1068B00053E40E948F9B6093770D7093780D8093C3
:1068C000790D90937A0D08954F925F926F927F9217
:1068D0008F929F92AF92BF92CF92DF92EF92FF92F0
:1068E000CF93DF93CDB7DEB76C970FB6F894DEBFCA
:1068F0000FBECDBF6B017C010E94498A6D8B7E8BE0
:106900008F8B988F85E790E10E94B78D61E0809131
:10691000E8040E94878B60E08091E6040E94878BE8
:106920008CEA9CE00E94C7846093730D7093740D91
:106930008093750D9093760DAADFDADE6D877E87E2
:106940008F87988B0E94558A698B7A8B8B8B9C8B57
:106950006AE070E080E090E00E94788A63E576E08B
:106960008AE89CE00E94559520E030E04AE754E434
:10697000C701B6010E948F9B698F7A8F8B8F9C8F86
:10698000412C512C3201C12CD12C7601C701B6010A
:106990000E94FB99298D3A8D4B8D5C8D0E942B991D
:1069A00087FF87C10E94498A2D893E894F89588D6A
:1069B000621B730B840B950B0E94F99920E030E069
:1069C0004AE754E40E942F99AB01BC0123E0CE01B9
:1069D00001960E94DA95BE016F5F7F4F84E89CE0CC
:1069E0000E943F95CE0101960E944D9481DE6B017D
:1069F0007C010E94558A4B015C0189899A89AB8987
:106A0000BC89881A990AAA0ABB0A91ED891697E0EF
:106A10009906A104B1040CF441C020E030E0A901C2
:106A2000C701B6010E94D09A18165CF426EA3BE929
:106A300044EC5BE3C701B6010E942B9987FF0BC0B2
:106A40002DC026EA3BE944EC5BEBC701B6010E948E
:106A5000D09A18161CF1C501B40128EE33E040E0CD
:106A600050E00E94F49CCA01B9010E94FB994B01BD
:106A70005C012D853E854F855889C701B6010E946E
:106A8000649820E030E04AE754E40E948F9BA5011F
:106A900094010E942F994B015C0103C0812C912C21
:106AA000540164E87CE0CE0101960E9437956AE7C4
:106AB00076E0CE0101960E94C296BC0184E89CE07B
:106AC0000E942295CE0101960E944D9423E0B701C9
:106AD000A601CE0107960E94DA95BE01695F7F4F3D
:106AE000CE0101960E94379561E776E0CE010196CE
:106AF0000E94C296BC018EE79CE00E942295CE01C6
:106B000001960E944D94CE0107960E944D9422E07A
:106B1000B501A401CE0101960E94DA956AE575E0FF
:106B2000CE0107960E94B89464E87CE0CE010796F7
:106B30000E94B19664E776E00E94C2966EE77CE020
:106B40000E94B1966DE776E00E94C296BE016F5F2B
:106B50007F4F0E94B19668E776E00E94C296BC0122
:106B60008AE89CE00E948996CE0107960E944D9487
:106B7000CE0101960E944D9420E030E0A901C501AC
:106B8000B4010E94D09A87FD06C062E375E08EE7EB
:106B90009CE00E948F9622E0B501A401CE010796E9
:106BA0000E94DA95BE01695F7F4FCE0101960E9477
:106BB000379568E776E0CE0101960E94C296BC0147
:106BC0008EE79CE00E948996CE0101960E944D942A
:106BD000CE0107960E944D946AE87CE0CE010196B2
:106BE0000E943795CE0101960E945D10CE0101965C
:106BF0000E944D94C301B20125E030E040E050E036
:106C00000E94F49C672B682B692B21F569E272E0E6
:106C1000CE0101960E94569645E050E060E070E09B
:106C2000CE0101960E94630ACE0101960E944D9406
:106C30006EE77CE0CE0101960E94379545E050E07A
:106C40006FEF7FEFCE0101960E94D70BCE01019628
:106C50000E944D9462E17BE08AE89CE00E94559599
:106C600065E070E080E090E00E94788A0E94498AA6
:106C70006B017C012D893E894F89588DC21AD30A38
:106C8000E40AF50A35DD6D877E878F87988B0E9431
:106C9000558A698B7A8B8B8B9C8B6AE070E080E0E5
:106CA00090E00E94788A3FEF431A530A630A730AFE
:106CB0006DCE60E08091E8040E94878B6C960FB6E1
:106CC000F894DEBF0FBECDBFDF91CF91FF90EF9064
:106CD000DF90CF90BF90AF909F908F907F906F90FC
:106CE0005F904F9008950F931F93CF93DF93CDB78D
:106CF000DEB72C970FB6F894DEBF0FBECDBF85E789
:106D000090E10E94B78D08EE14E061E0F801808107
:106D10000E94878B60E08091E6040E94878B8CEA5A
:106D20009CE00E94C7846093730D7093740D8093F0
:106D3000750D9093760DABDDDBDCAB01BC0123E080
:106D4000CE0107960E94DA95BE01695F7F4FCE01A2
:106D500001960E94379564EF76E0CE0101960E947D
:106D6000C296BC0184E89CE00E942295CE01019667
:106D70000E944D94CE0107960E944D9465E776E0FF
:106D8000CE0101960E94B89464E87CE0CE010196A1
:106D90000E94B196BC018AE89CE00E942295CE0137
:106DA00001960E944D94E6DCAB01BC0122E0CE01CD
:106DB00007960E94DA95BE01695F7F4FCE0101966A
:106DC0000E94379568E776E0CE0101960E94C29650
:106DD000BC018EE79CE00E942295CE0101960E94A4
:106DE0004D94CE0107960E944D946CE776E0CE015B
:106DF00001960E94B8946EE77CE0CE0101960E9455
:106E0000B196BC018AE89CE00E948996CE01019669
:106E10000E944D9462E375E0CE0101960E94B89401
:106E20006EE77CE0CE0101960E94B196BC0184E839
:106E30009CE00E948996CE0101960E944D9462E2E8
:106E400072E0CE0101960E9456964AE050E060E062
:106E500070E0CE0101960E94630ACE0101960E9465
:106E60004D9464E87CE0CE0101960E94379545E0A0
:106E700050E06FEF7FEFCE0101960E94D70BCE015D
:106E800001960E944D9460E876E08AE89CE00E94BA
:106E90008F9660E0F80180810E94878B2C960FB658
:106EA000F894DEBF0FBECDBFDF91CF911F910F9140
:106EB0000895EF920F9320E044E064E18FE89DE0B5
:106EC0000E94FC7E63E976E081E89DE00E94B89430
:106ED00069E976E08BE79DE00E94B8946AE582E775
:106EE0009DE00E94B88920E141E168E18FE69DE0E4
:106EF0000E94037EA4E0EA2E04E02AEC34E04EEC8B
:106F000054E062ED74E080E09DE00E94B4808CEE7D
:106F10009CE00E94387962E17BE082EE9CE00E9476
:106F2000B8948091BE049091BF049093E10C80933B
:106F3000E00C209141023091420240914302509175
:106F400044026091450270914602809147029091FF
:106F500048020E9464986093DC0C7093DD0C80936F
:106F6000DE0C9093DF0C4FEF5FEFBA0183EC9CE0F7
:106F70000E9421748CEA9CE00E94A98362E17BE07C
:106F800082EA9CE00E94B89462E17BE08CE99CE09C
:106F90000E94B89462E17BE086E99CE00E94B8948C
:106FA00062E17BE080E99CE00E94B89462E17BE0D2
:106FB0008AE89CE00E94B89462E17BE084E89CE06F
:106FC0000E94B89462E17BE08EE79CE00E94B89456
:106FD000609132027091330282E69BE00F91EF9054
:106FE0000C941F668EE79CE00E944D9484E89CE020
:106FF0000E944D948AE89CE00E944D9480E99CE0B8
:107000000E944D9486E99CE00E944D948CE99CE09E
:107010000E944D9482EA9CE00E944D9487E39AE09E
:107020009093C40C8093C30C82EE9CE00E944D941C
:107030008BE79DE00E944D9481E89DE00C944D9477
:107040008F929F92AF92BF92CF92DF92EF92FF9278
:107050000F931F93CF93DF93CDB7DEB72C970FB667
:10706000F894DEBF0FBECDBF61E08091F8040E94AE
:10707000878B61E08091F8040E94C08B8FE89DE0CF
:107080000E940A7F8FE89DE00E9454804EEE54E0FB
:1070900060E08FE89DE00E9415800E949E0C0E9497
:1070A000702F8EED93E090930C0C80930B0C0E944C
:1070B000A2A080939F0D8FED93E00E94A2A08093E9
:1070C000A00D80919F0D9091A00D1816190654F4F3
:1070D0001092FA04019731F41092A00D10929F0DB6
:1070E0000E94130A6AE17DE0CE0101960E94569645
:1070F0004AE050E06FEF7FEFCE0101960E94630AF5
:10710000CE0101960E944D9440E052EC61E070E0A7
:107110008BE39FE00E94C0098091FA04882331F03C
:1071200068EE73E080E090E00E94788A8BE39FE055
:107130000E94628C182F823709F441C110920C0C06
:1071400010920B0C33E6C32E3BE0D32EE12CF12C36
:10715000C7010E94A2A0D6018D936D01BFEFEB1A6B
:10716000FB0AE8E7EE16F10499F78091630B909122
:10717000640BA091650BB091660B85369105A10556
:10718000B1050CF41CC18093380290933902A0938E
:107190003A02B0933B028091670B9091680BA091EB
:1071A000690BB0916A0B8093340290933502A093DF
:1071B0003602B093370280916B0B90916C0BA091CB
:1071C0006D0BB0916E0B80932E0290932F02A093C3
:1071D0003002B09331026FE77BE0CE0101960E944E
:1071E000B894BE016F5F7F4F81E89DE00E943F959C
:1071F000CE0101960E944D9480916F0B9091700B7F
:10720000A091710BB091720B809322029093230294
:10721000A0932402B09325028091730B9091740B7C
:10722000A091750BB091760B80931E0290931F0274
:10723000A0932002B09321028091770B9091780B5C
:10724000A091790BB0917A0B80931A0290931B0254
:10725000A0931C02B0931D0280917B0B90917C0B3C
:10726000A0917D0BB0917E0B809316029093170234
:10727000A0931802B09319028091870B9091880B0C
:10728000A091890BB0918A0B80934502909346029E
:10729000A0934702B093480280918B0B90918C0B86
:1072A000A0918D0BB0918E0B80934102909342027E
:1072B000A0934302B093440280918F0B9091900B66
:1072C000A091910BB091920B8093490290934A0246
:1072D000A0934B02B0934C028091930B9091940B2E
:1072E000A091950BB091960B80933D0290933E0236
:1072F000A0933F02B09340028091970B9091980B1E
:10730000A091990BB0919A0B80934D0290934E02ED
:10731000A0934F02B0935002C090AD0BD090AE0B33
:10732000E090AF0BF090B00BA7019601C701B6013A
:107330000E94839C811108C0C0921202D092130255
:10734000E0921402F09215026091D90B7091DA0B61
:10735000882777FD8095982F0E94FB999B01AC01AF
:107360000E94839C882321F01092DA0B1092D90B93
:1073700091EBA92E9BE0B92E23EE822E2BE0922ECC
:10738000D501CD90DD90ED90FD905D01A7019601B6
:10739000C701B6010E94839C811105C0F401C0821F
:1073A000D182E282F382F4E08F0E911C89EDA8165F
:1073B0008BE0B80629F781E090E00E94332E0EE8BA
:1073C000010F023080F01E3671F08091630B9091B6
:1073D000640BA091650BB091660B85369105A105F4
:1073E000B1050CF045C18091380290913902A0910D
:1073F0003A02B0913B028093630B9093640BA0938D
:10740000650BB093660B8091340290913502A09188
:107410003602B09137028093670B9093680BA0936C
:10742000690BB0936A0B80912E0290912F02A0916C
:107430003002B091310280936B0B90936C0BA09350
:107440006D0BB0936E0B133751F020E030E048E045
:1074500050E06FE77BE081E89DE00E941E978091FD
:10746000220290912302A0912402B09125028093E0
:107470006F0B9093700BA093710BB093720B809174
:107480001E0290911F02A0912002B09121028093D0
:10749000730B9093740BA093750BB093760B809144
:1074A0001A0290911B02A0911C02B0911D028093C0
:1074B000770B9093780BA093790BB0937A0B809114
:1074C000160290911702A0911802B09119028093B0
:1074D0007B0B90937C0BA0937D0BB0937E0B8091E4
:1074E000450290914602A0914702B09148028093D4
:1074F000870B9093880BA093890BB0938A0B809194
:10750000410290914202A0914302B09144028093C3
:107510008B0B90938C0BA0938D0BB0938E0B809163
:10752000490290914A02A0914B02B0914C02809383
:107530008F0B9093900BA093910BB093920B809133
:107540003D0290913E02A0913F02B0914002809393
:10755000930B9093940BA093950BB093960B809103
:107560004D0290914E02A0914F02B0915002809333
:10757000970B9093980BA093990BB0939A0B8091D3
:10758000120290911302A0911402B09115028093FF
:10759000AD0B9093AE0BA093AF0BB093B00BE3EE9B
:1075A000FBE021EB3BE04191519161917191D90157
:1075B0004D935D936D937D939D01BCE0EB30FB0794
:1075C00091F764E07DE0CE0101960E945696CE01CF
:1075D00001960E94370ACE0101960E944D94B4E9AB
:1075E000CB2EB4E0DB2E8BE9A82E8BE0B82EE12C5D
:1075F000F12C80919404909195048E159F0574F15F
:10760000F60180819181D5018D939D935D018091DB
:10761000790C8823E1F065EA76E08BE39FE00E9435
:1076200003914AE050E0B7018BE39FE00E94ED91A7
:1076300062EA76E08BE39FE00E940391F6016081AD
:1076400071814AE050E08BE39FE00E94F491FFEFEC
:10765000EF1AFF0A82E0C80ED11CCBCF023040F4F3
:1076600010920C0C10920B0C80E090E00E94EA0942
:107670008091D90B9091DA0B892B41F440E855E2C7
:1076800060E070E082E191E10E94C0098091D90B35
:107690009091DA0B019741F440E052EC61E070E028
:1076A00082E191E10E94C00964E670E080E090E030
:1076B0000E94788A8091D90B9091DA0B892B09F07E
:1076C000B7C01E3671F08091630B9091640BA0914E
:1076D000650BB091660B85369105A105B1050CF0DF
:1076E000A7C062E17BE0CE0107960E94B89467EAEA
:1076F00076E0CE0101960E94B89461E87DE0CE016B
:1077000001960E94B196BC01CE0107960E94229577
:10771000CE0101960E944D94BE01695F7F4F82E1C8
:1077200091E10E94F59068EB7BE080E090E00E94A0
:10773000788ABE01695F7F4FCE0101960E9437951E
:10774000CE0101960E94370ACE0101960E944D9407
:107750006CE271E080E090E00E94788A4091850DB3
:107760005091860D4250510961E87DE0CE010196AD
:107770000E94B409BE016F5F7F4FCE0107960E9441
:107780003F95CE0101960E944D94BE01695F7F4FE7
:10779000CE0101960E943795BE01695F7F4FCE01F1
:1077A00001960E94B196BC01CE0107960E942295D7
:1077B000CE0101960E944D946FEA76E0CE010196CB
:1077C0000E94B894BE01695F7F4FCE0101960E946E
:1077D000B196BC01CE0107960E942295CE0101967A
:1077E0000E944D94BE01695F7F4F82E191E10E944A
:1077F000F59068EB7BE080E090E00E94788ABE0123
:10780000695F7F4FCE0101960E943795CE010196A8
:107810000E94370ACE0101960E944D946CE271E0FD
:1078200080E090E00E94788ACE0107960E944D94F5
:1078300064E670E080E090E00E94788A82E69BE057
:107840000E94246664EF7CE0CE0101960E94569669
:107850004AE050E06FEF7FEFCE0101960E94630A8D
:10786000CE0101960E944D948091D90B9091DA0B34
:10787000892B09F56CE075E0CE0107960E94B8945B
:1078800061E87DE0CE0107960E94B196BC01CE0171
:1078900001960E9437954AE050E06FEF7FEFCE01EE
:1078A00001960E94D70BCE0101960E944D94CE0105
:1078B00007960E944D948091D90B9091DA0B019715
:1078C00009F560E175E0CE0107960E94B89461E881
:1078D0007DE0CE0107960E94B196BC01CE010196D3
:1078E0000E9437954AE050E06FEF7FEFCE0101969E
:1078F0000E94D70BCE0101960E944D94CE010796AF
:107900000E944D9465EA76E0CE0107960E94B894F5
:1079100061E87DE0CE0107960E94B19666EB76E0C5
:107920000E94C296BC01CE0101960E943795CE01FD
:1079300001960E945D10CE0101960E944D94CE01E9
:1079400007960E944D9464E670E080E090E00E940B
:10795000788A82E79EE00E94987664E670E080E094
:1079600090E00E94788A63E270E082E79EE00E94E5
:10797000AB7661E070E082E79EE00E94C30982E797
:107980009EE00E941F7783E090E090939E0D80938D
:107990009D0D60E070E08FE69DE00E94FA7E6B0135
:1079A0007C0162E370E080E090E00E94788AA701A9
:1079B0009601C701B6010E94839C882309F44CC03C
:1079C00060E070E08FE69DE00E94F87E6B017C0134
:1079D00062E370E080E090E00E94788AA70196015F
:1079E000C701B6010E94839C8823B1F110929E0DBD
:1079F00010929D0D85E790E10E94B78D64E670E0DE
:107A000080E090E00E94788A40E855E260E070E013
:107A100085E790E10E94C00985E790E10E94498CCA
:107A2000892BD1F06AED7CE0CE0101960E9456963A
:107A3000CE0101960E94370ACE0101960E944D9414
:107A400082E090E090939E0D80939D0D64E670E03F
:107A500080E090E00E94788A80919D0D90919E0D2B
:107A6000039779F465EC7CE0CE0101960E9456966E
:107A7000CE0101960E94370ACE0101960E944D94D4
:107A800012C082E79DE00E94FD8920E030E048E4DA
:107A900053E40E942B9987FF06C082E090E0909308
:107AA000E3048093E20463E08CEA9CE00E94698432
:107AB000811111C06FE97CE0CE0101960E945696BB
:107AC000CE0101960E945D10CE0101960E944D9458
:107AD00010923C02A3C06CE87CE08AE89CE00E9423
:107AE000369640E050E0BA018CEA9CE00E9488861D
:107AF0000E94FB9920E030E048EC52E40E942F996C
:107B0000AB01BC0122E0CE0107960E94DA95BE01CE
:107B1000695F7F4FCE0101960E94379563EC78E054
:107B2000CE0101960E94C296BC018AE89CE00E94A8
:107B30008996CE0101960E944D94CE0107960E942F
:107B40004D946AE87CE0CE0101960E943795CE0103
:107B500001960E94370ACE0101960E944D9466E775
:107B60007CE08AE89CE00E94369660913802709131
:107B7000390280913A0290913B020E94FB9920E0E9
:107B800030E048EC52E40E942F99AB01BC0122E0A6
:107B9000CE0107960E94DA95BE01695F7F4FCE0144
:107BA00001960E94379563EC78E0CE0101960E9421
:107BB000C296BC018AE89CE00E948996CE0101969B
:107BC0000E944D94CE0107960E944D946AE87CE095
:107BD000CE0101960E943795CE0101960E94370A88
:107BE000CE0101960E944D94113629F481E00E9445
:107BF0001D1A81E011C08BE39FE00E94628C182F58
:107C000064E670E080E090E00E94788A113671F3BB
:107C100080E00E941D1A80E00E94731064E670E00C
:107C200080E090E00E94788A80919D0D90919E0D59
:107C3000892BE1F485E790E10E94B78D61E08091A6
:107C4000E8040E94878B60E08091E6040E94878BA5
:107C50008CEA9CE00E94C7846093730D7093740D4E
:107C60008093750D9093760D0E9447348091FA04AD
:107C7000882331F068EE73E080E090E00E94788A1B
:107C80006DE477E086E99CE00E94559582E090E003
:107C90009093780C8093770C8091FA0481110E9464
:107CA0006F182C960FB6F894DEBF0FBECDBFDF91D4
:107CB000CF911F910F91FF90EF90DF90CF90BF90E9
:107CC000AF909F908F9008956F927F928F929F9226
:107CD000AF92BF92CF92DF92EF92FF920F931F93DA
:107CE000CF93DF93CDB7DEB7E8970FB6F894DEBF3A
:107CF0000FBECDBF4B015C0185E790E10E94B78DBF
:107D000064E670E080E090E00E94788A40E855E206
:107D100060E070E085E790E10E94C00964E670E0F1
:107D200080E090E00E94788A6CEE72E084E89CE04B
:107D30000E94369664E87CE0CE0101960E94379559
:107D400042E350E06FEF7FEFCE0101960E94630A9D
:107D5000CE0101960E944D9461EE72E084E89CE0B1
:107D60000E94369664E87CE0CE0101960E94379529
:107D700042E350E06FEF7FEFCE0101960E94D70BF8
:107D8000CE0101960E944D9480919D0D90919E0D83
:107D90008D7F712CC12CD12CE12CF12C00E010E056
:107DA000019709F459C072E4672E0E94498A681944
:107DB00079098A099B09683B7B408105910508F098
:107DC0004BC085E790E10E94498C892BF1F14CED85
:107DD00055E060E070E085E790E10E94659368AE51
:107DE00041E050E0BE01685C7F4F85E790E10E9472
:107DF0004C94882351F14FE150E0BE016F5F7F4FFB
:107E000085E790E10E946B9389818D34F1F46FE1F5
:107E1000CE0101960E94E72A8823B9F00C8110E078
:107E2000102F00278D81080F111DEE80F12CFE2CE4
:107E3000EE248F81E80EF11CC884D12CDC2CCC24DC
:107E40008985C80ED11C7724739462E370E080E0CA
:107E500090E00E94788AA9CF0E94498A681979091E
:107E60008A099B09683B7B408105910510F47110DC
:107E7000C1C00E949E0C64E87CE0CE0180960E9406
:107E8000379542E350E066E070E0CE0180960E94B4
:107E9000630ACE0180960E944D94772009F4CFC0EA
:107EA00082E090E090939E0D80939D0D4AE0B60194
:107EB000CE0180960E9483954AE0B701CE01869656
:107EC0000E9483954AE0B801CE01C2960E94839534
:107ED000BE016E5C7F4FCE018C960E94379563E7A2
:107EE00079E0CE018C960E94C296BE016A5D7F4FFA
:107EF0000E94B19663E779E00E94C296BE01605E7F
:107F00007F4F0E94B196BC018AE89CE00E942295B6
:107F1000CE018C960E944D94CE01C2960E944D9443
:107F2000CE0186960E944D94CE0180960E944D947B
:107F30006AE87CE0CE0180960E9437954AE050E0E6
:107F40006FEF7FEFCE0180960E94D70BCE01809617
:107F50000E944D946BED72E08FE89DE00E94D290FC
:107F60004AE0B601CE0180960E9483954AE0B701AF
:107F7000CE0186960E9483954AE0B801CE01C29652
:107F80000E94839568ED76E0CE018C960E94B894AD
:107F9000BE016E5C7F4FCE018C960E94B19662E36B
:107FA00075E00E94C296BE016A5D7F4F0E94B19645
:107FB00062E375E00E94C296BE01605E7F4F0E9440
:107FC000B19668EE76E00E94C296BC018AE89CE019
:107FD0000E942295CE018C960E944D94CE01C296AD
:107FE0000E944D94CE0186960E944D94CE018096BB
:107FF0000E944D9462E370E080E090E00E94788AF5
:1080000085E790E10E94B78D62E370E080E090E048
:108010000E94788AE8960FB6F894DEBF0FBECDBFF7
:10802000DF91CF911F910F91FF90EF90DF90CF9054
:10803000BF90AF909F908F907F906F90089560ED6C
:1080400072E08AE89CE00E9436966AE87CE0CE0105
:1080500080960E9437954AE050E060E070E0CE01E3
:1080600080960E94D70BCE0180960E944D946DEBB6
:1080700072E08AE89CE00E94369680919D0D909176
:108080009E0D029709F0B6CF10929E0D10929D0D95
:10809000B1CF7F928F929F92AF92BF92CF92DF9299
:1080A000EF92FF920F931F93CF93DF9300D000D0F6
:1080B000CDB7DEB74C0188ED9FE00E94B78D40E060
:1080C00052EC61E070E088ED9FE00E94C0094CED49
:1080D00055E060E070E088ED9FE00E94659364E603
:1080E00070E080E090E00E94788AA12CB12C712C85
:1080F000A814B9040CF051C065E070E080E090E095
:108100000E94788A00E010E0C12CD12C7601711019
:108110000FC088ED9FE00E94498C892B31F485E1E6
:10812000C816D104E104F1041CF40330110554F025
:108130008FEFA81AB80A64E670E080E090E00E9431
:10814000788AD6CF88ED9FE00E94498C892B69F010
:1081500088ED9FE00E94628CE1E0F0E0EC0FFD1FF3
:10816000E00FF11F80830F5F1F4F65E070E080E03C
:1081700090E00E94788A023011054CF089818B3B97
:1081800031F4772473948A818A3A09F0712C8FEF45
:10819000C81AD80AE80AF80ABACF872D26960FB669
:1081A000F894DEBF0FBECDBFDF91CF911F910F912D
:1081B000FF90EF90DF90CF90BF90AF909F908F9007
:1081C0007F9008952F923F924F925F926F927F928D
:1081D0008F929F92AF92BF92CF92DF92EF92FF92D7
:1081E0000F931F93CF93DF93CDB7DEB72B970FB6C7
:1081F000F894DEBF0FBECDBF1C018BEB8F838AEAE4
:10820000888781E0898784E6829D9001839D300D77
:1082100011243B872A87E12CF12CC12CD12C812CF5
:10822000912C5401C214D30494F1C501B4010E94ED
:10823000FB9920E030E040E251E40E942F996B016D
:108240007C01B101882777FD8095982F0E94FB99CA
:108250009B01AC01C701B6010E942F992B960FB666
:10826000F894DEBF0FBECDBFDF91CF911F910F916C
:10827000FF90EF90DF90CF90BF90AF909F908F9046
:108280007F906F905F904F903F902F9008952A8538
:108290003B85E216F3064CF6C7016AE070E00E94E7
:1082A000BF9C892B79F4E091D80FF091D90F02800F
:1082B000F381E02D43E050E0BE01695F7F4F88ED20
:1082C0009FE0199565E070E080E090E00E94788A78
:1082D0003FEFE31AF30A00E010E0412C512C320189
:1082E00088ED9FE00E94498C892B39F424E04216E6
:1082F0005104610471040CF095CF063011050CF0A7
:1083000091CF88ED9FE00E94498C892B69F088ED20
:108310009FE00E94628CE1E0F0E0EC0FFD1FE00FB7
:10832000F11F80830F5F1F4F65E070E080E090E0F9
:108330000E94788A0630110501F599818F81981382
:108340001CC09A818885981318C09B8189859813D1
:1083500014C02C818D8190E0A0E0B0E0BA2FA92F4D
:10836000982F8827820F911DA11DB11D880E991E7F
:10837000AA1EBB1E8FEFC81AD80A9FEF491A590AC6
:10838000690A790AADCFCF92DF92EF92FF92CF9335
:10839000DF93CDB7DEB72C970FB6F894DEBF0FBED4
:1083A000CDBF88ED9FE00E94B78D40E052EC61E0C8
:1083B00070E088ED9FE00E94C0094CED55E060E060
:1083C00070E088ED9FE00E94659364E670E080E0D5
:1083D00090E00E94788A80919B0D90919C0D01976E
:1083E00051F483E090E055DE81111AC010929C0D8B
:1083F00010929B0D15C081E090E04BDE81110AC008
:1084000083E090E046DE811105C083E090E041DE2C
:10841000882331F081E090E090939C0D80939B0D38
:1084200080919B0D90919C0D0197D9F061EB72E0CA
:1084300084E89CE00E94369664E87CE0CE010196D8
:108440000E94379544E150E06FEF7FEFCE01019637
:108450000E94D70BCE0101960E944D9465EA72E00E
:1084600079C069E972E08AE89CE00E9436966AE881
:108470007CE0CE0101960E943795CE0101960E94C4
:10848000370ACE0101960E944D9462E370E080E0CD
:1084900090E00E94788A6AE87CE0CE0101960E9412
:1084A000379542E350E06FEF7FEFCE0101960E94D7
:1084B000630ACE0101960E944D946DE872E084E853
:1084C0009CE00E94369664E87CE0CE0101960E9412
:1084D000379544E150E06FEF7FEFCE0101960E94A7
:1084E000D70BCE0101960E944D9484E090E06ADEA5
:1084F0006B017C0120E030E040EA51E40E94D09A18
:10850000181634F521E0B701A601CE0107960E94A6
:10851000DA9568E379E0CE0101960E94B894BE0135
:10852000695F7F4FCE0101960E94B1966EEE76E0B4
:108530000E94C296BC018AE89CE00E942295CE016E
:1085400001960E944D94CE0107960E944D9406C05C
:1085500061E872E08AE89CE00E9436966AE87CE076
:10856000CE0101960E9437954AE050E060E070E04D
:10857000CE0101960E94630ACE0101960E944D949D
:108580006AE87CE0CE0101960E94379562E375E0CF
:10859000CE0101960E94C29664E87CE00E94B196EA
:1085A000BC018AE89CE00E942295CE0101960E94BF
:1085B0004D9488ED9FE00E94B78D80917B0C8823BD
:1085C00031F060E273E080E090E00E94788A2C96BF
:1085D0000FB6F894DEBF0FBECDBFDF91CF91FF90F5
:1085E000EF90DF90CF9008952F923F924F925F923D
:1085F0006F927F928F929F92AF92BF92CF92DF92B3
:10860000EF92FF920F931F93CF93DF93CDB7DEB717
:1086100066970FB6F894DEBF0FBECDBF6C0188ED34
:108620009FE00E94B78D40E855E260E070E088ED81
:108630009FE00E94C00964E670E080E090E00E9444
:10864000788A4CED55E060E070E088ED9FE00E9494
:10865000659364E670E080E090E00E94788A8FEF96
:10866000898381E08A8386E88B831C821D821E8237
:108670001F82188689E78987C601880F991F9E8BFC
:108680008D8B212C312CE12CF12C812C912C54013F
:10869000EC14FD044CF088ED9FE00E94B78DE114CE
:1086A000F104B9F1670135C08D899E892816390614
:1086B00094F788ED9FE00E94D98D08977CF0E091B7
:1086C000D80FF091D90F0280F381E02D49E050E0FE
:1086D000BE016F5F7F4F88ED9FE0199565E070E008
:1086E00080E090E00E94788A00E010E0412C512C5C
:1086F000320188ED9FE00E94498C892B31F4E4E03F
:108700004E1651046104710484F5023011056CF5B4
:1087100030C0C501B4010E94FB994B015C01B60158
:10872000882777FD8095982F0E94FB999B01AC01CB
:10873000C501B4010E942F9966960FB6F894DEBF6A
:108740000FBECDBFDF91CF911F910F91FF90EF90A2
:10875000DF90CF90BF90AF909F908F907F906F9061
:108760005F904F903F902F900895FFEF2F1A3F0A90
:108770008FCF88ED9FE00E94498C892B69F088EDAE
:108780009FE00E94628CEAE0F0E0EC0FFD1FE00F3A
:10879000F11F80830F5F1F4F65E070E080E090E085
:1087A0000E94788A0230110569F59A8589819813AB
:1087B00029C09B858B81981325C0FE013C96FC8BBC
:1087C000EB8B88ED9FE00E94498C892B31F4F4E01B
:1087D0004F16510461047104DCF409301105E1F411
:1087E0002D858C8590E0982F8827820F911DAA27D0
:1087F00097FDA095BA2F880E991EAA1EBB1E8FEF5B
:10880000E81AF80A9FEF491A590A690A790A71CFDA
:1088100004301105A4F3E4CF88ED9FE00E94628C40
:10882000EB89FC898193FC8BEB8B0F5F1F4FC9CFCA
:108830008091F704882349F08091F604882329F079
:1088400060E08FE89DE00C944F8008952F923F9256
:108850004F925F926F927F928F929F92AF92BF9250
:10886000CF92DF92EF92FF920F931F93CF93DF93FC
:10887000CDB7DEB763970FB6F894DEBF0FBECDBF9E
:108880008B8B60E00E94878B80917B0C811105C0EF
:108890008FE090E0A0E0B0E004C082E090E0A0E0D3
:1088A000B0E08F87988BA98BBA8B64E772E08AE877
:1088B0009CE00E9436966AE87CE0CE0101960E9418
:1088C00037954AE050E06FEF7FEFCE0101960E94AE
:1088D000630ACE0101960E944D94C12CD12C7601E1
:1088E000312C1D861E86212C02E310E0412C512CD8
:1088F00032018B890E940E8BAA2797FDA095BA2F73
:10890000480E591E6A1E7B1E65E070E080E090E014
:108910000E94788A0150110961F7809012029090AC
:108920001302A0901402B0901502C301B2010E947C
:10893000FB9920E030E040EA50E40E948F9B20E069
:1089400030E040E85AE30E948F9B20E030E048E4AA
:1089500052E40E942F99A50194010E94649820E09E
:1089600030E040E751E40E948F9B2B013C01A501C0
:1089700094016AE979E989E390E40E9464989B0193
:10898000AC01C301B2010E942F9920E030E0A9019F
:108990000E94659820E030E040E251E40E948F9B05
:1089A0005B018C01232D3D854E85522D0E94D09A6E
:1089B000181624F43A2CBD860E87212E20E030E0D4
:1089C000A901B501C8010E942B9987FF04C0A12C01
:1089D000B12C00E010E022E0A501B801CE0107961D
:1089E0000E94DA95BE01695F7F4FCE0101960E9419
:1089F000379561EF76E0CE0101960E94C296BC01E8
:108A000084E89CE00E942295CE0101960E944D943C
:108A1000CE0107960E944D9464E87CE0CE01019659
:108A20000E9437954AE050E060E070E0CE01019688
:108A30000E94D70BCE0101960E944D940E94498A54
:108A40008090EA049090EB04A090EC04B090ED04C8
:108A50000091870D1091880D2091890D30918A0D1C
:108A6000800E911EA21EB31E86169706A806B90692
:108A700008F4E9C00E94498A0E94F9994B015C01FF
:108A80006091EA047091EB048091EC049091ED0404
:108A90000E94FB9920E030E040E85EE30E948F9B5B
:108AA0002B013C016091870D7091880D8091890D9B
:108AB00090918A0D0E94FB999B01AC01C301B20108
:108AC0000E9465989B01AC01C501B4010E942B99DD
:108AD00087FDB9C06CE370E080E090E00E94788A86
:108AE0009FEFC91AD90AE90AF90A8F859889A989D5
:108AF000BA898C159D05AE05BF050CF0F5CE64E670
:108B000070E080E090E00E94788A0E949E0C64E60B
:108B100070E080E090E00E94788A6CE672E084E881
:108B20009CE00E94369664E87CE0CE0101960E94AB
:108B3000379544E150E060E070E0CE0101960E947C
:108B4000630ACE0101960E944D9422E0432D5D857B
:108B50006E85722DCE0107960E94DA95BE01695F7F
:108B60007F4FCE0101960E94379561EF76E0CE01EE
:108B700001960E94C296BC0184E89CE00E94229566
:108B8000CE0101960E944D94CE0107960E944D940D
:108B900064E87CE0CE0101960E94379542E350E004
:108BA0006FEF7FEFCE0101960E94D70BCE010196A9
:108BB0000E944D9464E170E080E090E00E94788A29
:108BC00037DE6EE170E080E090E00E94788A6EE12E
:108BD00070E080E090E00E94788A66EF76E0CE0157
:108BE00001960E94B89464E87CE0CE0101960E9450
:108BF000B1966AEF76E00E94C2966AE87CE00E9435
:108C0000B196BC018AE89CE00E942295CE010196B3
:108C10000E944D9463960FB6F894DEBF0FBECDBF91
:108C2000DF91CF911F910F91FF90EF90DF90CF9048
:108C3000BF90AF909F908F907F906F905F904F907C
:108C40003F902F900895F4DD45CFFF920F931F932F
:108C5000CF93DF93CDB7DEB72C970FB6F894DEBF76
:108C60000FBECDBF10927C0C62E17BE082EA9CE0FB
:108C70000E94559511E08BE39FE00E94498C209162
:108C80007C0C18161906C4F5211136C08BE39FE041
:108C90000E94628C80937D0C8A3041F08D3031F0DF
:108CA000682F82EA9CE00E949E961FC010937C0C65
:108CB0006EEF76E0CE0107960E94B89462EA7CE0FF
:108CC000CE0107960E94B196BC01CE0101960E948A
:108CD0003795CE0101960E94370ACE0101960E9477
:108CE0004D94CE0107960E944D946AE070E080E0BA
:108CF00090E00E94788ABFCF222361F020917C0C03
:108D00008091A60C9091A70C211174C0009709F0D6
:108D100071C0B8C000E010E0FF24F39482E191E15B
:108D20000E94498C18161906A4F582E191E10E946F
:108D3000628C80937D0C8A3071F08D3061F090915F
:108D40007C0C911108C0682F82EA9CE00E949E96DC
:108D50000F5F1F4F17C08091A60C9091A70C892B15
:108D600089F0F0927C0C82E191E10E94498C181606
:108D7000190644F462E17BE082EA9CE00E9455958A
:108D800010927C0C6FE070E080E090E00E94788AA6
:108D9000C5CF62E370E080E090E00E94788A012B0A
:108DA00009F4ACCF67E077E0CE0107960E94B89453
:108DB00062EA7CE0CE0107960E94B196BC01CE012A
:108DC00001960E943795CE0101960E94370ACE0186
:108DD00001960E944D94CE0107960E944D9482E127
:108DE00091E10E94D08C64E670E080E090E00E9407
:108DF000788A84CF019709F069C06AE776E0CE01EE
:108E000007960E94B894BE01695F7F4F82EA9CE09A
:108E10000E94FE96811115C06DE077E0CE010196AB
:108E20000E94B894BE016F5F7F4F82EA9CE00E946F
:108E3000FE9611E0811110E0CE0101960E944D9442
:108E400001C010E0CE0107960E944D94112399F0C5
:108E500040E050E062EA7CE0CE0101960E94B40955
:108E6000BE016F5F7F4F86E99CE00E943F95CE0177
:108E700001960E944D9464E170E080E090E00E94D1
:108E8000788A24C064E670E080E090E00E94788AEE
:108E90000E94498ACB0168EE73E00E94BF9CCB011F
:108EA00064E670E00E94BF9C823691057CF0809160
:108EB0007B0C81110BC086E99CE00E943E986130DA
:108EC00071058105910511F40E946F182C960FB65B
:108ED000F894DEBF0FBECDBFDF91CF911F910F91F0
:108EE000FF900895BF92CF92DF92EF92FF920F937F
:108EF0001F93CF93DF93CDB7DEB72B970FB6F894C0
:108F0000DEBF0FBECDBF6C0188ED9FE00E94B78D24
:108F100040E855E260E070E088ED9FE00E94C00903
:108F200064E670E080E090E00E94788A4CED55E0C5
:108F300060E070E088ED9FE00E94659364E670E079
:108F400080E090E00E94788A8FEF898381E08A83B5
:108F500086E88B831C821D821E821F82188689E709
:108F6000898788ED9FE00E94D08C62E370E080E00A
:108F700090E00E94788A88ED9FE00E94D98D089742
:108F80007CF0E091D80FF091D90F0280F381E02DB1
:108F900049E050E0BE016F5F7F4F88ED9FE019957B
:108FA00062E370E080E090E00E94788AE12CF12C8E
:108FB000B12CEC14FD040CF05BC088ED9FE00E9426
:108FC000498C892B21F188ED9FE00E94D98D08976B
:108FD0007CF0E091D80FF091D90F0280F381E02D61
:108FE00049E050E0BE016F5F7F4F88ED9FE019952B
:108FF00065E070E080E090E00E94788A00E010E098
:1090000088ED9FE00E94498C0230110554F062E324
:1090100070E080E090E00E94788A8FEFE81AF80A0A
:10902000C8CF88ED9FE00E94498C892B69F088EDBC
:109030009FE00E94628CEAE0F0E0EC0FFD1FE00F81
:10904000F11F80830F5F1F4F65E070E080E090E0CC
:109050000E94788A0230110599F69A8589819813C1
:10906000CFCF9B858B819813CBCFBB24B394C8CF34
:1090700088ED9FE00E94B78D8B2D2B960FB6F8944C
:10908000DEBF0FBECDBFDF91CF911F910F91FF903B
:10909000EF90DF90CF90BF900895CF92DF92EF9244
:1090A000FF920F931F93CF93DF93CDB7DEB72C972B
:1090B0000FB6F894DEBF0FBECDBF0E949E0C6CE2CF
:1090C00073E08AE89CE00E9436966AE87CE0CE0174
:1090D00001960E9437954AE050E060E070E0CE01D2
:1090E00001960E94630ACE0101960E944D9463E2AC
:1090F00073E084E89CE00E94369664E87CE0CE0150
:1091000001960E94379544E150E06FEF7FEFCE016A
:1091100001960E94D70BCE0101960E944D9480913A
:109120009B0D90919C0D8230910551F481E090E06F
:10913000D9DE81111CC010929C0D10929B0D17C09E
:10914000892BA9F481E090E0CDDE81110AC081E095
:1091500090E0C8DE811105C081E090E0C3DE882385
:1091600031F082E090E090939C0D80939B0D809174
:109170009B0D90919C0D029791F167E173E08AE855
:109180009CE00E9436966AE87CE0CE0101960E943F
:1091900037954AE050E060E070E0CE0101960E9411
:1091A000630ACE0101960E944D946AE87CE0CE01EC
:1091B00001960E94379562E375E0CE0101960E9408
:1091C000C29664E87CE00E94B196BC018AE89CE00B
:1091D0000E942295CE0101960E944D9497C08AE08C
:1091E00090E002DA6B017C0120E030E0A9010E94EE
:1091F0002B9918162CF08AE090E0F6D96B017C01CF
:109200000BE010E020E030E042ED53E4C701B6018E
:109210000E942B99181684F420E030E0A901C701C0
:10922000B6010E942B991816B4F069E073E08AE841
:109230009CE00E94369640C00150110969F368EC29
:1092400070E080E090E00E94788A83E090E0CCD9E2
:109250006B017C01D7CF20E030E048EC52E4C7013D
:10926000B6010E942B9987FF02C021E001C020E0D7
:10927000B701A601CE0107960E94DA9569EE75E066
:10928000CE0101960E94B894BE01695F7F4FCE0166
:1092900001960E94B1966EEE75E00E94C296BC01E6
:1092A0008AE89CE00E942295CE0101960E944D948E
:1092B000CE0107960E944D946AE87CE0CE010196AB
:1092C0000E94379542E350E06FEF7FEFCE010196A9
:1092D0000E94D70BCE0101960E944D9460E073E08E
:1092E00084E89CE00E94369664E87CE0CE0101961A
:1092F0000E94379542E350E060E070E0CE010196B5
:109300000E94630ACE0101960E944D9480917B0CCD
:10931000882331F060E273E080E090E00E94788A78
:109320002C960FB6F894DEBF0FBECDBFDF91CF9164
:109330001F910F91FF90EF90DF90CF9008954F9283
:109340005F926F927F928F929F92AF92BF92CF92D5
:10935000DF92EF92FF92CF93DF93CDB7DEB76097A6
:109360000FB6F894DEBF0FBECDBF80917B0C81118C
:1093700005C08EE190E0A0E0B0E004C082E090E0A3
:10938000A0E0B0E08D879E87AF87B88B69EA73E075
:109390008AE89CE00E9436966AE87CE0CE0101965D
:1093A0000E9437954AE050E06FEF7FEFCE010196C3
:1093B0000E94D70BCE0101960E944D94812C912CD6
:1093C0005401C12CD12C760163E270E082E79EE06B
:1093D0000E94AB7667E070E082E79EE00E94C309DE
:1093E00082E79EE00E941F7766E970E080E090E0EF
:1093F0000E94788A63E270E082E79EE00E94AB768A
:1094000060E270E082E79EE00E94C30982E79EE08E
:109410000E941F7766E970E080E090E00E94788A01
:1094200042E050E063E270E082E79EE00E941D7738
:10943000412C512C320182E79EE00E9403761816DF
:1094400019066CF482E79EE00E940B76762C652C60
:10945000542C4424480E511C611C711CECCFC301D8
:10946000B2010E94FB992AE939E949E95FE30E94C8
:109470002F990E94C899AB01BC01C416D506E60617
:10948000F70614F46A017B012AE0CE0107960E94D8
:10949000AE95BE01695F7F4FCE0101960E94379560
:1094A0006FE077E0CE0101960E94C296BC0184E88D
:1094B0009CE00E942295CE0101960E944D94CE011F
:1094C00007960E944D9464E87CE0CE0101960E94CC
:1094D00037954EE150E060E070E0CE0101960E94C9
:1094E0000C0BCE0101960E944D949FEF891A990AA8
:1094F000A90AB90A8D859E85AF85B8898815990511
:10950000AA05BB050CF060CF2AE0B701A601CE0189
:1095100007960E94AE95BE01695F7F4FCE0101960E
:109520000E9437956FE077E0CE0101960E94C296C7
:10953000BC0184E89CE00E942295CE0101960E9425
:109540004D94CE0107960E944D9464E87CE0CE01D4
:1095500001960E9437954AE050E060E070E0CE014D
:1095600001960E94630ACE0101960E944D942AE062
:10957000B701A601CE0107960E94AE9563E177E0A0
:10958000CE0101960E94B894BE01695F7F4FCE0163
:1095900001960E94B19666E177E00E94C2966AE861
:1095A0007CE00E94B196BC018AE89CE00E94229572
:1095B000CE0101960E944D94CE0107960E944D94D3
:1095C00062E370E080E090E00E94788A60960FB6D7
:1095D000F894DEBF0FBECDBFDF91CF91FF90EF902B
:1095E000DF90CF90BF90AF909F908F907F906F90C3
:1095F0005F904F9008958F929F92AF92BF92CF92BB
:10960000DF92EF92FF920F931F93CF93DF93CDB72B
:10961000DEB72C970FB6F894DEBF0FBECDBF8C011E
:10962000E090770CF090780C8091790C882369F0A9
:109630006BE177E08BE39FE00E9403914AE050E00A
:10964000B8018BE39FE00E94F491C801059605974D
:1096500008F18091770C9091780C8017910709F1AF
:109660000E949E0C0E94702F1093780C0093770C30
:109670004AE0B801CE0101960E948395BE016F5F5A
:109680007F4F86E99CE00E943F95CE0101960E94A3
:109690004D9407C00E3F8FEF1807A9F40E94832F47
:1096A0004FC262E375E0CE0101960E94B8944AE091
:1096B00050E06FEF7FEFCE0101960E940C0BCE01C0
:1096C00001960E944D94F8017996E533F10508F072
:1096D000D6C1EE58FF4F0C94109D80917B0C8823CF
:1096E00019F00E947336F9C160910A0270910B0261
:1096F00080910C0290910D020E946434EEC1809121
:10970000E4049091E5040E949E2FE7C18091C80473
:109710009091C9049BD8E1C18091BC049091BD0493
:109720000E947F2DDAC18091BE049091BF04B5DC08
:10973000D4C10E94498A0E94643ECFC160E070E0BB
:109740008091C2049091C3040E943C27C6C18091BD
:10975000B8049091B9040E94332BBFC180917A0C58
:1097600091E0892780937A0C80917B0C882331F0DB
:109770006AE87CE082E191E10E941E9168EC70E071
:1097800080E090E00E94788AA8C110927B0CA5C16D
:1097900081E080937B0C66E97CE08CE99CE00E9490
:1097A00022958091770C9091780C9093760C809311
:1097B000750C93C10E94C30C90C10E94C3418DC11E
:1097C0000E942D178AC180913C02882309F485C12B
:1097D00062E17BE0CE0101960E94B8944AE050E03D
:1097E00061E070E0CE0101960E94630ACE0101960D
:1097F0000E944D940E94F50E70C1A1DD6EC1809152
:10980000C4049091C5040E94C02C67C18091BA0421
:109810009091BB040E94CA2B60C180913C028823B6
:1098200009F45BC180917B0C882329F082E090E0F1
:109830000E94401152C183E090E00E946F154DC11B
:109840000E943F2582E191E10E94D08C46C1809127
:109850008102909182020E9465293FC180913C0261
:10986000882309F43AC180917B0C811127C0C090F4
:109870000A02D0900B02E0900C02F0900D0220E062
:1098800030E04AE754E4C701B6010E948F9B0E9472
:10989000C8994B015C0120E030E040EA50E4C70188
:1098A000B6010E948F9B20E030E040EA50E40E9425
:1098B00065980E94C899A501940108C021E030E094
:1098C00040E050E06AE070E080E090E00E94781FA5
:1098D00004C18091D90B9091DA0B892BF1F581E0CD
:1098E00090E09093DA0B8093D90B65E277E0CE019C
:1098F00001960E94B894CE0101960E94370ACE01CB
:1099000001960E944D9460E175E0CE0107960E9499
:10991000B89461E87DE0CE0107960E94B196BC0143
:10992000CE0101960E94379548EC50E06FEF7FEF33
:10993000CE0101960E94630ACE0101960E944D94C9
:10994000CE0107960E944D9482E191E10E94B78D6D
:1099500040E052EC61E070E03BC01092DA0B1092F4
:10996000D90B6EE277E0CE0101960E94B894CE0149
:1099700001960E94370ACE0101960E944D946CE038
:1099800075E0CE0107960E94B89461E87DE0CE01B3
:1099900007960E94B196BC01CE0101960E943795B0
:1099A00048EC50E06FEF7FEFCE0101960E94630A12
:1099B000CE0101960E944D94CE0107960E944D94CF
:1099C00082E191E10E94B78D40E855E260E070E0ED
:1099D00082E191E10E94C00910920C0C10920B0CD4
:1099E00080E090E00E94EA0966E175E0CE0107960A
:1099F0000E94B8946BE77DE0CE0107960E94B19675
:109A0000BC01CE0101960E94379540ED57E06FEF03
:109A10007FEFCE0101960E94D70BCE0101960E94E6
:109A20004D94CE0107960E944D9457C080919F0D92
:109A30009091A00D892BA1F481E090E09093A00D6E
:109A400080939F0D8EED93E090930C0C80930B0C04
:109A50000E94130A68EC70E080E090E00E94788A2F
:109A6000E091400BF091410B199537C08FE89DE0D4
:109A70000E9454800E949E0C0E94702F2EC0F09273
:109A8000780CE092770C6EEC78E08AE89CE00E941B
:109A9000369662E17BE0CE0101960E94B8944AE0DE
:109AA00050E060E070E0CE0101960E94630ACE01B2
:109AB00001960E944D946AE87CE0CE0101960E94D6
:109AC00037954AE050E06FEF7FEFCE0101960E949C
:109AD000D70BCE0101960E944D9480918E0C9091EF
:109AE0008F0C009799F0419718F402301105ACF4EF
:109AF0006AE87CE0CE0101960E943795CE0101967E
:109B00000E945D10CE0101960E944D9464E670E0C3
:109B100080E090E00E94788A13C06AE87CE0CE0181
:109B200001960E9437954AE050E06FEF7FEFCE013B
:109B300001960E94D70BCE0101960E944D94D8CF7A
:109B40002C960FB6F894DEBF0FBECDBFDF91CF913C
:109B50001F910F91FF90EF90DF90CF90BF90AF904B
:109B60009F908F900895FF920F931F93CF93DF9351
:109B700000D000D0CDB7DEB7823409F441C0CCF4B8
:109B8000803309F45DC07CF4833209F450C08A321A
:109B900009F075C06FE477E082EA9CE00E94559579
:109BA0008FEF9FEF6AC0813309F459C08134E9F027
:109BB00066C08136D1F02CF4833469F1843439F0F5
:109BC0005EC0833641F1E4F0843609F058C08091DC
:109BD0009A0C90919B0C892B09F4E3C086E99CE0D8
:109BE0000E943E9897FF68C0DCC063E477E082EA99
:109BF0009CE00E9455958091770C9091780C3DC027
:109C000066E477E082EA9CE00E94559510927B0C16
:109C10008CEF9FEF32C069E477E082EA9CE00E941B
:109C2000559581E080937B0C8DEF9FEF26C06CE40F
:109C300077E082EA9CE00E9455958EEF9FEF1DC071
:109C400062E677E086E99CE00E94559562E677E05F
:109C500082EA9CE00E94559580E090E00EC060E5AD
:109C600077E086E99CE00E94559560E577E082EA1E
:109C70009CE00E94559581E090E0BDDC9AC0682F81
:109C8000CE0101960E946B95BE016F5F7F4F86E902
:109C90009CE00E943F95CE0101960E944D9486E97A
:109CA0009CE00E943E98CB01A6DC64E670E080E078
:109CB00090E00E94788A7DC08091790C882361F0C1
:109CC0006CE377E08BE39FE00E94039166E97CE020
:109CD0008BE39FE00E941E9186E99CE00E943E98E3
:109CE000DC01CB014AEF5FEF6FEF7FEF481B590BB1
:109CF0006A0B7B0B2AE0CE0101960E94AE95BE0155
:109D00006F5F7F4F86E99CE00E943F95CE010196F0
:109D10000E944D9486E99CE040C00F5F1F4F093EB2
:109D200083E0180769F06EE170E080E090E00E9447
:109D3000788A80E09DE00E948983F82EFF2069F3F5
:109D40006AE270E06F197109F7FC73954AE0CE0181
:109D500001960E948395BE016F5F7F4F82EA9CE06F
:109D60000E943F95CE0101960E944D9462EA7CE0EC
:109D700086E99CE00E9422958091790C882359F015
:109D80006CE377E08BE39FE00E9403916F2D8BE300
:109D90009FE00E943E9182EA9CE00E943E98CB01A7
:109DA0006CCF80E09DE00E948983F82E00E010E0F7
:109DB000C5CF26960FB6F894DEBF0FBECDBFDF919C
:109DC000CF911F910F91FF9008950F931F93CF9301
:109DD000DF9300D000D0CDB7DEB78091790C882317
:109DE000A1F062E577E08BE39FE00E940391409150
:109DF000560B5091570B6091580B7091590B20E105
:109E000030E08BE39FE00E943B928091560B909153
:109E1000570BA091580BB091590B883025E0920751
:109E2000A105B10509F4FCC108F08DC0893421E019
:109E30009207A105B10509F4F6C1E0F5843421E0EB
:109E40009207A105B10509F4DFC1E8F4813421E0EE
:109E50009207A105B10509F4C8C138F480349140D6
:109E6000A105B10509F4B2C1E1C1823421E0920734
:109E7000A105B10509F4C2C183349140A105B10522
:109E800009F4BFC1D3C1863421E09207A105B10511
:109E900009F4C0C108F4BBC1873421E09207A105D1
:109EA000B10509F4BAC188349140A105B10509F49E
:109EB000B7C1BCC1823025E09207A105B10509F404
:109EC0009DC1E8F4843721E09207A105B10509F4AA
:109ED00048C138F482379140A105B10509F44CC15D
:109EE000A5C1811525E09207A105B10509F46EC150
:109EF00081309540A105B10509F477C197C185303E
:109F000025E09207A105B10509F481C170F4833001
:109F100025E09207A105B10509F473C1843095408D
:109F2000A105B10509F470C181C1863025E0920711
:109F3000A105B10509F46EC187309540A105B105B1
:109F400009F46BC173C18D3B22E492072FEFA20786
:109F5000B10509F42CC108F04BC08F3E20E19207F7
:109F60002FEFA207B10509F458C118F5823325E097
:109F70009207A105B10509F4FFC038F48930954076
:109F8000A105B10509F44FC151C1843325E0920701
:109F9000A105B10509F4E5C08D3F9240AF4FB10571
:109FA00009F044C163E477E082EA9CE00E945595A1
:109FB000E0C08D3D22E292072FEFA207B10509F420
:109FC000D0C038F4873E9841AF4FB10509F41FC1A6
:109FD0002DC18F3C20E392072FEFA207B10509F4B2
:109FE00013C1873C9843AF4FB10509F419C11EC195
:109FF000873928E692072FEFA207B10509F4F5C0CB
:10A0000048F58D3A22E592072FEFA207B10509F432
:10A01000BFC038F4853B9A44AF4FB10509F4D6C0B0
:10A0200005C1853A2AE592072FEFA207B10509F489
:10A03000FAC08D399246AF4FB10509F0F7C066E41A
:10A0400077E082EA9CE00E94559510927B0C8CEFA1
:10A050009FEF85C0873528EA92072FEFA207B10549
:10A06000F9F078F485382AE792072FEFA207B105B7
:10A0700009F4D0C087369849AF4FB10509F4BEC086
:10A08000D5C08F3420EB92072FEFA207B10509F45A
:10A09000B8C08D33924CAF4FB10509F46DC0C6C046
:10A0A00082E69BE00E943B6600E010E062E47BE019
:10A0B00082E69BE00E94F066892B39F40F5F1F4F08
:10A0C000093E83E0180709F09DC18091790C88232F
:10A0D000A1F06BEB78E08BE39FE00E94D29040917F
:10A0E000460B5091470B6091480B7091490B2AE049
:10A0F00030E08BE39FE00E943B928091460B909171
:10A10000470BA091480BB091490B853025E0920791
:10A11000A105B10509F461C108F0E1C0873421E06F
:10A120009207A105B10509F464C108F0B8C08334F1
:10A1300021E09207A105B10509F43DC108F0A5C0D1
:10A14000813421E09207A105B10509F097C067E5C8
:10A1500077E086E99CE00E94559589EF9FEF4BDA06
:10A160007EC063E477E082EA9CE00E9455951092FD
:10A170007B0C8BEF9FEFF3CF69E477E082EA9CE002
:10A180000E94559581E080937B0C8DEF9FEFE7CF88
:10A190006CE477E086E99CE00E9455956CE477E0FA
:10A1A00082EA9CE00E9455958EEF9FEFD8CF6FE436
:10A1B00077E086E99CE00E9455956FE477E082EABB
:10A1C0009CE00E9455958FEF9FEFC9CF62E677E044
:10A1D00086E99CE00E94559562E677E082EA9CE081
:10A1E0000E94559580E090E0BACF60E577E086E97F
:10A1F0009CE00E94559581E090E0B1CF82E090E034
:10A20000AECF83E090E0ABCF84E090E0A8CF85E0D4
:10A2100090E0A5CF86E090E0A2CF87E090E09FCFCE
:10A2200088E090E09CCF89E090E099CF40E050E05A
:10A2300062EA7CE0CE0101960E94B409BE016F5F24
:10A240007F4F86E99CE00E943F95CE0101960E94D7
:10A250004D9464E670E080E090E00E94788A82E6A7
:10A260009BE00E943B6626960FB6F894DEBF0FBEB9
:10A27000CDBFDF91CF911F910F910895823491400E
:10A28000A105B10509F48EC0E4CF853421E0920721
:10A29000A105B10509F4A1C008F496C0A7C081309A
:10A2A00025E09207A105B10509F451CF70F4883477
:10A2B00021E09207A105B10509F49EC089349140BF
:10A2C000A105B10509F49BC0C4CF833025E09207F6
:10A2D000A105B10509F46FC008F464C075C08F3CD6
:10A2E00020E392072FEFA207B10509F46DC068F5CE
:10A2F000883025E09207A105B10509F47DC070F40E
:10A30000863025E09207A105B10509F46FC08730BA
:10A310009540A105B10509F46CC09BCF8F3E20E1AB
:10A3200092072FEFA207B10509F463C0873E28E129
:10A3300092072FEFA207B10509F44FC0893095406D
:10A34000A105B10509F085CF5AC0873928E69207E3
:10A350002FEFA207B10509F4FACE78F4873C28E381
:10A3600092072FEFA207B10509F446C0853A9A4536
:10A37000AF4FB10509F443C06CCF873628E9920787
:10A380002FEFA207B10571F08F3420EB92072FEF6A
:10A39000A207B10581F085389A47AF4FB10509F0A2
:10A3A00058CF24C06AE577E086E99CE00E94559585
:10A3B00088EF9FEFD4CE6DE577E086E99CE00E94C0
:10A3C000559587EF9FEFCBCE60E677E086E99CE07E
:10A3D0000E94559586EF9FEFC2CE64E677E086E94E
:10A3E0009CE00E94559585EF9FEFB9CE84EF9FEFDB
:10A3F000B6CE83EF9FEFB3CE82EF9FEFB0CE81EF6B
:10A400009FEFADCE6EE170E080E090E00E94788A30
:10A410004DCE8F929F92AF92BF92CF92DF92EF92EA
:10A42000FF920F931F93CF93DF93CDB7DEB7A6971D
:10A430000FB6F894DEBF0FBECDBF62E57BE082E6CB
:10A440009BE00E94F066892BC9F00E94702F0E9449
:10A450009E0C62E375E0CE0101960E94B8944AE03A
:10A4600050E060E070E0CE0101960E94630ACE01E8
:10A4700001960E944D94A9DC0C94156462E17BE086
:10A4800082EA9CE00E9455950E9425466AE070E0B1
:10A4900080E090E00E94788A8091A60C9091A70CB1
:10A4A000009711F40C94F663019709F046C062EF2F
:10A4B00075E0CE010F960E94B894BE01615F7F4F98
:10A4C00082EA9CE00E94FE9681112AC06FEE76E03F
:10A4D000CE0109960E94B894BE01675F7F4F82EA61
:10A4E0009CE00E94FE96811115C069E775E0CE01DF
:10A4F00001960E94B894BE016F5F7F4F82EA9CE094
:10A500000E94FE9611E0811110E0CE0101960E949A
:10A510004D9401C010E0CE0109960E944D9401C0F7
:10A5200010E0CE010F960E944D94112331F062EAA3
:10A530007CE086E99CE00E9422958091A60C909197
:10A54000A70C0497F0F568E677E0CE0101960E942B
:10A55000B894BE016F5F7F4F82EA9CE00E94FE9636
:10A56000182FCE0101960E944D94112351F141E024
:10A5700050E062EA7CE0CE0109960E94B409CE0167
:10A5800009960E943E98DC01CB014AEF5FEF6FEF26
:10A590007FEF481B590B6A0B7B0B2AE0CE0101961B
:10A5A0000E94AE95BE016F5F7F4F86E99CE00E94DE
:10A5B0003F95CE0101960E944D94CE0109960E94CE
:10A5C0004D946AE677E0CE0109960E94B894BE01E8
:10A5D000675F7F4F82EA9CE00E94FE96811116C061
:10A5E0006EE677E0CE0101960E94B894BE016F5FDF
:10A5F0007F4F82EA9CE00E94FE9611E0811101C02B
:10A6000010E0CE0101960E944D9401C011E0CE01F0
:10A6100009960E944D94112309F417C362E777E06D
:10A62000CE0101960E94B894CE0101960E945D1061
:10A63000CE0101960E944D946EE777E0CE01099617
:10A640000E94B89461E87DE0CE0109960E94B1961F
:10A65000BC01CE0101960E943795CE0101960E9461
:10A660005D10CE0101960E944D94CE0109960E9484
:10A670004D94609138027091390280913A02909124
:10A680003B020E94FB9920E030E048EC52E40E943B
:10A690002F99AB01BC0122E0CE010F960E94DA9502
:10A6A00064E977E0CE0109960E94B894BE01615F2B
:10A6B0007F4FCE0109960E94B19663EC78E00E942C
:10A6C000C296BC01CE0101960E943795CE0101963B
:10A6D0000E945D10CE0101960E944D94CE01099614
:10A6E0000E944D94CE010F960E944D9440913402E9
:10A6F00050913502609136027091370224E0CE010C
:10A700000F960E94DA9569EA77E0CE0109960E94D9
:10A71000B894BE01615F7F4FCE0109960E94B19649
:10A72000BC01CE0101960E943795CE0101960E9490
:10A730005D10CE0101960E944D94CE0109960E94B3
:10A740004D94CE010F960E944D9440911E0250915F
:10A750001F02609120027091210222E0CE01099631
:10A760000E94DA95409116025091170260911802EA
:10A770007091190223E0CE010F960E94DA95409164
:10A78000220250912302609124027091250222E05E
:10A79000CE0145960E94DA9540911A0250911B0213
:10A7A00060911C0270911D0223E0CE0181960E94EF
:10A7B000DA9566EC77E0CE014B960E94B894BE0124
:10A7C0006F5D7F4FCE014B960E94B1966BED77E0A7
:10A7D0000E94C296BE016B5E7F4F0E94B1966EEDE5
:10A7E00077E00E94C296BE01615F7F4F0E94B196E2
:10A7F0006BED77E00E94C296BE01675F7F4F0E94BB
:10A80000B19664EE77E00E94C296BC01CE0101963B
:10A810000E943795CE0101960E945D10CE010196EF
:10A820000E944D94CE014B960E944D94CE0181968C
:10A830000E944D94CE0145960E944D94CE010F96F4
:10A840000E944D94CE0109960E944D94409145027C
:10A8500050914602609147027091480223E0CE0178
:10A8600009960E94DA952091490230914A0240915E
:10A870004B0250914C0260E070E080E291E40E9453
:10A88000F29BAB01BC0121E0CE0145960E940896E7
:10A8900069EE77E0CE010F960E94B894BE016B5E20
:10A8A0007F4FCE010F960E94B1966CEF77E00E9429
:10A8B000C296BE01675F7F4F0E94B19664EF75E05C
:10A8C0000E94C296BC01CE0101960E943795CE012E
:10A8D00001960E945D10CE0101960E944D94CE011A
:10A8E0000F960E944D94CE0145960E944D94CE0144
:10A8F00009960E944D94409141025091420260910C
:10A9000043027091440223E0CE0109960E94DA9539
:10A9100020913D0230913E0240913F025091400211
:10A9200060E070E080E291E40E94F29BAB01BC0128
:10A9300021E0CE0145960E94089662E078E0CE01C3
:10A940000F960E94B894BE016B5E7F4FCE010F96AA
:10A950000E94B1966CEF77E00E94C296BE01675FDD
:10A960007F4F0E94B19664EF75E00E94C296BC01D1
:10A97000CE0101960E943795CE0101960E945D108E
:10A98000CE0101960E944D94CE010F960E944D94E7
:10A99000CE0145960E944D94CE0109960E944D9499
:10A9A00040914D0250914E0260914F0270915002C1
:10A9B00022E0CE010F960E94DA9565E178E0CE01A3
:10A9C00009960E94B894BE01615F7F4FCE0109963F
:10A9D0000E94B1966BE278E00E94C296BC01CE0163
:10A9E00001960E943795CE0101960E945D10CE011E
:10A9F00001960E944D94CE0109960E944D94CE017D
:10AA00000F960E944D944091120250911302609152
:10AA100014027091150222E0CE010F960E94DA9581
:10AA200062E378E0CE0109960E94B894BE01615FAE
:10AA30007F4FCE0109960E94B19664EF75E00E94A7
:10AA4000C296BC01CE0101960E943795CE010196B7
:10AA50000E945D10CE0101960E944D94CE01099690
:10AA60000E944D94CE010F960E944D9426E9C22E6D
:10AA700024E0D22E01E010E037E1E32E809194042F
:10AA800090919504801791070CF44FC0D601AD90BA
:10AA9000BD906D014AE0B501CE0109960E948395F3
:10AAA0004AE0B801CE0145960E94839565E478E0BE
:10AAB000CE010F960E94B894BE016B5E7F4FCE010F
:10AAC0000F960E94B19662E178E00E94C296BE01A4
:10AAD000675F7F4F0E94B1966DE478E00E94C29656
:10AAE000EA9CB001EB9C700D11246D577D4F0E94C4
:10AAF000C296BC01CE0101960E943795CE01019607
:10AB00000E945D10CE0101960E944D94CE010F96D9
:10AB10000E944D94CE0145960E944D94CE01099617
:10AB20000E944D940F5F1F4FA9CF8091D90B909138
:10AB3000DA0B892B71F463E578E0CE0101960E946F
:10AB4000B894CE0101960E945D10CE0101960E943C
:10AB50004D948091D90B9091DA0B019771F462E6D4
:10AB600078E0CE0101960E94B894CE0101960E9431
:10AB70005D10CE0101960E944D9440910E025091BD
:10AB80000F02609110027091110222E0CE010F9627
:10AB90000E94DA956CE678E0CE0109960E94B8949E
:10ABA000BE01615F7F4FCE0109960E94B1966AE7B0
:10ABB00076E00E94C296BC01CE0101960E943795B4
:10ABC000CE0101960E945D10CE0101960E944D9427
:10ABD000CE0109960E944D94CE010F960E944D948D
:10ABE00040910A0250910B0260910C0270910D028B
:10ABF00022E0CE010F960E94DA956CE778E0CE0154
:10AC000009960E94B894BE01615F7F4FCE010996FC
:10AC10000E94B1966AE776E00E94C296BC01CE011E
:10AC200001960E943795CE0101960E945D10CE01DB
:10AC300001960E944D94CE0109960E944D94CE013A
:10AC40000F960E944D9410E001C011E08091A60C77
:10AC50009091A70C039708F08EC00E94702F0E945D
:10AC60009E0C62E375E0CE0101960E94B8944AE022
:10AC700050E060E070E0CE0101960E940C0BCE0126
:10AC800001960E944D948091A60C9091A70C01977B
:10AC900039F460E070E082EA9CE00E941D97F82E93
:10ACA0008091A60C9091A70C029709F055C068E618
:10ACB00077E0CE0101960E94B894BE016F5F7F4F8E
:10ACC00082EA9CE00E94FE96182FCE0101960E9417
:10ACD0004D94112309F440C061E070E082EA9CE0E9
:10ACE0000E941D97682FCE0101960E946B95BE01B0
:10ACF0006F5F7F4F86E99CE00E944A95CE010196E6
:10AD00000E944D9460E070E082EA9CE00E941D97F2
:10AD1000F82E8091790C8823F9F06CE878E0CE0168
:10AD200001960E94B89462EA7CE0CE0101960E94EE
:10AD3000B19662E375E00E94C296BC018BE39FE08E
:10AD40000E94F590CE0101960E944D9466E97CE048
:10AD50008BE39FE00E941E918F2D0E94B34D0E94B5
:10AD6000498A6093A80C7093A90C8093AA0C9093C5
:10AD7000AB0C0C94156421E030E040E050E062EA56
:10AD80007CE0CE0101960E949F97BE016F5F7F4FCE
:10AD900084E89CE00E943F95CE0101960E944D946C
:10ADA0006FEB78E0CE0109960E94B894BE01675F10
:10ADB0007F4F82EA9CE00E94FE96811116C06EECE5
:10ADC00075E0CE0101960E94B894BE016F5F7F4F7F
:10ADD00082EA9CE00E94FE9601E0811101C000E041
:10ADE000CE0101960E944D9401C001E0CE0109966A
:10ADF0000E944D94002309F4DCC042E050E062EA76
:10AE00007CE0CE0101960E94B409BE016F5F7F4FC6
:10AE100084E89CE00E943F95CE0101960E944D94EB
:10AE200064E87CE0CE0101960E943795CE01019640
:10AE30000E94370ACE0101960E944D9484E89CE05E
:10AE40000E94489820E030E048EC52E40E948F9B3A
:10AE50000E94C899AB01BC0140933802509339025B
:10AE600060933A0270933B022AE0CE0101960E9461
:10AE7000AE95CE0101960E94370ACE0101960E943E
:10AE80004D94609138027091390280913A0290910C
:10AE90003B028B019C0100591F45214031090134BF
:10AEA0001C4921053105D0F062E978E0CE01019618
:10AEB0000E94B89464E87CE0CE0101960E94B196AD
:10AEC00065EA78E00E94C296BC018AE89CE00E9494
:10AED0002295CE0101960E944D944DC019821A828E
:10AEE0001B821C821D821E821F8218860E94FB9973
:10AEF00020E030E048EC52E40E942F998E010F5F71
:10AF00001F4F22E047E00E94709DBC018AE89CE050
:10AF10000E94559565EB78E0CE0109960E94B894A1
:10AF20006AE87CE0CE0109960E94B19662EC78E076
:10AF30000E94C296BC018AE89CE00E942295CE0144
:10AF400009960E944D9410920C0C10920B0C80915B
:10AF5000380290913902A0913A02B0913B0280935D
:10AF6000630B9093640BA093650BB093660B80E02A
:10AF700090E00E94EA0965EA76E0CE0109960E9417
:10AF8000B8946AE87CE0CE0109960E94B196BC01B3
:10AF9000CE0101960E943795CE0101960E945D1068
:10AFA000CE0101960E944D94CE0109960E944D94C7
:10AFB000F3C067EC78E0CE0109960E94B894BE0118
:10AFC000675F7F4F82EA9CE00E94FE96811116C067
:10AFD0006DEC78E0CE0101960E94B894BE016F5FDF
:10AFE0007F4F82EA9CE00E94FE9601E0811101C041
:10AFF00000E0CE0101960E944D9401C001E0CE0117
:10B0000009960E944D94002309F475C026E030E0B3
:10B0100045E050E062EA7CE0CE0101960E949F97F5
:10B02000BE016F5F7F4F84E89CE00E943F95CE0198
:10B0300001960E944D9484E89CE00E943E986B012A
:10B040007C0169E278E0CE0109960E94B894BE01C5
:10B05000675F7F4F82EA9CE00E949697AC014F5F4A
:10B060005F4F62EA7CE0CE0101960E94B409BE0106
:10B070006F5F7F4F84E89CE00E943F95CE01019670
:10B080000E944D94CE0109960E944D9484E89CE064
:10B090000E943E98DB01E6E9F4E021E030E04091D7
:10B0A000940450919504421753075CF040815181FC
:10B0B0004A175B0711F4118210822F5F3F4F3296BF
:10B0C000EECFF601EE0FFF1FEC56FB4F718360834E
:10B0D00082E090E00E94332E62EA7CE0CE0101968D
:10B0E0000E943795CE0101960E94370ACE01019643
:10B0F0000E944D9449C063ED78E0CE0109960E940C
:10B10000B894BE01675F7F4F82EA9CE00E94FE9682
:10B11000811116C069ED78E0CE0101960E94B894C5
:10B12000BE016F5F7F4F82EA9CE00E94FE9601E0C5
:10B13000811101C000E0CE0101960E944D9401C032
:10B1400001E0CE0109960E944D94002331F1E6E919
:10B15000F4E081E090E02091940430919504281768
:10B16000390774F0863091051CF49183808305C003
:10B170009C012E5F3F4F3183208301963296EBCFA7
:10B1800082E090E00E94332E10920C0C10920B0C77
:10B1900080E090E00E94EA0910E06FED78E0CE01D7
:10B1A00009960E94B894BE01675F7F4F82EA9CE0D7
:10B1B0000E94FE96811116C067EE78E0CE010196DE
:10B1C0000E94B894BE016F5F7F4F82EA9CE00E94AC
:10B1D000FE9601E0811101C000E0CE0101960E94BF
:10B1E0004D9401C001E0CE0109960E944D940023C8
:10B1F00049F06FEE78E0CE0101960E94B8946BE7BB
:10B200007DE034C069EF78E0CE0109960E94B894E1
:10B21000BE01675F7F4F82EA9CE00E94FE9681112B
:10B2200016C060E079E0CE0101960E94B894BE019C
:10B230006F5F7F4F82EA9CE00E94FE9601E08111E1
:10B2400001C000E0CE0101960E944D9401C001E0D2
:10B25000CE0109960E944D940023A1F166E877E0A3
:10B26000CE0101960E94B89461E87DE0CE0101967E
:10B270000E94B196BC018AE89CE00E942295CE0112
:10B2800001960E944D9465EA76E0CE0109960E94EF
:10B29000B8946AE87CE0CE0109960E94B196BC01A0
:10B2A000CE0101960E943795CE0101960E945D1055
:10B2B000CE0101960E944D94CE0109960E944D94B4
:10B2C0000C94156467E079E0CE0109960E94B89469
:10B2D000BE01675F7F4F82EA9CE00E94FE9681116B
:10B2E00016C06CE079E0CE0101960E94B894BE01D0
:10B2F0006F5F7F4F82EA9CE00E94FE9601E0811121
:10B3000001C000E0CE0101960E944D9401C001E011
:10B31000CE0109960E944D940023D9F169E278E0AC
:10B32000CE0109960E94B894BE01675F7F4F82EA02
:10B330009CE00E949697AC014F5F5F4F62EA7CE011
:10B34000CE0101960E94B409BE016F5F7F4F84E871
:10B350009CE00E943F95CE0101960E944D94CE0143
:10B3600009960E944D9484E89CE00E943E986115E5
:10B37000710521F481E08093F70407C06130710505
:10B3800011F00C9415641092F7040E94832F0C9412
:10B39000156461E179E0CE0109960E94B894BE017E
:10B3A000675F7F4F82EA9CE00E94FE96811116C083
:10B3B00065E179E0CE0101960E94B894BE016F5F0D
:10B3C0007F4F82EA9CE00E94FE9601E0811101C05D
:10B3D00000E0CE0101960E944D9401C001E0CE0133
:10B3E00009960E944D94002309F464C043E050E0A4
:10B3F00062EA7CE0CE0101960E94B409BE016F5F53
:10B400007F4F84E89CE00E943F95CE0101960E9408
:10B410004D9464E87CE0CE0101960E943795CE0100
:10B4200001960E94370ACE0101960E944D94109217
:10B430000C0C10920B0C64E87CE081E89DE00E940B
:10B44000229520E030E048E050E06FE77BE081E8C3
:10B450009DE00E941E9780910B0C90910C0C0E9415
:10B46000EA0967EA76E0CE0101960E94B89461E8A5
:10B470007DE0CE0101960E94B196BC01CE010996F5
:10B480000E943795CE0101960E944D94BE01675FE0
:10B490007F4F82E191E10E94F59068EB7BE080E0D4
:10B4A00090E00E94788A6FE77BE0CE0101960E94CF
:10B4B000B89469C069E179E0CE0109960E94B89418
:10B4C000BE01675F7F4F82EA9CE00E94FE96811179
:10B4D00016C06EE179E0CE0101960E94B894BE01DB
:10B4E0006F5F7F4F82EA9CE00E94FE9601E081112F
:10B4F00001C000E0CE0101960E944D9401C001E020
:10B50000CE0109960E944D94002309F448C044E0FE
:10B5100050E062EA7CE0CE0101960E94B409BE01CF
:10B520006F5F7F4F84E89CE00E943F95CE010196BB
:10B530000E944D946FEA76E0CE0101960E94B89485
:10B5400064E87CE0CE0101960E94B196BC01CE0178
:10B5500009960E943795CE0101960E944D94BE0136
:10B56000675F7F4F82E191E10E94F59068EB7BE09D
:10B5700080E090E00E94788ABE01675F7F4FCE0135
:10B5800001960E943795CE0101960E94370ACE019E
:10B5900001960E944D94CE0109960C94F36363E2E8
:10B5A00079E0CE0109960E94B894BE01675F7F4F93
:10B5B00082EA9CE00E94FE96811116C068E279E062
:10B5C000CE0101960E94B894BE016F5F7F4F82EA60
:10B5D0009CE00E94FE9601E0811101C000E0CE01D6
:10B5E00001960E944D9401C001E0CE0109960E948F
:10B5F0004D940023A9F125E030E044E050E062EAF8
:10B600007CE0CE0101960E949F97BE016F5F7F4F45
:10B6100084E89CE00E943F95CE0101960E944D94E3
:10B6200084E89CE00E943E987093DA0B6093D90BFB
:10B6300062EA7CE0CE0101960E943795CE01019628
:10B640000E94370ACE0101960E944D9410920C0C74
:10B6500010920B0C80E090E00E94EA090C941564B3
:10B660006DE279E0CE0109960E94B894BE01675F51
:10B670007F4F82EA9CE00E94FE96811116C064E32F
:10B6800079E0CE0101960E94B894BE016F5F7F4FB2
:10B6900082EA9CE00E94FE9601E0811101C000E078
:10B6A000CE0101960E944D9401C001E0CE010996A1
:10B6B0000E944D94002321F127E030E046E050E065
:10B6C00062EA7CE0CE0101960E949F97BE016F5F07
:10B6D0007F4F84E89CE00E943F95CE0101960E9436
:10B6E0004D9484E89CE00E943E98672B21F41092D0
:10B6F000790C0C94E76381E08093790C0C94E763F8
:10B700006BE379E0CE010F960E94B894BE01615FB1
:10B710007F4F82EA9CE00E94FE9681112BC06EE36F
:10B7200079E0CE0109960E94B894BE01675F7F4F11
:10B7300082EA9CE00E94FE96811116C061E479E0E5
:10B74000CE0101960E94B894BE016F5F7F4F82EADE
:10B750009CE00E94FE9601E0811101C000E0CE0154
:10B7600001960E944D9401C001E0CE0109960E940D
:10B770004D9401C001E0CE010F960E944D9400232C
:10B7800009F42DC10AE0A02EB12CC12CD12C7601D8
:10B7900088248A9483E0982E6EE170E080E090E047
:10B7A0000E94788A809181020E940E8BB4010E94CF
:10B7B000BF9C882777FD8095982F0E94FB9920E0F9
:10B7C00030E040EA50E40E948F9B9B01AC01C7012E
:10B7D000B6010E9465986B017C01E1E0AE1AB108E8
:10B7E000D9F620E030E040E251E40E942F996B014D
:10B7F0007C0164E479E0CE0109960E94B894BE0110
:10B80000675F7F4F82EA9CE00E94FE96811116C01E
:10B8100068E479E0CE0101960E94B894BE016F5FA2
:10B820007F4F82EA9CE00E94FE9601E0811101C0F8
:10B8300000E0CE0101960E944D9401C001E0CE01CE
:10B8400009960E944D94002309F43FC020E030E0A7
:10B8500040E650E4C701B6010E948F9B9B01AC01FA
:10B8600060E070E080E890E40E946498AB01BC0165
:10B8700040932A0250932B0260932C0270932D0266
:10B8800022E0CE0101960E94DA95BE016F5F7F4FE4
:10B890008AE89CE00E943F95CE0101960E944D945B
:10B8A0006CE479E0CE0101960E94B8946AE87CE0ED
:10B8B000CE0101960E94B196BC018AE89CE00E94EC
:10B8C0002295CE0101960E944D946BE579E0CE0160
:10B8D00009960E94B894BE01675F7F4F82EA9CE0A0
:10B8E0000E94FE96811116C060E679E0CE010196B5
:10B8F0000E94B894BE016F5F7F4F82EA9CE00E9475
:10B90000FE9601E0811101C000E0CE0101960E9487
:10B910004D9401C001E0CE0109960E944D94002390
:10B9200009F43FC020E030E040E650E4C701B60132
:10B930000E948F9B9B01AC0160E070E080E291E48B
:10B940000E946498AB01BC014093260250932702E9
:10B95000609328027093290222E0CE0101960E9492
:10B96000DA95BE016F5F7F4F8AE89CE00E943F95A9
:10B97000CE0101960E944D9465E679E0CE010196D4
:10B980000E94B8946AE87CE0CE0101960E94B196CC
:10B99000BC018AE89CE00E942295CE0101960E949B
:10B9A0004D9465EA76E0CE0109960E94B8946AE863
:10B9B0007CE0CE0109960E94B196BC01CE010196B1
:10B9C0000E943795CE0101960E945D10CE0101962E
:10B9D0000E944D94CE0109960E944D94F6C665E7EB
:10B9E00079E0CE0101960E94B894BE016F5F7F4F4F
:10B9F00082EA9CE00E94FE96082FCE0101960E94EA
:10BA00004D94002309F46EC08091A60C9091A70C70
:10BA1000079708F4DAC646E050E062EA7CE0CE011F
:10BA200001960E94B409BE016F5F7F4F84E89CE0DD
:10BA30000E943F95CE0101960E944D9484E89CE0BF
:10BA40000E944898AB01BC0140930E0250930F0234
:10BA5000609310027093110221E0CE0109960E94BA
:10BA6000DA956CE678E0CE0101960E94B894BE01AA
:10BA7000675F7F4FCE0101960E94B1966AE776E03C
:10BA80000E94C296BC018AE89CE00E942295CE01E9
:10BA900001960E944D94CE0109960E944D946AE849
:10BAA0007CE0CE0101960E943795CE0101960E945E
:10BAB0005D10CE0101960E944D940E94498A28EEA5
:10BAC00033E040E050E00E94D29CCA01B9010E94DC
:10BAD000F9996093DF0B7093E00B8093E10B9093E7
:10BAE000E20B73C66CE779E0CE0101960E94B89430
:10BAF000BE016F5F7F4F82EA9CE00E94FE96082F96
:10BB0000CE0101960E944D940023E9F18091A60C8C
:10BB10009091A70C079708F458C646E050E062EAF7
:10BB20007CE0CE0101960E94B409BE016F5F7F4F99
:10BB300084E89CE00E943F95CE0101960E944D94BE
:10BB400084E89CE00E944898AB01BC0140930A0243
:10BB500050930B0260930C0270930D0221E0CE0112
:10BB600009960E94DA956CE778E0CE0101960E9472
:10BB7000B894BE01675F7F4FCE0101960E94B196D7
:10BB80006AE776E0F5C163E879E0CE0109960E94A4
:10BB9000B894BE01675F7F4F82EA9CE00E94FE96E8
:10BBA000811116C067E879E0CE0101960E94B89431
:10BBB000BE016F5F7F4F82EA9CE00E94FE9601E02B
:10BBC000811101C000E0CE0101960E944D9401C098
:10BBD00001E0CE0109960E944D94002309F45AC059
:10BBE0008091C2049091C3040E94112760931A02AD
:10BBF00070931B0280931C0290931D026093770B3D
:10BC00007093780B8093790B90937A0B80E090E09F
:10BC1000A0E8BFE38093220290932302A093240222
:10BC2000B093250280936F0B9093700BA093710BD0
:10BC3000B093720B8091790C8823A1F06AE57CE0C7
:10BC40008BE39FE00E94D29040911A0250911B0218
:10BC500060911C0270911D0222E030E08BE39FE0B6
:10BC60000E94279310920C0C10920B0C80E090E035
:10BC70000E94EA0940911A0250911B0260911C0235
:10BC800070911D0222E0CE0109960E94DA956BE8C0
:10BC900079E078C564E979E0CE0109960E94B8940C
:10BCA000BE01675F7F4F82EA9CE00E94FE96811191
:10BCB00016C06AE979E0CE0101960E94B894BE01EF
:10BCC0006F5F7F4F82EA9CE00E94FE9601E0811147
:10BCD00001C000E0CE0101960E944D9401C001E038
:10BCE000CE0109960E944D94002309F469C0809109
:10BCF000A60C9091A70C0797F8F046E050E062EA96
:10BD00007CE0CE0101960E94B409BE016F5F7F4FB7
:10BD100084E89CE00E943F95CE0101960E944D94DC
:10BD200084E89CE00E94489860934D0270934E0214
:10BD300080934F02909350028091BC040E94F62D94
:10BD400080914D0290914E02A0914F02B09150020D
:10BD50008093970B9093980BA093990BB0939A0BA9
:10BD60008091790C8823A1F068E47CE08BE39FE06C
:10BD70000E94D29040914D0250914E0260914F022C
:10BD80007091500222E030E08BE39FE00E94279305
:10BD900010920C0C10920B0C80E090E00E94EA09CB
:10BDA00040914D0250914E0260914F0270915002AD
:10BDB00022E0CE0109960E94DA9560EA79E0E2C4B9
:10BDC0006AEA79E0CE0109960E94B894BE01675FE5
:10BDD0007F4F82EA9CE00E94FE96811116C06FEAB6
:10BDE00079E0CE0101960E94B894BE016F5F7F4F4B
:10BDF00082EA9CE00E94FE9601E0811101C000E011
:10BE0000CE0101960E944D9401C001E0CE01099639
:10BE10000E944D94002309F4AEC08091A60C90912D
:10BE2000A70C069708F145E050E062EA7CE0CE01FD
:10BE300001960E94B409BE016F5F7F4F84E89CE0C9
:10BE40000E943F95CE0101960E944D9484E89CE0AB
:10BE50000E9448980E94119B6093490270934A0285
:10BE600080934B0290934C028091BE049091BF044A
:10BE70000E94A42A20E030E048E051E40E942F997B
:10BE80006093450270934602809347029093480264
:10BE90006093870B7093880B8093890B90938A0B28
:10BEA0008091490290914A02A0914B02B0914C02BC
:10BEB00080938F0B9093900BA093910BB093920B68
:10BEC0008091790C882381F167E37CE08BE39FE02C
:10BED0000E94D2902091490230914A0240914B0237
:10BEE00050914C0260E070E080E291E40E94F29B8D
:10BEF000AB01BC0121E030E08BE39FE00E94269380
:10BF000064EB79E08BE39FE00E940391409145024E
:10BF100050914602609147027091480222E030E061
:10BF20008BE39FE00E94279310920C0C10920B0C55
:10BF300080E090E00E94EA0940914502509146025B
:10BF4000609147027091480223E0CE0109960E9459
:10BF5000DA956BEB79E0CE0101960E94B894BE01B0
:10BF6000675F7F4FCE0101960E94B19663EE75E048
:10BF70000E94C29612C464EC79E0CE0109960E9438
:10BF8000B894BE01675F7F4F82EA9CE00E94FE96F4
:10BF9000811116C069EC79E0CE0101960E94B89437
:10BFA000BE016F5F7F4F82EA9CE00E94FE9601E037
:10BFB000811101C000E0CE0101960E944D9401C0A4
:10BFC00001E0CE0109960E944D94002309F49FC020
:10BFD0008091A60C9091A70C069708F145E050E0DF
:10BFE00062EA7CE0CE0101960E94B409BE016F5F57
:10BFF0007F4F84E89CE00E943F95CE0101960E940D
:10C000004D9484E89CE00E9448980E94119B6093A4
:10C010003D0270933E0280933F02909340028091D4
:10C02000BE049091BF040E94A42A20E030E048E0C2
:10C0300051E40E942F9960934102709342028093D1
:10C0400043029093440260938B0B70938C0B80930C
:10C050008D0B90938E0B80913D0290913E02A091AA
:10C060003F02B09140028093930B9093940BA09366
:10C07000950BB093960B8091790C882381F167E240
:10C080007CE08BE39FE00E94D29020913D023091B2
:10C090003E0240913F025091400260E070E080E239
:10C0A00091E40E94F29BAB01BC0121E030E08BE304
:10C0B0009FE00E94269364EB79E08BE39FE00E946F
:10C0C000039140914102509142026091430270916C
:10C0D000440222E030E08BE39FE00E94279310921D
:10C0E0000C0C10920B0C80E090E00E94EA09409149
:10C0F000410250914202609143027091440223E058
:10C10000CE0109960E94DA956EEC79E024CF67EDB6
:10C1100079E0CE0109960E94B894BE01675F7F4F17
:10C1200082EA9CE00E94FE96811116C06BED79E0D8
:10C13000CE0101960E94B894BE016F5F7F4F82EAE4
:10C140009CE00E94FE9601E0811101C000E0CE015A
:10C1500001960E944D9401C001E0CE0109960E9413
:10C160004D94002309F46FC060E08091C8040E94E0
:10C17000878B09E110E0C12CD12C76018091C80495
:10C180000E940E8BBC01882777FD8095982F0E9416
:10C19000FB999B01AC01C701B6010E9465986B0138
:10C1A0007C016AE070E080E090E00E94788A0150B3
:10C1B000110921F720E030E040EA50E4C701B60160
:10C1C0000E948F9B20E030E040E85AE30E948F9B62
:10C1D00020E030E048EC51E40E942F996093120275
:10C1E0007093130280931402909315026093AD0B29
:10C1F0007093AE0B8093AF0B9093B00B10920C0C1E
:10C2000010920B0C80E090E00E94EA09409112022B
:10C2100050911302609114027091150222E0CE0138
:10C2200009960E94DA9562E378E0CE0101960E94B9
:10C23000B894BE01675F7F4FCE0101960E94B19610
:10C2400064EF75E095CE6FED79E0CE0109960E941E
:10C25000B894BE01675F7F4F82EA9CE00E94FE9621
:10C26000811116C063EE79E0CE0101960E94B89468
:10C27000BE016F5F7F4F82EA9CE00E94FE9601E064
:10C28000811101C000E0CE0101960E944D9401C0D1
:10C2900001E0CE0109960E944D94002309F473C079
:10C2A00026E030E044E050E062EA7CE0CE01019616
:10C2B0000E949F97BE016F5F7F4F84E89CE00E94C1
:10C2C0003F95CE0101960E944D9484E89CE00E9427
:10C2D0003E986B017C0169E278E0CE0109960E94EC
:10C2E000B894BE01675F7F4F82EA9CE00E949697F8
:10C2F000AC014F5F5F4F62EA7CE0CE0101960E9485
:10C30000B409BE016F5F7F4F84E89CE00E943F95B7
:10C31000CE0101960E944D94CE0109960E944D9443
:10C320000091E4041091E50484E89CE00E944898A0
:10C33000AB01BC019801C6010E943532E3EEFBE07F
:10C3400021EB3BE04191519161917191D9014D9364
:10C350005D936D937D939D01BCE0EB30FB0791F7FE
:10C3600010920C0C10920B0C80E090E00E94EA09F5
:10C3700044E050E062EA7CE0CE0109960E94B409F4
:10C3800067EE79E0FFC168E07AE0CE0109960E948D
:10C39000B894BE01675F7F4F82EA9CE00E94FE96E0
:10C3A000811116C06CE07AE0CE0101960E94B8942B
:10C3B000BE016F5F7F4F82EA9CE00E94FE9601E023
:10C3C000811101C000E0CE0101960E944D9401C090
:10C3D00001E0CE0109960E944D94002309F45AC051
:10C3E0008091C2049091C3040E94112760931602A9
:10C3F00070931702809318029093190260937B0B3D
:10C4000070937C0B80937D0B90937E0B80E090E586
:10C41000A3ECB7E480931E0290931F02A093200226
:10C42000B09321028093730B9093740BA093750BC0
:10C43000B093760B8091790C8823A1F069E07CE0C1
:10C440008BE39FE00E94D290409116025091170218
:10C45000609118027091190222E030E08BE39FE0B6
:10C460000E94279310920C0C10920B0C80E090E02D
:10C470000E94EA0940911602509117026091180239
:10C480007091190222E0CE0109960E94DA9560E1CE
:10C490007AE078C16BE17AE0CE0109960E94B89407
:10C4A000BE01675F7F4F82EA9CE00E94FE96811189
:10C4B00016C06FE17AE0CE0101960E94B894BE01E9
:10C4C0006F5F7F4F82EA9CE00E94FE9601E081113F
:10C4D00001C000E0CE0101960E944D9401C001E030
:10C4E000CE0109960E944D94002309F48CC08091DE
:10C4F000A60C9091A70C0497F8F044E050E062EA93
:10C500007CE0CE0101960E94B409BE016F5F7F4FAF
:10C5100084E89CE00E943F95CE0101960E944D94D4
:10C5200084E89CE00E944898609322027093230262
:10C5300080932402909325028091220290912302FD
:10C54000A0912402B091250280936F0B9093700B01
:10C55000A093710BB093720B8091790C8823A1F09A
:10C5600060EF7BE08BE39FE00E94D290409122023B
:10C5700050912302609124027091250222E030E064
:10C580008BE39FE00E9426938091C2049091C304A4
:10C590000E94112760931A0270931B0280931C0261
:10C5A00090931D026093770B7093780B8093790BB7
:10C5B00090937A0B8091790C8823A1F066EE7BE052
:10C5C0008BE39FE00E94D29040911A0250911B028F
:10C5D00060911C0270911D0222E030E08BE39FE02D
:10C5E0000E94279310920C0C10920B0C80E090E0AC
:10C5F0000E94EA0940911A0250911B0260911C02AC
:10C6000070911D02B8C06BE27AE0CE0109960E94DB
:10C61000B894BE01675F7F4F82EA9CE00E94FE965D
:10C62000811116C06FE27AE0CE0101960E94B894A3
:10C63000BE016F5F7F4F82EA9CE00E94FE9601E0A0
:10C64000811101C000E0CE0101960E944D9401C00D
:10C6500001E0CE0109960E944D94002309F4B5C073
:10C660008091A60C9091A70C0497F8F044E050E05C
:10C6700062EA7CE0CE0101960E94B409BE016F5FC0
:10C680007F4F84E89CE00E943F95CE0101960E9476
:10C690004D9484E89CE00E94489860931E02709339
:10C6A0001F02809320029093210280911E0290919C
:10C6B0001F02A0912002B09121028093730B9093EE
:10C6C000740BA093750BB093760B8091790C882333
:10C6D000A1F06DEC7BE08BE39FE00E94D290409153
:10C6E0001E0250911F02609120027091210222E0EF
:10C6F00030E08BE39FE00E9426938091C2049091EA
:10C70000C3040E941127609316027093170280934E
:10C7100018029093190260937B0B70937C0B8093AB
:10C720007D0B90937E0B8091790C8823A1F063ECB4
:10C730007BE08BE39FE00E94D290409116025091E3
:10C740001702609118027091190222E030E08BE329
:10C750009FE00E94279310920C0C10920B0C80E02B
:10C7600090E00E94EA0940911602509117026091F0
:10C7700018027091190222E0CE0109960E94DA9502
:10C7800063E27AE0CE0101960E94B894BE01675F31
:10C790007F4FCE0101960E94B196BC018AE89CE0D1
:10C7A0000E942295CE0101960E944D94CE010996D9
:10C7B0000E944D946AE87CE0CE0101960E94379574
:10C7C000CE0101960E945D100CC0112371F162EA46
:10C7D0007CE0CE0101960E943795CE0101960E9421
:10C7E000370ACE0101960E944D941FC080E09DE063
:10C7F0000E948983182F882319F162E17BE086E982
:10C800009CE00E9455958091790C882359F06DEB3E
:10C810007BE08BE39FE00E94D290612F8BE39FE04F
:10C820000E943E91812F0E94B34D0E94498A6093DD
:10C83000A80C7093A90C8093AA0C9093AB0C49C0E0
:10C8400080917B0C882309F44FC00E94498A18EE1E
:10C85000C12E13E0D12EE12CF12CA70196010E94EC
:10C86000D29CCA01B9010E94F9992091DF0B309145
:10C87000E00B4091E10B5091E20B0E9464982091F3
:10C880000E0230910F0240911002509111020E944D
:10C89000D09A18164CF50E94498AA70196010E9469
:10C8A000D29CCA01B9010E94F9996093DF0B709381
:10C8B000E00B8093E10B9093E20B8091750C9091CB
:10C8C000760C0E94FB4A64E170E080E090E00E94F8
:10C8D000788A80917B0C8823E9F064E670E080E040
:10C8E00090E00E94788A16C00E94498AC090A80CE5
:10C8F000D090A90CE090AA0CF090AB0C6C197D09BB
:10C900008E099F0968347E4E8105910510F30E94BF
:10C910007C2FDFCFA6960FB6F894DEBF0FBECDBF3B
:10C92000DF91CF911F910F91FF90EF90DF90CF900B
:10C93000BF90AF909F908F900895CF92DF92EF922B
:10C94000FF92CF93DF93EC01882777FD8095982F96
:10C950000E94FB996B017C0120E030E040E45FE342
:10C960000E948F9B20E030E048E452E40E942F991F
:10C970000E94C899C617D707ECF020E030E040EAE3
:10C980005FE3C701B6010E948F9B20E030E048E4DE
:10C9900052E40E942F9920E030E040E85FE30E94DB
:10C9A00065980E94C89921E06C177D070CF420E07F
:10C9B000822F01C080E090E0DF91CF91FF90EF9057
:10C9C000DF90CF900895CF92DF92EF92FF92CF93B6
:10C9D000DF93EC016C597F4F882777FD8095982F66
:10C9E0000E94FB996B017C0120E030E040E45FE3B2
:10C9F0000E948F9B20E030E048E452E40E942F998F
:10CA00000E94C899C617D707ECF020E030E040EA52
:10CA10005FE3C701B6010E948F9B20E030E048E44D
:10CA200052E40E942F9920E030E040E85FE30E944A
:10CA300065980E94C89921E06C177D070CF420E0EE
:10CA4000822F01C080E090E0DF91CF91FF90EF90C6
:10CA5000DF90CF900895CF92DF92EF92FF92CF9325
:10CA6000DF93EC0164567109882777FD8095982F34
:10CA70000E94FB996B017C0120E030E040E45FE321
:10CA80000E948F9B20E030E048E452E40E942F99FE
:10CA90000E94C899C617D707ECF020E030E040EAC2
:10CAA0005FE3C701B6010E948F9B20E030E048E4BD
:10CAB00052E40E942F9920E030E040E85FE30E94BA
:10CAC00065980E94C89921E06C177D070CF420E05E
:10CAD000822F01C080E090E0DF91CF91FF90EF9036
:10CAE000DF90CF9008951F920F920FB60F921124EE
:10CAF0000BB60F922F933F934F935F936F937F9358
:10CB00008F939F93AF93BF93EF93FF938091A20D69
:10CB10000E94F58B2091A50D3091A60D2F5F3F4F00
:10CB20003093A60D2093A50D9091A40D953618F085
:10CB300096E09093A10D9091A10D9430C9F128F445
:10CB4000923069F09330D1F05EC0953009F451C055
:10CB5000963009F058C091E09093710E51C0811148
:10CB600052C02091A50D3091A60D2436310508F450
:10CB700042C01092710E1092A40D1CC0813009F0B9
:10CB800042C0E091A40D91E09E0F9093A40DF0E0BF
:10CB90002091A50D3091A60DEE0FFF1FE955F24F24
:10CBA000318320831092A60D1092A50D94E029C028
:10CBB000811117C0E091A40D91E09E0F9093A40DF8
:10CBC000F0E02091A50D3091A60DEE0FFF1FE95565
:10CBD000F24F318320831092A60D1092A50D93E0A1
:10CBE00010C02091A50D3091A60D2536310558F0C5
:10CBF00007C0811108C01092A60D1092A50D03C0A8
:10CC000095E09093A10D9091A30D992329F08111A6
:10CC100002C02F9A01C02F98FF91EF91BF91AF9161
:10CC20009F918F917F916F915F914F913F912F9144
:10CC30000F900BBE0F900FBE0F901F901895609332
:10CC4000A20D1092A30D0895F89482E08093B00095
:10CC50008093B10094E69093B3001092B200809359
:10CC6000700078948093A10D1092A40D8091A20D74
:10CC700060E00C94878B82E08093A10D1092A40D4C
:10CC800008958F929F92AF92BF92CF92DF92EF92D0
:10CC9000FF927B01BA0180E090E00E94F9994B017C
:10CCA0005C01B70180E090E00E94F9996B017C0182
:10CCB0002DEC3CEC4CE45FE30E948F9B9B01AC01AC
:10CCC000C501B4010E942B9987FD17C02DEC3CECE7
:10CCD0004CE45FE3C501B4010E948F9B9B01AC0152
:10CCE000C701B6010E942B99992787FD9095882747
:10CCF000990F881F9927019602C080E090E0FF906D
:10CD0000EF90DF90CF90BF90AF909F908F9008955D
:10CD10008F929F92AF92BF92CF92DF92EF92FF924B
:10CD20000F931F93CF93DF936C01EB01EC84FD8491
:10CD300086E0E816F1040CF443C0EE0CFF1C06E09C
:10CD400010E045EC842E4DE9942E4CE1A42E41E8F0
:10CD5000B42E8A859B85FC01E00FF11F4081518133
:10CD6000F8013497E80FF91F60817181C60189DFEE
:10CD7000FC01A501940163E971E080E091E00E946B
:10CD80009C9C4F01AA2497FCA094BA2C8626972637
:10CD9000A826B9260E5F1F4F0E151F05D1F68C82EF
:10CDA0009D82AE82BF8280E290E0998788878FEF74
:10CDB0009FEF9983888361E070E080E090E003C09A
:10CDC00060E070E0CB01DF91CF911F910F91FF9058
:10CDD000EF90DF90CF90BF90AF909F908F9008958D
:10CDE0000F931F93CF93DF938C01EB0187EA9DE0B4
:10CDF0009B878A878091A40D90E09D878C87809186
:10CE0000710E90E09F878E878091A10D853009F08B
:10CE100051C0C8011BD3882319F081E090E04CC0B9
:10CE2000BE01C801B0D78111F8CFBE01C80107D734
:10CE30008111F3CFBE01C8017ED28111EECFBE01B8
:10CE4000C801CCD48111E9CFBE01C80169D58111D7
:10CE5000E4CFBE01C80192D38111DFCFBE01C8016A
:10CE6000E3D18111DACFBE01C8012DD18111D5CF17
:10CE7000BE01C80145D68111D0CFBE01C8010E94B4
:10CE80005E6F8111CACFBE01C8011BD08111C5CF11
:10CE9000BE01C801A2D08111C0CFBE01C80138DFD8
:10CEA000672B682B692B09F0B8CF82E08093A10D26
:10CEB0001092A40D80E090E0DF91CF911F910F912F
:10CEC0000895AF92BF92CF92DF92EF92FF920F93AD
:10CED0001F93CF93DF93EB018091A40D883510F45D
:10CEE00080E070C0EA85FB858281938160E672E212
:10CEF0006ADD892BA9F3EA85FB858481958164E944
:10CF000071E1A9DD892B61F3BEE1CB2ED12C1DE1AE
:10CF1000E12EF12C00E010E08091A40D90E0049748
:10CF2000E816F906ACF5EA85FB85C701880F991F5D
:10CF3000E80FF91F8081918164EF71E044DD892B56
:10CF400079F25601AA0CBB1CEA85FB85EA0DFB1D94
:10CF50008081918168E572E07EDD892B21F0000FF0
:10CF6000111F01600DC0EA85FB85EA0DFB1D808164
:10CF7000918164EA76E06FDD892B49F0000F111F83
:10CF800082E0E80EF11C82E0C80ED11CC5CF76010C
:10CF900081E0E81AF108F594E794F986E8868AE2D8
:10CFA000E816F1040CF49CCFC801AA2797FDA095C0
:10CFB000BA2F8C839D83AE83BF8389E090E09983F1
:10CFC000888381E0DF91CF911F910F91FF90EF90C7
:10CFD000DF90CF90BF90AF900895AF92BF92CF9265
:10CFE000DF92EF92FF920F931F93CF93DF93EB01AA
:10CFF0008091A40D803211F080E05AC0EA85FB8553
:10D00000828193816CE271E0DEDC892BA9F3EA85F1
:10D01000FB85848195816EEE72E01DDD892B61F3C5
:10D0200006E010E0C12CD12C7601EA85FB85E00FEB
:10D03000F11F808191816CE271E0C5DC892BE1F206
:10D04000580182E0A80EB11CEA85FB85EA0DFB1DA4
:10D050008081918168E077E0FEDC892B39F0CC0C8F
:10D06000DD1CEE1CFF1C6894C0F810C0EA85FB852F
:10D07000EA0DFB1D808191816EEE72E0ECDC892B64
:10D0800009F4BACFCC0CDD1CEE1CFF1C0C5F1F4F4B
:10D090000E33110551F68EE090E099878887CC8297
:10D0A000DD82EE82FF828FE090E09983888381E0C9
:10D0B000DF91CF911F910F91FF90EF90DF90CF9074
:10D0C000BF90AF900895AF92BF92CF92DF92EF9250
:10D0D000FF920F931F93CF93DF93EB018091A40DE9
:10D0E000823251F5EA85FB858281938168E572E0A1
:10D0F0006ADC892B09F18091A40D90E08150904861
:10D10000880F991FEA85FB85E80FF91F80819181BF
:10D1100068E572E058DC892B79F0198618868FEF64
:10D120009FEFDC018C839D83AE83BF8386E090E01C
:10D130009983888381E06DC0EA85FB858281938134
:10D1400060E47FE140DC892B21F08091A40D8132E5
:10D1500010F480E05EC0EA85FB858481958160EAF9
:10D160007FE079DC892BA9F358E0A52EB12C03E0F0
:10D1700010E0C12CD12C7601EA85FB85C801880F0F
:10D18000991FE80FF91F8081918168E572E01BDC2F
:10D19000892BF9F2EA85FB85EA0DFB1D80819181DF
:10D1A00060E476E058DC892B39F0CC0CDD1CEE1CF9
:10D1B000FF1C6894C0F810C0EA85FB85EA0DFB1DD2
:10D1C0008081918166E272E046DC892B09F4C1CF4F
:10D1D000CC0CDD1CEE1CFF1C0E5F1F4F84E0A80E64
:10D1E000B11C0332110541F6EA85FB85EA5BFF4F6E
:10D1F0008081918168E572E0E6DB892B09F4A9CF93
:10D2000080E190E099878887CC82DD82EE82FF8280
:10D210008DCFDF91CF911F910F91FF90EF90DF9015
:10D22000CF90BF90AF900895AF92BF92CF92DF9210
:10D23000EF92FF920F931F93CF93DF93EB018091B7
:10D24000A40D893310F480E06BC0EA85FB858281F0
:10D25000938160E47FE1B7DB892BA9F3EA85FB8545
:10D260008481958160EA7FE0F6DB892B61F338E009
:10D27000A32EB12C03E010E0C12CD12C7601EA855D
:10D28000FB85C801880F991FE80FF91F80819181E4
:10D2900068E572E098DB892BB1F2EA85FB85EA0D3F
:10D2A000FB1D8081918160E476E0D5DB892B39F02C
:10D2B000CC0CDD1CEE1CFF1C6894C0F810C0EA8585
:10D2C000FB85EA0DFB1D8081918166E272E0C3DB84
:10D2D000892B09F4B8CFCC0CDD1CEE1CFF1C0E5FB3
:10D2E0001F4F84E0A80EB11C0B33110541F6EA85EF
:10D2F000FB85EA58FF4F8081918168E572E063DB2E
:10D30000892B09F4A0CF8CE190E099878887CC82A3
:10D31000DD82EE82FF828AE090E09983888381E05B
:10D32000DF91CF911F910F91FF90EF90DF90CF9001
:10D33000BF90AF9008956F927F928F929F92AF921D
:10D34000BF92CF92DF92EF92FF920F931F93CF93F2
:10D35000DF93EB018091A40D823208F45DC0EA8571
:10D36000FB85828193816EE571E02DDB892B09F4C9
:10D3700053C063E0A62EB12C02E010E0C12CD12CEA
:10D38000760135018091A40D90E0A816B906CCF580
:10D390004801880C991CEA85FB85E80DF91D808100
:10D3A00091816EE977E00FDB892B39F0CC0CDD1C25
:10D3B000EE1CFF1C6894C0F80FC0EA85FB85E80DE1
:10D3C000F91D808191816EEE72E0FDDA892B21F1E9
:10D3D000CC0CDD1CEE1CFF1CC501880F991FEA85D3
:10D3E000FB85E80FF91F808191816EE571E033DBE9
:10D3F00022E0A20EB11C892B19F00E5F1F4FC1CF86
:10D400008301015011091595079519870887003187
:10D41000110524F41986188680E009C0CC82DD82CB
:10D42000EE82FF828CE090E09983888381E0DF9137
:10D43000CF911F910F91FF90EF90DF90CF90BF9011
:10D44000AF909F908F907F906F900895AF92BF9212
:10D45000CF92DF92EF92FF920F931F93CF93DF93C0
:10D46000EB01EA85FB858281938168E273E2ABDAA6
:10D47000892B11F480E077C08091A40D843009F5E8
:10D48000EA85FB85848195816AEC78E0E4DA892B72
:10D49000C1F0EA85FB858681978160E372E093DACB
:10D4A000892B79F0198618868FEF9FEFDC018C832A
:10D4B0009D83AE83BF8383E090E09983888381E07E
:10D4C00052C08091A40D8434A8F2EA85FB85848142
:10D4D000958164E971E1BFDA892B61F206E010E021
:10D4E000C12CD12C7601EA85FB85E00FF11F8081EC
:10D4F000918160E372E067DA892B09F4BBCF5801B0
:10D5000082E0A80EB11CEA85FB85EA0DFB1D808137
:10D5100091816AE976E09FDA892B39F0CC0CDD1C29
:10D52000EE1CFF1C6894C0F810C0EA85FB85EA0D6C
:10D53000FB1D8081918160E372E08DDA892B09F413
:10D5400099CFCC0CDD1CEE1CFF1C0C5F1F4F063866
:10D55000110549F680E290E099878887CC82DD82C8
:10D56000EE82FF82A8CFDF91CF911F910F91FF90A4
:10D57000EF90DF90CF90BF90AF9008958F929F92E1
:10D58000AF92BF92CF92DF92EF92FF920F931F93D1
:10D59000CF93DF9300D01F92CDB7DEB74B01DB01F5
:10D5A0001A96ED91FC911B97828193816EEA7DE042
:10D5B0000ADA892B11F480E08FC0D4011A96ED911C
:10D5C000FC911B978481958166ED76E0FCD9892BCF
:10D5D00091F3E6E0EE2EF12C20E030E040E050E068
:10D5E000A12CB12CC12CD12CD4011A96ED91FC9117
:10D5F0001B97EE0DFF1D8081918166EF71E02983FD
:10D600003A834B835C83DFD9892BA9F287010E5FB4
:10D610001F4FD4011A96ED91FC911B97E00FF11F5B
:10D62000808191816CED74E016DA29813A814B8119
:10D630005C81892B39F0B501C60101E00E942A9D69
:10D6400021601CC0D4011A96ED91FC911B97E00F4C
:10D65000F11F8081918160E971E029833A834B83D6
:10D660005C83F9D929813A814B815C81892B09F44A
:10D67000A2CFB501C60101E00E942A9D5B016C01A9
:10D68000B4E0EB0EF11CE6ECEE16F10409F0ACCFC1
:10D69000D40114962C93149715963C9315971696CF
:10D6A0004C93169717965C931797B501C60100E245
:10D6B0000E94459D12962C93129713963C931397B4
:10D6C00085E090E011969C938E9380E390E019960C
:10D6D0009C938E93189781E00F900F900F900F906E
:10D6E000DF91CF911F910F91FF90EF90DF90CF903E
:10D6F000BF90AF909F908F9008958F929F92AF921E
:10D70000BF92CF92DF92EF92FF920F931F93CF932E
:10D71000DF937A016901DA01CD91DC91FB01848507
:10D720009585C817D9070CF047C0CE01880F991FFF
:10D730000284F385E02DE80FF91FA080B180C1704D
:10D74000DD27F1E0CF27209719F484E690E002C0AE
:10D750008CE99FEF4801880E991EB401C501EDD8F0
:10D76000892B89F4800E911EB401C501E6D8892B5E
:10D7700069F4B401600F711FC501DFD8892BF9F07E
:10D7800023E030E005C021E030E002C022E030E0DC
:10D79000D6018D919C91119701968217930744F0C1
:10D7A000F60111821082D7018D919C9111970196FB
:10D7B0008D939C93CE0105C081E090E002C08FEF75
:10D7C0009FEFDF91CF911F910F91FF90EF90DF902E
:10D7D000CF90BF90AF909F908F9008954F925F929F
:10D7E0006F927F928F929F92AF92BF92CF92DF9271
:10D7F000EF92FF920F931F93CF93DF9300D01F926E
:10D80000CDB7DEB76C017B011C821B8281E090E00A
:10D810009A8389838091A40D8D3010F480E06BC0D1
:10D8200009E713E09E012D5F3F4FAE014F5F5F4F51
:10D83000C60163DF892B91F79E012D5F3F4FAE013B
:10D840004F5F5F4FB701C60158DF019739F79E015F
:10D850002D5F3F4FAE014F5F5F4FB701C6014DDFF8
:10D86000892BE1F6412C512C3201A12CB12C809155
:10D87000A40D90E029813A81281739078CF509E732
:10D8800013E09E012D5F3F4FAE014F5F5F4FB70129
:10D89000C60133DF4C019E012D5F3F4FAE014F5F4C
:10D8A0005F4FB701C60129DF21E08216910451F4D0
:10D8B000892B09F0B3CF440C551C661C771C689467
:10D8C00040F80AC0892809F0A9CF019709F0A6CF2E
:10D8D000440C551C661C771C8FEFA81AB80AC7CFDA
:10D8E000F701B186A086448255826682778281E004
:10D8F00090E0918380830F900F900F900F90DF91B5
:10D90000CF911F910F91FF90EF90DF90CF90BF903C
:10D91000AF909F908F907F906F905F904F90089501
:10D920002F923F924F925F926F927F928F929F922F
:10D93000AF92BF92CF92DF92EF92FF920F931F931D
:10D94000CF93DF9300D01F92CDB7DEB76C017B0180
:10D950001C821B82DB011C968D919C911D971816D1
:10D96000190614F080E0B5C0DB011A96ED91FC9128
:10D970001B9782E090E09A838983828193816AE693
:10D980007AE021D8892B71F3D7011A96ED91FC9199
:10D990001B9789819A819C012F5F3F4F3A8329838E
:10D9A000880F991FE80FF91F8081918169E773E063
:10D9B00052D8892BB9F20CEB11E09E012D5F3F4F3D
:10D9C000AE014F5F5F4FB701C60197DE892B51F65D
:10D9D0009E012D5F3F4FAE014F5F5F4FB701C60104
:10D9E0008CDE019709F0BECF212C312C2101A12C16
:10D9F000B12C29813A81F70184859585281739074B
:10DA00000CF05CC00CEB11E09E012D5F3F4FAE01AE
:10DA10004F5F5F4FB701C60170DE3C01B3E0AB164C
:10DA2000B10489F00CEB11E09E012D5F3F4FAE0178
:10DA30004F5F5F4FB701C60160DE4C01E3E0AE16F9
:10DA4000B104F9F40FC00CEB11E09E012D5F3F4FC4
:10DA5000AE014F5F5F4FB701C6014FDE6816790612
:10DA600009F380CF0CEB11E09E012D5F3F4FAE011B
:10DA70004F5F5F4FB701C60140DE8816990609F077
:10DA800071CF6114710459F48A94892809F06ACF1E
:10DA9000220C331C441C551C689420F80BC06A945B
:10DAA000672809F05FCF892809F05CCF220C331C6E
:10DAB000441C551CAFEFAA1ABA0A9BCFB186A086A8
:10DAC000248235824682578282E090E0918380836F
:10DAD00081E00F900F900F900F90DF91CF911F91E9
:10DAE0000F91FF90EF90DF90CF90BF90AF909F90FD
:10DAF0008F907F906F905F904F903F902F90089500
:10DB0000AF92BF92CF92DF92EF92FF920F931F934B
:10DB1000CF93DF93EB01EA85FB858281938168E8EF
:10DB200073E10E94E364892B11F480E07DC0809151
:10DB3000A40D843019F5EA85FB85848195816AEC12
:10DB400078E00E942B65892BC9F0EA85FB858681E8
:10DB5000978160E372E00E94E364892B79F0198673
:10DB600018868FEF9FEFDC018C839D83AE83BF838C
:10DB700087E090E09983888381E056C08091A40D6E
:10DB8000843498F2EA85FB858481958168E873E1A5
:10DB90000E942B65892B49F206E010E0C12CD12CA4
:10DBA0007601EA85FB85E00FF11F8081918160E3BA
:10DBB00072E00E94E364892B09F4B7CF580182E038
:10DBC000A80EB11CEA85FB85EA0DFB1D80819181C1
:10DBD00060E476E00E942B65892B39F0CC0CDD1CCB
:10DBE000EE1CFF1C6894C0F811C0EA85FB85EA0DA5
:10DBF000FB1D8081918160E372E00E942B65892B7F
:10DC000009F493CFCC0CDD1CEE1CFF1C0C5F1F4FE6
:10DC10000638110531F680E290E099878887CC823A
:10DC2000DD82EE82FF82A4CFDF91CF911F910F9111
:10DC3000FF90EF90DF90CF90BF90AF9008958F92BC
:10DC40009F92AF92BF92CF92DF92EF92FF920F938B
:10DC50001F93CF93DF93EB018091A40D8A3108F4D9
:10DC60007AC0EA85FB85808191818032934050F4AF
:10DC7000198618868FEF9FEFDC018C839D83AE831E
:10DC8000BF836FC0828193816CEA7DE00E94E36470
:10DC9000892B09F460C0EA85FB85848195816CEA53
:10DCA0007DE00E94E364892B09F455C054E0A52E61
:10DCB000B12C03E010E0C12CD12C76018091A40D91
:10DCC00090E0A816B906E4F5EA85FB85C801880F3F
:10DCD000991FE80FF91F8081918166EB73E00E9424
:10DCE0002B65892B61F14501880C991CEA85FB8520
:10DCF000E80DF91D8081918160E679E00E94E3647E
:10DD0000892B39F0CC0CDD1CEE1CFF1C6894C0F88C
:10DD100010C0EA85FB85E80DF91D808191816CEBCF
:10DD200072E00E94E364892BB1F0CC0CDD1CEE1C88
:10DD3000FF1C0E5F1F4F82E0A80EB11CBFCF8501F4
:10DD40000150110915950795198708870C301105A1
:10DD500024F41986188680E009C0CC82DD82EE8228
:10DD6000FF828BE090E09983888381E0DF91CF91FF
:10DD70001F910F91FF90EF90DF90CF90BF90AF90E9
:10DD80009F908F9008958F929F92AF92BF92CF9263
:10DD9000DF92EF92FF920F931F93CF93DF93EB01EC
:10DDA0008091A40D8A3108F471C0EA85FB858081D9
:10DDB0009181843F914060F4198618868FEF9FEF20
:10DDC000DC018C839D83AE83BF838BE090E066C0D3
:10DDD0008281938160E679E00E94E364892B09F4F3
:10DDE00055C073E0A72EB12C02E010E0C12CD12C5D
:10DDF00076018091A40D90E0A816B906E4F5EA85B5
:10DE0000FB85C801880F991FE80FF91F8081918158
:10DE100068E572E00E942B65892B61F14501880C51
:10DE2000991CEA85FB85E80DF91D8081918160EBE5
:10DE300074E00E94E364892B39F0CC0CDD1CEE1CED
:10DE4000FF1C6894C0F810C0EA85FB85E80DF91D39
:10DE50008081918168E572E00E94E364892BB1F0D2
:10DE6000CC0CDD1CEE1CFF1C0E5F1F4F82E0A80EC9
:10DE7000B11CBFCF85010150110915950795198770
:10DE800008870C30110524F41986188680E009C033
:10DE9000CC82DD82EE82FF8284E090E099838883E9
:10DEA00081E0DF91CF911F910F91FF90EF90DF9074
:10DEB000CF90BF90AF909F908F900895AF92BF92F8
:10DEC000CF92DF92EF92FF920F931F93CF93DF9346
:10DED000EB018091A40D863410F480E086C0EA85C1
:10DEE000FB85828193816EEE72E00E94E364892B50
:10DEF000A1F3EA85FB85848195816EEE72E00E9434
:10DF00002B65892B51F3EA85FB858681978162E237
:10DF10007BE00E94E364892B01F3EA85FB85808521
:10DF2000918562E27BE00E942B65892BB1F25CE077
:10DF3000A52EB12C05E010E0C12CD12C7601EA858C
:10DF4000FB85C801880F991FE80FF91F8081918117
:10DF50006EEE72E00E94E364892B09F4BECFEA857D
:10DF6000FB85EA0DFB1D8081918166E678E00E94C9
:10DF70002B65892B39F0CC0CDD1CEE1CFF1C689442
:10DF8000C0F811C0EA85FB85EA0DFB1D80819181F7
:10DF90006EEE72E00E942B65892B09F49ECFCC0CAB
:10DFA000DD1CEE1CFF1C0E5F1F4F84E0A80EB11C91
:10DFB0000534110521F6EA85FB85E657FF4F808180
:10DFC00091816EEE72E00E94E364892B09F485CFA3
:10DFD00080E290E099878887CC82DD82EE82FF82A2
:10DFE00088E090E09983888381E0DF91CF911F9151
:10DFF0000F91FF90EF90DF90CF90BF90AF9008957A
:10E00000FB018081883251F028F4803139F082326E
:10E0100039F404C08B3311F0823411F481E0089597
:10E0200080E00895FC017783668314821582108254
:10E0300089E0818381E0828383830895CF93DF9396
:10E04000EC01F0DF1B8A1A8ADF91CF910895FC0161
:10E0500085810895CF93DF93EB0167E0CE010E94A5
:10E06000A28991E02F81821390E0892FDF91CF91D7
:10E070000895EF92FF920F931F93CF93DF93EC01DC
:10E080008B01E42E8E819F810E94D788F12C41E084
:10E09000B8018E819F810E940A89882351F0FE1069
:10E0A00005C0B801CE01D6DF811104C0F394EF148E
:10E0B00070F780E0DF91CF911F910F91FF90EF906B
:10E0C0000895CF92DF92EF92FF920F931F93CF9319
:10E0D000DF931F921F92CDB7DEB76C01F42EE52EB1
:10E0E000FC018681978169837A830E94BF87698159
:10E0F0007A81882311F1F601868197810E94AE888A
:10E1000040E06EEBF601868197810E9452880F2DC8
:10E110001E2D89E0F82EF601868197810E94938852
:10E12000F80181938F01FA94B1F7F6018681978106
:10E130000E94BF8791E0813009F090E0892F0F9015
:10E140000F90DF91CF911F910F91FF90EF90DF9093
:10E15000CF900895CF93DF93EA01B3DF882351F086
:10E1600068E0CE010E94A28991E02885821390E0A8
:10E17000892F01C080E0DF91CF910895EF92FF9247
:10E180000F931F93CF93DF93EC018B017A018E8164
:10E190009F810E94BF87B8018E819F810E94AE88B7
:10E1A00040E06EE48E819F810E94528840E0F7013A
:10E1B00062818E819F810E94528840E0F7016381D5
:10E1C0008E819F810E945288F8018081803139F0D0
:10E1D00040E0F70164818E819F810E9452888E8188
:10E1E0009F810E94BF87B8018E819F810E94AE8867
:10E1F000488168E48E819F810E94528864E170E0CA
:10E2000080E090E00E94788A8881882331F06AE07B
:10E2100070E080E090E00E94788A8E819F81DF919B
:10E22000CF911F910F91FF90EF900C94BF87EF92C9
:10E23000FF921F93CF93DF931F921F92CDB7DEB74C
:10E240007C01FC018681978169837A830E94BF8764
:10E2500069817A81F701868197810E94AE8840E0CA
:10E2600064EBF701868197810E945288F7018681CD
:10E2700097810E942A88182FF701868197810E9432
:10E28000BF8781E0111180E00F900F90DF91CF9157
:10E290001F91FF90EF900895CF93DF93CDB7DEB736
:10E2A00029970FB6F894DEBF0FBECDBFFB012081CA
:10E2B0002031C9F0AE014F5F5F4F4CDF882379F00A
:10E2C0008D818F3351F020F48F3149F489E00CC0F7
:10E2D0008F3539F08F3739F002C08AE005C080E011
:10E2E00003C08BE001C08CE029960FB6F894DEBF26
:10E2F0000FBECDBFDF91CF910895FF920F931F9373
:10E30000CF93DF93CDB7DEB728970FB6F894DEBF73
:10E310000FBECDBF8C01FC01868197810E94D788FA
:10E32000F8011482158241E0BE016F5F7F4FF80152
:10E33000868197810E940A898823C1F1BE016F5F9F
:10E340007F4FC80187DE882371F3F8018081811136
:10E3500007C0BE016F5F7F4FC80169DF811122C016
:10E36000F801F180BE016F5F7F4FC80195DF8F1507
:10E3700018F4F801818105C0BE016F5F7F4FC801AD
:10E380008BDFF801818384818F5F8483BE016F5F9F
:10E390007F4FC80135DE882331F2F80185818F5F18
:10E3A0008583C1CF81E0F8018083DACF28960FB64C
:10E3B000F894DEBF0FBECDBFDF91CF911F910F91BB
:10E3C000FF900895DF92EF92FF920F931F93CF93E8
:10E3D000DF93CDB7DEB762970FB6F894DEBF0FBEFE
:10E3E000CDBF8C017B01D22E493028F0342F4D3027
:10E3F00018F03CE001C039E0B701C8013A8B4CDFAE
:10E400003A89831709F458C0AE014F5F5F4FB701D7
:10E41000C8013A8B9FDE3A89882309F44FC0F7017F
:10E420008081803109F448C03B3041F03C3021F01C
:10E430003A3031F48FE305C08FE703C08FE501C0A8
:10E440008FE18D83AE014F5F5F4FB701C8013A8BFB
:10E4500095DEF80191813A89832F391708F4892FC5
:10E46000F8018183D11028C0381730F53183E12CB1
:10E47000F12CF801848190E0E816F906ECF44E2DB9
:10E48000BE01665F7F4FC801F4DDF801D180BE0197
:10E49000665F7F4FC80100DF8D1518F4F801818198
:10E4A00005C0BE01665F7F4FC801F6DEF8018183BB
:10E4B000FFEFEF1AFF0ADDCF81E001C080E0629636
:10E4C0000FB6F894DEBF0FBECDBFDF91CF911F9185
:10E4D0000F91FF90EF90DF900895EF92FF920F93CE
:10E4E0001F93CF93DF93CDB7DEB728970FB6F8947D
:10E4F000DEBF0FBECDBF8C01693020F06D3018F04B
:10E500006CE001C069E0F8016183E12CF12CF801B5
:10E51000848190E0E816F90694F44E2DBE016F5FF9
:10E520007F4FC801A6DD21E0F8014181BE016F5F88
:10E530007F4FC80147DFFFEFEF1AFF0AE8CF2896A9
:10E540000FB6F894DEBF0FBECDBFDF91CF911F9104
:10E550000F91FF90EF900895FC01868197810E94B2
:10E560002A8891E0813009F090E0892F08958F92F8
:10E570009F92AF92BF92CF92DF92EF92FF920F9352
:10E580001F93CF93DF93EC016950633048F4E62F7B
:10E59000F0E0EE0FFF1FEF5BF54F0081118102C02D
:10E5A0000EEE12E08B818823E1F08881811119C081
:10E5B0000E94498A6B017C014801AA2497FCA0941F
:10E5C000BA2CCE01C9DF81111FC00E94498A681987
:10E5D00079098A099B096C157D058E059F05A0F4B4
:10E5E000F0CFB801882777FD8095982FDF91CF91E4
:10E5F0001F910F91FF90EF90DF90CF90BF90AF9061
:10E600009F908F900C94788ADF91CF911F910F91FA
:10E61000FF90EF90DF90CF90BF90AF909F908F9042
:10E620000895CF93DF93EC018E819F810E94BF8775
:10E630008E819F810E94D488488164E48E819F816D
:10E640000E9452888A81882329F06981CE01DF9156
:10E65000CF918DCFDF91CF910895FA01208148E0CD
:10E66000249F90011124818190E0982F8827990F91
:10E67000990F990F282B392BDB018C918031C1F434
:10E68000678170E08681AB01481B5109CA019695EC
:10E69000982F8827979587950E94BF9C6051710994
:10E6A000207F53E0220F331F5A95E1F7260F371FC3
:10E6B000C9010895EF92FF920F931F93CF93DF93B9
:10E6C000CDB7DEB729970FB6F894DEBF0FBECDBF2A
:10E6D0008C017B01AE014F5F5F4F3CDD882339F039
:10E6E000AE014F5F5F4FB701C801B7DF02C080E8DE
:10E6F00094EE29960FB6F894DEBF0FBECDBFDF9122
:10E70000CF911F910F91FF90EF900895813824EEE3
:10E7100092076CF0BC01882777FD8095982F0E94A6
:10E72000FB9920E030E040E05CE30C948F9B60E0DC
:10E7300070E08EEF92EC0895BDDFE8CF0F931F934A
:10E74000CF93DF93CDB7DEB728970FB6F894DEBF2F
:10E750000FBECDBF8C01462FBE016F5F7F4F89DC9E
:10E76000882331F0BE016F5F7F4FC801E5DF04C031
:10E7700060E070E08EEF92EC28960FB6F894DEBF62
:10E780000FBECDBFDF91CF911F910F91089527E369
:10E790003AE0FC0131832083089527E33AE0FC014D
:10E7A000318320830C9462980F931F93CF93DF9350
:10E7B0008C01EB0188E2FB0111928A95E9F74BE0AD
:10E7C00050E067E47AE0CE010E94FE9F1B8641E0A4
:10E7D00050E060E070E04C875D876E877F87F801CE
:10E7E000458956896789708D488B598B6A8B7B8BDD
:10E7F00042E050E060E070E04C8B5D8B6E8B7F8B75
:10E800001CA21DA21EA21FA240E050E068E474E416
:10E81000488F598F6A8F7B8F40E050E068E474EC3A
:10E820004C8F5D8F6E8F7F8F4DEC5CEC6CE47EE3E4
:10E8300048A359A36AA37BA3DF91CF911F910F91A6
:10E84000089523E53AE0FC0131832083458B568B04
:10E85000678B708F0895CF93DF931F921F92CDB770
:10E86000DEB782E79EE02A8349836BD24981642F19
:10E8700082E79EE01FD22A81622F82E79EE01AD2B1
:10E8800082E79EE00F900F90DF91CF91D8C20F9357
:10E890001F93CF93DF938C01EB01262F41E06EE1B4
:10E8A000DADFF801D483C383C038D10509F45BC033
:10E8B000DCF4C034D105A9F1C036D10509F442C059
:10E8C000A09709F08AC080E090E8A9E8B4E48093BA
:10E8D000FF0490930005A0930105B093020580E02A
:10E8E00090E0A5E7B4E471C0C03CD10509F44CC088
:10E8F000C03ED10509F459C0C03AD10509F06DC038
:10E9000080E090E0A8ECB3E48093FF0490930005CE
:10E91000A0930105B093020580E090E0AFE7B3E477
:10E9200054C080E090ECA5E5B4E48093FF0490939C
:10E930000005A0930105B093020580E090E0AEE3EE
:10E94000B4E443C080E090E8A7E2B4E48093FF041D
:10E9500090930005A0930105B093020580E090E03C
:10E96000A6E1B4E432C080E090E0A1EEB3E480938D
:10E97000FF0490930005A0930105B093020580E089
:10E9800090E0A8ECB3E421C080E090E0A5EAB3E415
:10E990008093FF0490930005A0930105B0930205B6
:10E9A00080E090E8A3E9B3E410C080E090E0A6E640
:10E9B000B3E48093FF0490930005A0930105B09306
:10E9C000020580E090E0ADE4B3E48093FB04909313
:10E9D000FC04A093FD04B093FE04DF91CF911F913E
:10E9E0000F910895CF93DF93EC0182E79EE0A0D1D1
:10E9F00020E042E06EE1CE012EDF60E270E0CE0169
:10EA000046DF81E0DF91CF9108956F927F928F92E0
:10EA10009F92AF92BF92CF92DF92EF92FF920F93AD
:10EA20001F93CF93DF93EC016EE182E79EE089D1E3
:10EA3000E091720EF091730E0190F081E02D63E091
:10EA400082E79EE0199582E79EE0F9D146E06EE10B
:10EA500082E79EE0F0D182E79EE0D5D00697DCF316
:10EA600082E79EE0D8D0682E82E79EE0D4D0782E50
:10EA700082E79EE0D0D0C82E82E79EE0CCD0D82E90
:10EA800082E79EE0C8D0882E82E79EE0C4D0982E10
:10EA9000B62CA12CA728B501882777FD8095982F43
:10EAA0000E94FB996D837E838F839887F82CE12CDD
:10EAB000E928B701882777FD8095982F0E94FB9958
:10EAC00069877A878B879C871C2D00E00D29B80108
:10EAD000882777FD8095982F0E94FB996D877E8708
:10EAE0008F87988B198A1A8A1B8A1C8ADF91CF918B
:10EAF0001F910F91FF90EF90DF90CF90BF90AF905C
:10EB00009F908F907F906F900895CF92DF92EF92B9
:10EB1000FF920F931F93CF93DF938C01EB0184E25D
:10EB2000FB0111928A95E9F7C8016FDF84E290E05A
:10EB3000A0E0B0E088839983AA83BB83F80185892C
:10EB40009689A789B08D8C839D83AE83BF8382E035
:10EB500090E0A0E0B0E088879987AA87BB87188AF1
:10EB6000198A1A8A1B8AC090FF04D0900005E09091
:10EB70000105F0900205A7019601658176818781E4
:10EB800090850E942F9920E030E048EC52E40E94EA
:10EB90008F9B6C8B7D8B8E8B9F8BA7019601F801D1
:10EBA00061857285838594850E942F9920E030E0ED
:10EBB00048EC52E40E948F9B688F798F8A8F9B8FDD
:10EBC0002091FB043091FC044091FD045091FE041F
:10EBD000F80165857685878590890E942F9920E0C8
:10EBE00030E048EC52E40E948F9B6C8F7D8F8E8FBB
:10EBF0009F8F81E0DF91CF911F910F91FF90EF9058
:10EC0000DF90CF9008958091A20E90E02091A30E06
:10EC1000821B910908952091A30E8091A20E2817BE
:10EC200050F4E22FF0E0EC55F14F808190E02F5F3F
:10EC30002093A30E08958FEF9FEF0895E091A30E08
:10EC40008091A20EE81730F4F0E0EC55F14F80818E
:10EC500090E008958FEF9FEF08950895CF92DF928F
:10EC6000EF92FF920F931F93CF93DF937C01CB0121
:10EC70008A0120917E0E222389F0EB016B01C40EE4
:10EC8000D51ECC15DD0561F06991D701ED91FC91A0
:10EC90000190F081E02DC7011995F3CF642F91D138
:10ECA000C801DF91CF911F910F91FF90EF90DF90FE
:10ECB000CF900895CF93DF931F92CDB7DEB76983CE
:10ECC00020917E0E2223D1F020917F0E203240F041
:10ECD00021E030E0FC013383228380E090E014C027
:10ECE0008091800EE82FF0E0EF57F14F99819083EB
:10ECF0008F5F8093800E80937F0E04C061E0CE0111
:10ED000001965FD181E090E00F90DF91CF9108955F
:10ED1000FC011382128248EE53E060E070E044830D
:10ED200055836683778381E69AE091838083089593
:10ED30001092A30E1092A20E1092800E10927F0ECF
:10ED400083C081E080937E0E6093A10E1092800EAE
:10ED500010927F0E0895F5CF0F93062F21E040917A
:10ED60007F0E61E87EE08091A10ED4D01092800EDB
:10ED700010927F0E10927E0E0F9108958F929F92A7
:10ED8000AF92BF92CF92DF92EF92FF920F931F93B9
:10ED9000CF93DF93EC01F62ED42E48015901EE20DB
:10EDA00009F1CFDF1E2D143008F013E01150B8F038
:10EDB000E881F98128E0129FB0011124A501940196
:10EDC00004C056954795379527956A95D2F7CA019D
:10EDD000B9010190F081E02DCE011995E7CF60E0F7
:10EDE000CE01BADF4D2D413208F040E22C2D64EA0D
:10EDF0007EE08F2D47D01092A30E8093A20EDF915C
:10EE0000CF911F910F91FF90EF90DF90CF90BF9027
:10EE1000AF909F908F900895CF92EF920F931F9392
:10EE2000C22EE12C00E010E09801A8DF1F910F91A5
:10EE3000EF90CF90089521E0EFCF21E0EDCF61E09A
:10EE40008BCF82E79EE064CF1092310F81E08093F8
:10EE50002F0F10922E0F61E084E10E94C08B61E0C1
:10EE600085E10E94C08BE9EBF0E080818E7F80839A
:10EE700080818D7F808388E48093B80085E48093CF
:10EE8000BC000895413208F043C09091310F9111B8
:10EE9000FCCF91E09093310F20932F0F2FEF209311
:10EEA000C40E1092090F240F2093080F9093300F77
:10EEB0009091300F880F892B8093300F80912E0F07
:10EEC000813061F410922E0F8091300F8093BB003F
:10EED0008091BC0083FDF8CF85EC01C085EE809366
:10EEE000BC008091310F8130E1F38091090F8417CC
:10EEF00010F44091090F2AE03FE0FB01D9018A2F6D
:10EF0000821B841718F48D918193F9CF842F089573
:10EF100080E008950F93413208F04AC09091310F7C
:10EF20009111FCCF92E09093310F00932F0F9FEF40
:10EF30009093C40E1092090F4093080FFB016AE0F2
:10EF40007FE0DB019A2F961B941718F491919D9303
:10EF5000F9CF1092300F9091300F880F892B80934A
:10EF6000300F80912E0F813061F410922E0F80911E
:10EF7000300F8093BB008091BC0083FDF8CF85ECFF
:10EF800001C085EE8093BC00222321F08091310FD7
:10EF90008230E1F38091C40E8F3F61F08091C40E06
:10EFA000803251F08091C40E803341F483E007C079
:10EFB00081E005C080E003C082E001C084E00F91E1
:10EFC0000895613298F42091310F243089F46093D0
:10EFD000E60EFC0188EE9EE0DC012A2F281B261796
:10EFE00018F421912D93F9CF80E0089581E00895E0
:10EFF00082E0089585ED8093BC008091BC0084FD83
:10F00000FCCF1092310F089585EC8093BC001092D4
:10F01000310F08951F920F920FB60F9211240BB665
:10F020000F922F933F934F935F936F937F938F93A1
:10F030009F93AF93BF93EF93FF938091B900887F25
:10F04000803609F49DC070F5883209F45CC090F4F4
:10F05000803109F455C038F4882309F4F3C08830AE
:10F0600009F44EC0F2C0883109F44DC0803209F471
:10F070005EC0EBC0803409F469C050F4803309F4F9
:10F0800056C0883309F0E1C08093C40EBDDFDDC0F7
:10F09000803509F44FC0883509F45DC0883409F023
:10F0A000D4C0D2C0883909F4C3C0A8F4883709F4A1
:10F0B00067C038F4883609F463C0803709F460C04B
:10F0C000C4C0883809F4B4C0803909F45FC08038FE
:10F0D00009F0BBC05BC0803B09F482C038F4803AC1
:10F0E00009F466C0883A09F47BC0AFC0803C09F4DB
:10F0F000A3C0883C09F4A0C0883B09F486C0A5C021
:10F100008091300F10C09091090F8091080F9817CF
:10F1100070F5E091090F81E08E0F8093090FF0E008
:10F12000E65FF04F80818093BB0085EC82C08093C6
:10F13000C40E8AC0E091090F81E08E0F8093090F01
:10F140008091BB00F0E0E65FF04F80839091090F63
:10F150008091080F6AC0E091090F81E08E0F8093C3
:10F16000090F8091BB00F0E0E65FF04F8083809153
:10F170002F0F811169C081E080932E0F84EA5DC05A
:10F1800083E08093310F1092C50ECFCF8091C50ED2
:10F19000803208F04DC0E091C50E81E08E0F809363
:10F1A000C50E8091BB00F0E0EA53F14F8083BDCFE4
:10F1B0002BDF8091C50E803230F4E091C50EF0E077
:10F1C000EA53F14F10826091C50E70E0E0912A0F72
:10F1D000F0912B0F86EC9EE019951092C50E35C06C
:10F1E00084E08093310F1092E70E1092E60EE091CA
:10F1F0002C0FF0912D0F19958091E60E811105C00D
:10F2000081E08093E60E1092E80EE091E70E81E037
:10F210008E0F8093E70EF0E0E851F14F80818093EC
:10F22000BB009091E70E8091E60E981708F47DCF11
:10F2300085E88093BC0009C085EC8093BC001092E7
:10F24000310F03C01092C40ED5DEFF91EF91BF9134
:10F25000AF919F918F917F916F915F914F913F916E
:10F260002F910F900BBE0F900FBE0F901F9018950F
:10F27000FC0181E08083118243EC5BEA66E77BE37B
:10F28000428353836483758348ED5BE666E77BE3E3
:10F29000468357836087718742EF54EE64E67BE3D1
:10F2A00042875387648775870895FC01DB014D9180
:10F2B0005D916D917C911397428353836483758331
:10F2C00014964D915D916D917C911797468357836C
:10F2D0006087718718964D915D916D917C911B9718
:10F2E00042875387648775870895CF93DF93FC0126
:10F2F000EB014281538164817581488359836A831C
:10F300007B8346815781608571854C835D836E83E5
:10F310007F8382859385A485B58588879987AA8709
:10F32000BB87DF91CF9108950F931F93CF93DF9306
:10F33000082F6FEE76E08BE39FE00E940391C7E019
:10F34000D0E010E0B8010C2E02C0759567950A94C4
:10F35000E2F76170772742E050E08BE39FE00E9484
:10F36000ED91219778F7DF91CF911F910F9108953B
:10F370001F93CF93DF931F92CDB7DEB7162F63E5B0
:10F3800070E082E79EE04983E6DC612F82E79EE041
:10F3900091DC4981642F82E79EE08CDC82E79EE06D
:10F3A0000F90DF91CF911F914ACDCF93DF93EC0166
:10F3B00082E79EE0BDDC40E06DE2CE01D9DF40E1B6
:10F3C0006DE2CE01D5DF48E06DE2CE01DF91CF9155
:10F3D000CFCF6F3F710534F4AB0177FF05C040E03C
:10F3E00050E002C04FEF50E06DE1C2CFEF92FF92CC
:10F3F0001F93CF93DF931F92CDB7DEB77C01142FFD
:10F40000462F6EE12983B4DF412F6FE1C701B0DFE2
:10F410002981422F60E2C7010F90DF91CF911F91A8
:10F42000FF90EF90A5CF6F3F710534F4AB0177FFEC
:10F4300005C040E050E002C04FEF50E061E298CFDD
:10F44000462F62E295CF6F3F710534F4AB0177FF31
:10F4500005C040E050E002C04FEF50E063E288CFCB
:10F460006F3F710534F4AB0177FF05C040E050E019
:10F4700002C04FEF50E064E27BCF6F3F710534F480
:10F48000AB0177FF05C040E050E002C04FEF50E015
:10F4900065E26ECF6F3F710534F4AB0177FF05C0B5
:10F4A00040E050E002C04FEF50E066E261CF6F3FB6
:10F4B000710534F4AB0177FF05C040E050E002C0B5
:10F4C0004FEF50E068E254CF6F3F710534F4AB0169
:10F4D00077FF05C040E050E002C04FEF50E069E226
:10F4E00047CFAF92BF92CF92DF92EF92FF920F93EE
:10F4F0001F93CF93DF938C01C62F7A01690163E5D7
:10F5000070E082E79EE027DC6C2F82E79EE0D2DB92
:10F5100082E79EE094DC63E570E082E79EE01BDC1E
:10F52000A70163E570E082E79EE087DCE6015E010B
:10F53000AC18BD0882E79EE066DB892B29F082E7E4
:10F540009EE069DB8993F3CFAE14BF0421F0F8018C
:10F55000108281E0818382E79EE0DF91CF911F914D
:10F560000F91FF90EF90DF90CF90BF90AF9067CC5E
:10F57000CF92DF92EF92FF920F931F93CF93DF937F
:10F58000EC016B017A0189019C01225F3F4F46E04B
:10F5900050E062E3A6DF8F8590E0982F88272E85C4
:10F5A000822BF60191838083898990E0982F8827A8
:10F5B0002889822BF701918380838B8990E0982F93
:10F5C00088272A89822BF80191838083DF91CF914C
:10F5D0001F910F91FF90EF90DF90CF9008959B01C6
:10F5E0002C5F3F4FAB014E5F5F4FC2CFAF92BF92D8
:10F5F000CF92DF92EF92FF920F931F93CF93DF93FF
:10F6000000D000D0CDB7DEB77C015B01BE016F5FDB
:10F610007F4FE5DFCE0101966C01870175015E0128
:10F6200097E0A90EB11CF601619171916F018827D5
:10F6300077FD8095982F0E94FB99F80122813381F4
:10F64000448155810E948F9BF7016193719381934F
:10F6500091937F010C5F1F4FCA14DB0421F726969C
:10F660000FB6F894DEBF0FBECDBFDF91CF911F91D3
:10F670000F91FF90EF90DF90CF90BF90AF900895E3
:10F68000CF93DF931F92CDB7DEB79E012F5F3F4F21
:10F6900041E050E06DE125DF898190E00F90DF913E
:10F6A000CF910895AF92BF92CF92DF92EF92FF92E7
:10F6B0000F931F93CF93DF931F92CDB7DEB78C01CB
:10F6C0005B016A0179019E012F5F3F4F41E050E0ED
:10F6D0006EE107DF898190E0F501918380839E01CF
:10F6E0002F5F3F4F41E050E06FE1C801FADE8981B2
:10F6F00090E0F601918380839E012F5F3F4F41E0B0
:10F7000050E060E2C801EDDE898190E0F70191836D
:10F7100080830F90DF91CF911F910F91FF90EF9019
:10F72000DF90CF90BF90AF900895CF93DF931F925B
:10F73000CDB7DEB79E012F5F3F4F41E050E061E261
:10F74000D0DE898190E00F90DF91CF910895CF9323
:10F75000DF931F92CDB7DEB79E012F5F3F4F41E091
:10F7600050E062E2BEDE898190E00F90DF91CF91A0
:10F770000895CF93DF931F92CDB7DEB79E012F5F21
:10F780003F4F41E050E063E2ACDE898190E00F90B2
:10F79000DF91CF910895CF93DF931F92CDB7DEB75E
:10F7A0009E012F5F3F4F41E050E064E29ADE898185
:10F7B00090E00F90DF91CF910895CF93DF931F9248
:10F7C000CDB7DEB79E012F5F3F4F41E050E065E2CD
:10F7D00088DE898190E00F90DF91CF910895CF93DB
:10F7E000DF931F92CDB7DEB79E012F5F3F4F41E001
:10F7F00050E066E276DE898190E00F90DF91CF9154
:10F800000895CF93DF931F92CDB7DEB79E012F5F90
:10F810003F4F41E050E068E264DE898190E00F9064
:10F82000DF91CF910895CF93DF931F92CDB7DEB7CD
:10F830009E012F5F3F4F41E050E069E252DE898137
:10F8400090E00F90DF91CF910895CF93DF931F92B7
:10F85000CDB7DEB79E012F5F3F4F41E050E06CE235
:10F8600040DE69816F7070E066507109882777FD0E
:10F870008095982F0E94FB999B01AC0160E070E09D
:10F8800080E090E40E94F29B20E030E048EC50E4FD
:10F890000E948F9B0F90DF91CF910895EF92FF927E
:10F8A0000F931F93CF93DF931F92CDB7DEB78C01D9
:10F8B000CB01BA0120E030E048EC50E40E942F99DF
:10F8C0000E94C899E12CF12C759567956115710519
:10F8D00021F08FEFE81AF80AF7CF8AE0E816F10472
:10F8E00084F49E012F5F3F4F41E050E06CE2C8017D
:10F8F000F8DD46E04E0D8981807F482B6CE2C8011F
:10F9000037DD0F90DF91CF911F910F91FF90EF9016
:10F910000895CF93DF931F92CDB7DEB79E012F5F7F
:10F920003F4F41E050E060E3DCDD89810F90DF91E3
:10F93000CF910895DF92EF92FF920F931F93CF9391
:10F94000DF931F92CDB7DEB78C01F62EE42ED22EB8
:10F950009E012F5F3F4F41E050E0C3DD898121E0F0
:10F9600030E00E2C01C0220F0A94EAF7DD2011F0DE
:10F97000282B02C020952823298349816F2DC80197
:10F98000F7DC0F90DF91CF911F910F91FF90EF90D7
:10F99000DF900895262F47E050E061E3CBCF262F7C
:10F9A00046E050E067E2C6CF262F45E050E067E230
:10F9B000C1CF262F44E050E067E2BCCF262F42E0C3
:10F9C00050E067E2B7CF262F41E050E067E2B2CFC8
:10F9D000262F40E050E067E2ADCF262F47E050E011
:10F9E00067E2A8CF262F43E050E067E2A3CF262F9F
:10F9F00043E050E06AE29ECF262F42E050E06AE208
:10FA000099CF262F41E050E06AE294CF262F40E0C4
:10FA100050E06AE28FCF262F44E050E06CE28ACFBC
:10FA2000242F462F50E06FE285CF242F462F50E041
:10FA30006EE280CF1F93CF93DF931F92CDB7DEB7D7
:10FA4000142F9E012F5F3F4F41E050E04ADD898136
:10FA500090E002C0959587951A95E2F781700F9016
:10FA6000DF91CF911F91089547E050E061E3E2CF2D
:10FA700046E050E067E2DECF45E050E067E2DACFF3
:10FA800044E050E067E2D6CF42E050E067E2D2CFF8
:10FA900041E050E067E2CECF40E050E067E2CACFFD
:10FAA00043E050E067E2C6CF43E050E06AE2C2CFF5
:10FAB00042E050E06AE2BECF41E050E06AE2BACFF5
:10FAC00040E050E06AE2B6CF46E050E06BE2B2CFF1
:10FAD00045E050E06BE2AECF44E050E06BE2AACFED
:10FAE00042E050E06BE2A6CF41E050E06BE2A2CFF3
:10FAF00040E050E06BE29ECF43E050E06BE29ACFF3
:10FB000044E050E06CE296CF462F50E060E392CFA5
:10FB1000462F50E06FE28ECF462F50E06EE28ACF44
:10FB2000EF92FF920F931F93CF93DF931F92CDB766
:10FB3000DEB77C016DE67AE08BE39FE00E940391E3
:10FB40009E012F5F3F4F41E050E060E0C701C9DCFC
:10FB50008981EADB62E17BE08BE39FE00E942E91EA
:10FB60000DE110E069E97AE08BE39FE00E940391E8
:10FB700040E150E0B8018BE39FE00E94ED9168EB1B
:10FB800079E08BE39FE00E9403919E012F5F3F4F3E
:10FB900041E050E0602FC701A4DC8981C5DB62E150
:10FBA0007BE08BE39FE00E942E910F5F1F4F0A3393
:10FBB0001105C1F60F90DF91CF911F910F91FF902A
:10FBC000EF900895FB016181828170E0762F6627B6
:10FBD000680F711D882777FD8095982F0E94FB99EB
:10FBE00020E030E040E85DE30E948F9B23E333E9AF
:10FBF00048E853E40C946498089521E06227FC01DE
:10FC000080810C94C08BCF93DF93EC01862F6883A7
:10FC100049832A8361E00E94878B61E088810E948A
:10FC2000C08B60E089810E94878B60E08A810E949E
:10FC3000878B61E089810E94C08B61E08A810E948C
:10FC4000C08B60E0CE01DF91CF91D7CFFB018181E6
:10FC50009081890F9281890F9381981304C081E06C
:10FC600094819D3009F080E008952F923F924F9249
:10FC70005F926F927F928F929F92AF92BF92CF923C
:10FC8000DF92EF92FF920F931F93CF93DF9300D0F9
:10FC900000D0CDB7DEB78C013B014E830E94498A6C
:10FCA0001B012C0180ED280E87E0381E411C511CE1
:10FCB00061E0C801A2DFFE0131966F014E01F6E05E
:10FCC0008F0E911CF60185E011928A95E9F7760175
:10FCD00027E0A22EB12CF80181810E94F58B0197BB
:10FCE00039F40E94498A621573058405950598F3D5
:10FCF000F80181810E94F58B892B39F40E94498A91
:10FD0000621573058405950598F3F80182810E94B8
:10FD1000F58B892B59F0F701208181E090E00A2CC6
:10FD200001C0880F0A94EAF7282B2083F1E0AF1A6C
:10FD3000B10888F69FEFE91AF90AE814F90441F6C8
:10FD40000E94498A621573058405950540F060E0BC
:10FD5000C80153DF20E030E040EC5FE72EC089812E
:10FD6000EE818E13AFCFB601C80170DF882309F48E
:10FD7000A9CF60E0C80141DFB601C80123DFFB0164
:10FD8000DC016A946728B9F420E030E040E151E4F6
:10FD9000BF01CD010E948F9B20E030E040EA50E49B
:10FDA0000E942F9920E030E040E052E40E946598E4
:10FDB0009B01AC0102C09F01AD01B901CA012696A9
:10FDC0000FB6F894DEBF0FBECDBFDF91CF911F916C
:10FDD0000F91FF90EF90DF90CF90BF90AF909F90EA
:10FDE0008F907F906F905F904F903F902F900895ED
:10FDF00046E63BCF4CE439CFFC011382128282EFFE
:10FE00009AE091838083148260874187228788E00B
:10FE100083870895FF920F931F93CF93DF938C01F5
:10FE200082E79EE00E94987664E77AE08BE39FE0A9
:10FE30000E942E91C0E0D0E087E2F82E6F2D82E77D
:10FE40009EE00E94A17682E79EE00E941F778111CA
:10FE50001EC060E87AE08BE39FE00E94039140E1DE
:10FE600050E06F2D8BE39FE00E942692F801F48210
:10FE70006CE97AE08BE39FE00E94039140E150E05F
:10FE80006F2D8BE39FE00E94269221960FC0843055
:10FE900069F466EB7AE08BE39FE00E94039140E116
:10FEA00050E06F2D8BE39FE00E942692F394F0E4E4
:10FEB000FF12C4CFCD2B19F461ED7AE002C067EEDA
:10FEC0007AE08BE39FE0DF91CF911F910F91FF903C
:10FED0000C942E911F93CF93DF93EC01162F6C811E
:10FEE00082E79EE00E94A176E091720EF091730E7F
:10FEF0006B85612B0190F081E02D82E79EE01995E2
:10FF000082E79EE0DF91CF911F910C941F77FC0157
:10FF1000138660E0DFCF28E0FC01238760E0DACFC2
:10FF20001F93CF93DF93EC01162F6460D3DF81E042
:10FF300090E00E949E8A612F6B7FCE01CBDF82E32F
:10FF400090E0DF91CF911F910C949E8A1F93CF93E5
:10FF5000DF93EC01162FBEDF612FCE01DF91CF9131
:10FF60001F91DECFEF92FF921F93CF93DF931F92EB
:10FF7000CDB7DEB77C01162F607F642B4983E6DFA7
:10FF800080E1189FB00111244981642BC7010F90B3
:10FF9000DF91CF911F91FF90EF90D8CF40E0E2CF5B
:10FFA00061E0FCDF80ED97E00C949E8A62E0F6DF72
:10FFB00080ED97E00C949E8ACF93DF93CDB7DEB7A8
:10FFC00028970FB6F894DEBF0FBECDBF28E0E4E05F
:10FFD000F5E0DE01119601900D922A95E1F7FC0102
:10FFE0002185241710F44FEF420FFE013196E40FE4
:10FFF000F11DE40FF11D2081260F2068622F289645
:020000021000EC
:100000000FB6F894DEBF0FBECDBFDF91CF91C6CF44
:10001000FC0166816B7F66836860C0CFFC016681EE
:10002000262F246026836C60B9CFCF92DF92EF92A7
:10003000FF920F931F93CF93DF931F921F92CDB721
:10004000DEB78C01677088E0689FB001112460649E
:10005000C80149835A83A2DF4981C42E5A81D52E13
:10006000E12CF12CD6016D916D01D801ED91FC913F
:100070000190F081E02DC8011995BFEFEB1AFB0A42
:10008000E8E0EE16F10471F70F900F90DF91CF9139
:100090001F910F91FF90EF90DF90CF90089541E076
:1000A00061DF81E090E00895CF93DF93EC0182E778
:1000B0009EE00E9498761D828985823010F098E03B
:1000C0009D839A85992329F0813019F48D8184606C
:1000D0008D8362E370E080E090E00E94788A6B8517
:1000E000CE01F8DE68EE73E080E090E00E94788A4E
:1000F00060E3CE012BDF84E991E10E949E8A60E3F8
:10010000CE0124DF84E991E10E949E8A60E3CE0162
:100110001DDF86E990E00E949E8A60E2CE0116DF34
:100120006D816062CE013ADF84E08E83CE0176DF9E
:10013000CE0136DF82E08F8366E0CE012FDFCE0175
:10014000DF91CF9133CFFC0110821482138215828C
:100150000895862F642F0C94878B862F642F0C9420
:10016000C08B862F0C94F58B4F925F926F927F928B
:100170008F929F92AF92BF92CF92DF92EF920F93A6
:10018000CF93DF93EC014B013A0159010296DBDF7B
:100190008AEF9AE0998388836E018CE1C80ED11CA6
:1001A00026018CE3480E511CC601CDDF86E0C80E47
:1001B000D11CC414D504C1F7FE01EE59FF4F718262
:1001C00060823296B182A082329600833196E082BC
:1001D00037979182808238968AE090E0918380837D
:1001E000329684EF91E0918380833396118210825E
:1001F00071971082118212821382C459DF4F1882C4
:10020000DF91CF910F91EF90DF90CF90BF90AF90A3
:100210009F908F907F906F905F904F9008952F9256
:100220003F924F925F926F927F928F929F92AF9286
:10023000BF92CF92DF92EF92FF920F931F93CF93D3
:10024000DF93CDB7DEB728970FB6F894DEBF0FBEA9
:10025000CDBF98878F83F12C4C0186E6880E911CC8
:100260000F8118850E591F4FD4018C91F816A0F4F8
:10027000AF81B8858D919C91F801A081B181AF0DBE
:10028000B11DFC012081318142E06C918F81988504
:10029000F9011995F394E8CF512CEF81F885E959CC
:1002A000FF4FFA83E9830F8118850C591F4FC12C2A
:1002B000D12C7601C3948F8198858E599F4F9C8352
:1002C0008B83A981BA818C91581608F088C0A52C1F
:1002D000B12CAF81B8858D919C91F801A081B1813D
:1002E000AA0DBB1DFC012081318141E06C918F8101
:1002F0009885F9011995AF81B8858D919C91F80188
:10030000A081B181AA0DBB1DFC012281338140E097
:100310006C918F819885F9011995D701C601052C3B
:1003200004C0880F991FAA1FBB1F0A94D2F79C0113
:100330001C0120943094412CD4018C91EF81F885DC
:1003400040815181481648F5642C712CEB81FC8169
:10035000A081B181A60DB71DFA01448155816C9130
:100360008F8198852D833E83FA011995660C771C41
:100370002D813E81EF81F885E60DF71D892B29F44B
:1003800080859185822B932B04C080859185822165
:100390009321918780874394CFCFF801A081B181C9
:1003A000AA0DBB1DFA012281338141E06C918F813E
:1003B0009885F9011995AF81B8858D919C91F801C7
:1003C000A081B181AA0DBB1DFC012081318140E0DB
:1003D0006C918F819885F9011995539472CF289665
:1003E0000FB6F894DEBF0FBECDBFDF91CF911F9146
:1003F0000F91FF90EF90DF90CF90BF90AF909F90C4
:100400008F907F906F905F904F903F902F900895C6
:10041000FC0180E090E0258D368D2617370739F0F6
:10042000019636968A309105B1F78FEF9FEF0895C8
:10043000DC0126E0629FA00DB11D112490965C9313
:100440004E935F9721E091962C939197FC01E4598C
:10045000FF4F208131960190F081E02D222331F071
:10046000309749F0611107C0DC0102C0309719F0E4
:100470005C968C9119940895CF92DF92FF920F931E
:100480001F93CF93DF931F92CDB7DEB76C01F62E8B
:10049000FC0186E0689FE00DF11D112411A2878DFB
:1004A00090A181309105E1F01CF4892B51F042C0FC
:1004B0008230910581F1039709F03CC040E050E0A3
:1004C0002EC04423B9F141E050E0C601B1DFE1D7CD
:1004D000F601E85AFF4F60837183828393832AC0B9
:1004E0004983D7D7F601E85AFF4F00811181228155
:1004F0003381601B710B820B930B7296008111810B
:1005000020E030E04981061717072807390718F45B
:1005100042E050E004C041110DC043E050E06F2DB7
:10052000C6010F90DF91CF911F910F91FF90DF9047
:10053000CF907ECF0F90DF91CF911F910F91FF90C1
:10054000DF90CF9008952F923F924F925F926F92DB
:100550007F928F929F92AF92BF92CF92DF92EF9253
:10056000FF920F931F93CF93DF931F92CDB7DEB708
:100570001C01FC014AE08FEF9FEF278D30A1232B58
:1005800021F4148E968F858F11A241503696411119
:10059000F4CF712C610126E6C20ED11C510187E611
:1005A000A80EB11C4101A0E68A0E911C46E0442E23
:1005B000D6018C91781608F053C0612C8101070D8B
:1005C000111D070D111D085F1F4FF501E0806E140E
:1005D00008F044C0F80140815181062C02C05695B4
:1005E00047950A94E2F741707E9C70011124E60C55
:1005F000F11CD401ED91FC91EE0DFF1D5080B7016F
:10060000C101498305DF498197FD02C0682F1BC0E6
:10061000019611F5442301F180E090E060E070E084
:10062000F101E80FF91F248D211110C0469EF00141
:10063000479EF00D1124E20DF31D548EF68EE58ECB
:1006400010A2178E41E0C10117DF06C06F5F7F4F18
:1006500006966A30710521F76394B7CF7394A8CFDB
:1006600020E030E080E0F101E20FF31F91A1911151
:1006700081E02A5F3F4F2C333105A9F70F90DF91BE
:10068000CF911F910F91FF90EF90DF90CF90BF908F
:10069000AF909F908F907F906F905F904F903F9022
:1006A0002F900895CF92DF92EF92FF920F931F93B6
:1006B000CF93DF938C01EDD6E801C45ADF4FC88099
:1006C000D980EA80FB806C197D098E099F09F801A9
:1006D000E859FF4FC080D180E12CF12CC616D70617
:1006E000E806F90658F4C8019ADDC8012CDF182F76
:1006F000D0D6688379838A839B8301C010E0812FE1
:10070000DF91CF911F910F91FF90EF90DF90CF90ED
:1007100008950F931F93CF93DF93EC018C0104593D
:100720001F4F81E0F8018083CE01BCDF882349F0B0
:1007300089A1882331F08F8D98A1019711F48C8DB8
:1007400003C0F801108280E0DF91CF911F910F91DB
:1007500008950895CF92DF92EF92FF92FC01858970
:100760009689481B590B61097109A389B4899A01BB
:10077000AB010E94169D6B017C018FE0F594E7941C
:10078000D794C7948A95D1F765857685882777FDB4
:100790008095982F2BE0660F771F881F991F2A9549
:1007A000D1F727853089442737FD4095542F2C0DEC
:1007B0003D1D4E1D5F1D0E94F49C2C0D3D1D4E1DC8
:1007C0005F1DCA01B901FF90EF90DF90CF900895AF
:1007D0001F93CF93DF931F92CDB7DEB7162F67E736
:1007E00070E082E79EE049830E94AB76612F82E74A
:1007F0009EE00E945A764981642F82E79EE00E9423
:100800005A7682E79EE00F90DF91CF911F910C9472
:100810001F77CF93C62F67E770E082E79EE00E94C4
:10082000AB766C2F82E79EE00E945A7682E79EE0CC
:100830000E941F7767E770E082E79EE00E94AB7638
:1008400041E050E067E770E082E79EE00E941D779C
:1008500082E79EE00E940B76C82F82E79EE00E940E
:100860001F778C2FCF910895CF93DF93C62F67E723
:1008700070E082E79EE00E94AB766C2F82E79EE0FC
:100880000E945A7682E79EE00E941F7767E770E039
:1008900082E79EE00E94AB7642E050E067E770E0BE
:1008A00082E79EE00E941D7782E79EE00E940B7621
:1008B000D82F80E0C82F82E79EE00E940B76C82BDD
:1008C000D92B82E79EE00E941F77CE01DF91CF9166
:1008D0000895CF93DF93EC01643008F063E0688300
:1008E00082E79EE00E94987660EDCE0192DF85352A
:1008F00009F039C06AEACE01B7DF9A8389836CEACE
:10090000CE01B2DF9C838B836EEACE01ADDF9E8386
:100910008D8360EBCE01A8DF9A8B898B62EBCE01D1
:10092000A3DF9C8B8B8B64EBCE019EDF9E8B8D8B2C
:1009300066EBCE0199DF98878F8368EBCE0194DF59
:100940009A8789876AEBCE018FDF9C878B876CEB58
:10095000CE018ADF9E878D876EEBCE0185DF988B77
:100960008F8781E001C080E0DF91CF910895CF9320
:10097000DF93EC014EE264EF2BDF65E070E080E096
:1009800090E0B6D566EFCE01DF91CF916DCFCF93DA
:10099000DF93EC01ECDFAC0160E070E0CE01DADE69
:1009A000685F7F4F8F4F9F4F34E095958795779580
:1009B00067953A95D1F70E94FB9920E030E040E23C
:1009C00051E40E942F99DF91CF910895CF92DF9249
:1009D000EF92FF92CF93DF93EC0148814295440F51
:1009E000440F407C4C5C64EFF3DE8881811105C0CC
:1009F00065E070E080E090E012C0813029F468E0AA
:100A000070E080E090E00BC0823029F46EE070E08E
:100A100080E090E004C06AE170E080E090E068D59A
:100A200066EFCE0121DF6C01E12CF12CFE2CED2CC8
:100A3000DC2CCC2468EFCE01ECDEA7019601282B3C
:100A4000CA01B901488128E030E0241B310904C003
:100A500096958795779567952A95D2F7DF91CF91EF
:100A6000FF90EF90DF90CF9008952F923F924F929A
:100A70005F926F927F928F929F92AF92BF92CF922E
:100A8000DF92EF92FF920F931F93CF93DF93CDB737
:100A9000DEB72A970FB6F894DEBF0FBECDBF9A8798
:100AA000898765DF8C0189859A8590DF6D837E83D8
:100AB0008F839887A80160E070E089859A854ADE77
:100AC0004B015C0180EA881A8FE0980AA108B108FE
:100AD000A5019401C501B4010E949C9C2B013C011D
:100AE0000CE075946794579447940A95D1F7A985BB
:100AF000BA8511962D903C9012971C9115960D90E9
:100B0000BC91A02D0E94209D6B017C018DE0F5948D
:100B1000E794D794C7948A95D1F7E985FA85A78198
:100B2000B085A30192010E94209DBB2797FDB0953F
:100B3000AB2FC80ED91EEA1EFB1EF2E0CF0ED11C51
:100B4000E11CF11C32E0F594E794D794C7943A95F0
:100B5000D1F780E8D80EE11CF11CE985FA85A1895E
:100B6000B289A70196010E94169DDC01CB014FE0DE
:100B7000B695A795979587954A95D1F789839A83D6
:100B8000AB83BC836101EE24D7FCE094FE2C52E0E1
:100B9000CC0CDD1CEE1CFF1C5A95D1F7A185B2854B
:100BA000A30192010E94209D2B013C016BE07594F2
:100BB0006794579447946A95D1F7A381B481A501AE
:100BC00094010E94209DEBE0959587957795679518
:100BD000EA95D1F7460E571E681E791EC40CD51C27
:100BE000E61CF71C012E04C0CC0CDD1CEE1CFF1C07
:100BF0000A94D2F792E0C90ED11CE11CF11CC70186
:100C0000B60124E030E040E050E00E94F49C8D8189
:100C10009E81AF81B885821B930BA40BB50B9C0101
:100C2000AD0160E573EC80E090E004C09695879597
:100C3000779567951A95D2F70E949C9C97FD0DC0F9
:100C4000660F771F881F991F29813A814B815C812C
:100C50000E94D29C49015A010CC029813A814B81E2
:100C60005C810E94D29C49015A01880C991CAA1CE3
:100C7000BB1C9927B7FC9A958B2D7A2D692D9B016A
:100C8000AC010E949C9C9B01AC01AEEDBBE00E94BC
:100C9000169D6C01FF24D7FCF094EF2CA3E4B3EE77
:100CA000A50194010E94229DBB2797FDB095AB2F13
:100CB000C80ED91EEA1EFB1E9FECC90E9EE0D91E6F
:100CC000E11CF11CA4E0F594E794D794C794AA958D
:100CD000D1F7C80CD91CEA1CFB1CC701B6012A9627
:100CE0000FB6F894DEBF0FBECDBFDF91CF911F913D
:100CF0000F91FF90EF90DF90CF90BF90AF909F90BB
:100D00008F907F906F905F904F903F902F900895BD
:100D10008F929F92AF92BF92CF92DF92EF92FF920B
:100D2000CF93DF9300D01F92CDB7DEB74A015B01AE
:100D30009CDE6B017C0120E03AE24DE257E4C50104
:100D4000B4010E942F999B01AC0160E070E080E843
:100D50009FE30E94649826EF38E248EA50E40E943C
:100D6000F29B9B01AC01C701B60129833A834B83F7
:100D70005C830E94FB9929813A814B815C810E94AE
:100D80002F990E94C8990F900F900F900F90DF91AC
:100D9000CF91FF90EF90DF90CF90BF90AF909F905A
:100DA0008F900895CF93DF9300D01F92CDB7DEB719
:100DB0009A01AB0129833A834B835C8356DE0E9400
:100DC000FB9929813A814B815C810E942F9921E016
:100DD0003EED42E45EE30E94F29B9B01AC0160E0C9
:100DE00070E080E89FE30E94649820E03AE24DE2E0
:100DF00057E40E948F9B0F900F900F900F90DF9100
:100E0000CF9108953F924F925F926F927F928F920F
:100E10009F92AF92BF92CF92DF92EF92FF920F9389
:100E20001F93CF93DF9300D01F921F92CDB7DEB7F1
:100E30005C01562E19821A821B821C821D8261E07F
:100E4000852D65D460E0852D9BD462E170E080E063
:100E500090E04ED361E0852D93D488E290E06ED38C
:100E600060E0852D54D401E117E2852DBED4892B95
:100E700031F401501109C9F78EEF9FEF69C001E10C
:100E800017E2852DB2D4019721F401501109C9F759
:100E9000F3CF08E210E0312C37E0432E882483940E
:100EA000912C21E1E22E27E2F22E852D9ED4892B72
:100EB00029F481E0E81AF108C1F7DECFF6D26B0120
:100EC0007C0191E1692E97E2792E852D8ED40197D0
:100ED00029F4E1E06E1A7108C1F7CECFE6D26C19A1
:100EE0007D098E099F09693271058105910578F0A8
:100EF000E1E0F0E0EC0FFD1FE30DF11D2081C401E6
:100F0000042C01C0880F0A94EAF7282B2083411093
:100F100004C0339487E0482E01C04A94015011095F
:100F200009F0BFCF2981822F90E0F5019183808362
:100F30003B81832F90E093838283230F81E090E0B5
:100F40003D81321302C080E090E091958195910936
:100F50000F900F900F900F900F90DF91CF911F91F6
:100F60000F91FF90EF90DF90CF90BF90AF909F9048
:100F70008F907F906F905F904F903F900895FF9279
:100F80000F931F93CF93DF93FC010081C181D28126
:100F9000F8948981F02EF0948F21898378941DE74D
:100FA000115009F182E090E0C9D288818023C1F319
:100FB000F8948A818F218A838981802B8983789410
:100FC00080EE91E0BBD2F89489818F21898386E4F9
:100FD00090E0B4D28881802311E009F010E0789489
:100FE0008AE991E0ABD2812FDF91CF911F910F91D0
:100FF000FF9008951F93CF93DF93FC011081C1816F
:10100000D281912F909560FF11C0F8948A81892335
:101010008A838981812B89838AE090E08FD28A81BB
:10102000812B8A83789487E390E010C0F8948A81BA
:1010300089238A838981812B898381E490E07ED210
:101040008A81812B8A83789485E090E0DF91CF912B
:101050001F9174C20F931F93CF93DF93FC011081F4
:10106000C181D281F8948981812B89838A81012F62
:10107000009580238A8383E090E060D28981802379
:1010800089838AE090E05AD2C881789485E390E021
:1010900055D21C2381E009F480E0DF91CF911F91AC
:1010A0000F910895CF92DF92EF92FF920F931F93CB
:1010B000CF93DF931F92CDB7DEB76C01E62E08E029
:1010C00010E0FF24F39461E09F2D9E2109F460E07D
:1010D000C60149838FDFFF0C0150110949810115B9
:1010E000110589F7411115C0F894D6011196ED91BB
:1010F000FC91129791818C9180958923818311961F
:10110000ED91FC91129792818C9180958923828335
:1011100078940F90DF91CF911F910F91FF90EF90F6
:10112000DF90CF900895EF92FF920F931F93CF938C
:10113000DF938C01C8E0D0E0F12CEE24E394C801E9
:1011400089DF8111FE28EE0C2197C9F78F2DDF91E1
:10115000CF911F910F91FF90EF900895CF92DF9262
:10116000FF920F931F93CF93DF931F92CDB7DEB7FC
:101170008C01F62E40E065E5798394DFCF2C7981F0
:10118000D72E88E0F82EF60161916F0140E0C8018A
:1011900089DFFA94C1F70F90DF91CF911F910F91E2
:1011A000FF90DF90CF90089540E06CEC7BCFFC0186
:1011B00013861586148627E030E0DF01A20FB31FE7
:1011C00013961C922115310519F021503109F5CFE4
:1011D00008951F93CF93DF93EC01162F60E0812FCA
:1011E00096D2612F70E0FB01EF56F24FE491E88355
:1011F000FB01E952F24FE491F0E0EE0FFF1FE35ED6
:10120000F14F859194919A838983CE01DF91CF919B
:101210001F91CDCFAF92BF92CF92DF92EF92FF920C
:101220000F931F93CF93DF931F92CDB7DEB75C016F
:10123000D62EE72EFC01158511115EC049839FDE75
:101240004981811105C0F5011386158614866DC08C
:10125000442319F040E060EF02C040E06CEEC501AD
:1012600021DF01E0F12CC12C11E0C501F3DE682F74
:10127000C5016983EFDE6981613019F48130B9F409
:1012800032C02F2D30E068131BC0F501838518177D
:1012900030F4E20FF31F8381802349F402C0181752
:1012A00031F060E0193058F4F501148708C0F501F9
:1012B000EF0DF11D8381802B838361E009C0C12E76
:1012C000F501E20FF31F8381902F9095892383838B
:1012D000C50190DE1F5F000F11F4F39401E0F7E009
:1012E000FF1508F0C2CF113438F0F501C386C110E4
:1012F00009C081E0858706C0F5011386158614862E
:1013000010E013C0F50183818823B1F3ED2DFE2D8C
:1013100080E090E0D501A80FB91F13962C9121937E
:10132000019688309105B1F711E0812F0F90DF9180
:10133000CF911F910F91FF90EF90DF90CF90BF90D2
:10134000AF900895DC0180E0615088F09D9198276E
:10135000E92FEF70F0E0E55DF24F249192959F70D8
:10136000E92FF0E0E55CF24F84918227EDCF0895FC
:10137000FC01608308951F93CF93DF93EC01162F38
:10138000688182E79EE00E94A176612F82E79EE05D
:101390000E945A7660E082E79EE00E94AC7643E0CD
:1013A000688182E79EE00E941B7782E79EE00E94B0
:1013B0000B76EC0182E79EE00E940B7620E030E0A5
:1013C000382FC9018C2B9D2BDF91CF911F91089550
:1013D000D2DFBC0180E090E00E94F9992AE037ED6D
:1013E00043EA5CE30E948F9B23E333E948E853E43C
:1013F0000C946498089567E0EBCF66E0E9CF1F9204
:101400000F920FB60F9211242F933F938F939F93B8
:10141000AF93BF938091330F9091340FA091350F0C
:10142000B091360F3091320F23E0230F2D3720F487
:101430000196A11DB11D05C026E8230F0296A11D2E
:10144000B11D2093320F8093330F9093340FA093EC
:10145000350FB093360F8091370F9091380FA091D0
:10146000390FB0913A0F0196A11DB11D8093370F2E
:101470009093380FA093390FB0933A0FBF91AF916B
:101480009F918F913F912F910F900FBE0F901F90C2
:1014900018952FB7F8946091330F7091340F8091A5
:1014A000350F9091360F2FBF08953FB7F894809174
:1014B000370F9091380FA091390FB0913A0F26B5A0
:1014C000A89B05C02F3F19F00196A11DB11D3FBF7C
:1014D0006627782F892F9A2F620F711D811D911D0C
:1014E00042E0660F771F881F991F4A95D1F708952C
:1014F000CF92DF92EF92FF92CF93DF936B017C014B
:10150000D4DFEB01C114D104E104F10481F00E94A5
:101510006398CBDF6C1B7D0B683E734098F381E0D2
:10152000C81AD108E108F108C851DC4FEBCFDF91B0
:10153000CF91FF90EF90DF90CF900895823091058A
:1015400038F0880F991F880F991F05970197F1F7B9
:101550000895789484B5826084BD84B5816084BD2B
:1015600085B5826085BD85B5816085BDEEE6F0E01C
:10157000808181608083E1E8F0E010828081826078
:101580008083808181608083E0E8F0E080818160F9
:101590008083E1EBF0E0808184608083E0EBF0E029
:1015A000808181608083E1E9F0E0808182608083D6
:1015B000808181608083E0E9F0E0808181608083C8
:1015C000E1EAF0E0808182608083808181608083B5
:1015D000E0EAF0E0808181608083E1E2F1E08081F7
:1015E00082608083808181608083E0E2F1E080819D
:1015F00081608083EAE7F0E080818460808380817D
:101600008260808380818160808380818068808324
:101610001092C1000895809303050895863308F061
:10162000865320917B00982F9870277F922B909360
:101630007B0087702091030590E4299F900111247D
:10164000822B80937C0080917A00806480937A0062
:1016500080917A0086FDFCCF8091780020917900FE
:1016600090E0922B089590E0FC013197E231F10572
:1016700008F04CC0E955FF4F0C94109D80918000FC
:101680008F7703C0809180008F7D809380000895C4
:1016900080918000877FF9CF84B58F7702C084B5B1
:1016A0008F7D84BD08958091B0008F7703C08091B5
:1016B000B0008F7D8093B0000895809190008F7767
:1016C00007C0809190008F7D03C080919000877F3C
:1016D0008093900008958091A0008F7707C080913B
:1016E000A0008F7D03C08091A000877F8093A00021
:1016F0000895809120018F7707C0809120018F7D10
:1017000003C080912001877F809320010895CF93AB
:10171000DF9390E0FC01EF56F24F2491FC01E95277
:10172000F24F8491882349F190E0880F991FFC01C2
:10173000EF5AF14FA591B491895C914FFC01C5918D
:10174000D4919FB7611108C0F8948C9120958223A1
:101750008C93888182230AC0623051F4F8948C9172
:10176000322F309583238C938881822B888304C009
:10177000F8948C91822B8C939FBFDF91CF91089529
:101780000F931F93CF93DF931F92CDB7DEB7282F10
:1017900030E0F901E55BF24F8491F901EF56F24F29
:1017A0001491F901E952F24F04910023C1F088230A
:1017B00019F0698358DF6981E02FF0E0EE0FFF1F19
:1017C000E95CF14FA591B4919FB7F8948C916111A8
:1017D00003C01095812301C0812B8C939FBF0F9074
:1017E000DF91CF911F910F910895CF93DF93282F11
:1017F00030E0F901E55BF24F8491F901EF56F24FC9
:10180000D491F901E952F24FC491CC2389F08111AE
:101810002ADFEC2FF0E0EE0FFF1FE35EF14FA59102
:10182000B4912C912D2381E090E021F480E002C05E
:1018300080E090E0DF91CF9108950F931F93762F72
:1018400090E0FC01EF56F24F6491FC01E952F24F37
:10185000E4917111762FF0E0EE0FFF1FE35EF14F80
:101860008591949189019A013F70472F0E940A083F
:10187000611571058105910531F06F5F7F4F8F4FC5
:101880009F4F9F7003C060E070E0CB011F910F91EC
:101890000895FC01818D228D90E0805C9F4F821B1A
:1018A00091098F7399270895FC01918D828D981766
:1018B00031F0828DE80FF11D858D90E008958FEF56
:1018C0009FEF0895FC01918D828D981761F0828DB4
:1018D000DF01A80FB11D5D968C91928D9F5F9F7364
:1018E000928F90E008958FEF9FEF089587E49EE830
:1018F000892B39F080E090E0892B19F0C8D1811153
:1019000022C082EF9EE8892B39F080E090E0892B9D
:1019100019F068D281111AC08DE99FE8892B39F03E
:1019200080E090E0892B19F008D3811112C088E47F
:1019300090E9892B99F080E090E0892B79F0A8D389
:1019400081110AC008950E940000DBCF0E940000B0
:10195000E3CF0E940000EBCF0C9400000895FC013F
:10196000848DDF01A80FB11DA35ABF4F2C91848D28
:1019700090E001968F739927848FA689B7892C935D
:10198000A089B1898C9180648C93938D848D9813F8
:1019900006C00288F389E02D80818F7D80830895C1
:1019A000CF93DF93EC01888D8823C1F0EA89FB890E
:1019B000808185FD05C0A889B9898C9186FD0EC0FE
:1019C0000FB607FCF5CF808185FFF2CFA889B989D2
:1019D0008C9185FFEDCFCE01C2DFE8CFDF91CF91B3
:1019E0000895CF92DF92FF920F931F93CF93DF93CF
:1019F0001F92CDB7DEB76C0181E0D60158968C936B
:101A000058975B969C915B975C968C915C9798132A
:101A100007C05096ED91FC915197808185FD2DC0B6
:101A2000F601038D10E00F5F1F4F0F731127F02E8B
:101A3000F601848DF81210C00FB607FCF9CFD6015D
:101A40005096ED91FC915197808185FFF1CFC601B1
:101A5000698385DF6981ECCF838DE80FF11DE35A3F
:101A6000FF4F6083D6015B960C935B975296ED9186
:101A7000FC915397808180620CC0D6015696ED91FF
:101A8000FC91579760835096ED91FC91519780811E
:101A90008064808381E090E00F90DF91CF911F916F
:101AA0000F91FF90DF90CF900895BF92CF92DF9279
:101AB000EF92FF92CF93DF93EC016A017B01B22E8C
:101AC000E889F98982E08083411581EE5807610534
:101AD0007105A1F060E079E08DE390E0A701960147
:101AE0000E94D29C215031094109510956954795D0
:101AF00037952795211580E1380798F0E889F9890D
:101B0000108260E874E88EE190E0A70196010E94DF
:101B1000D29C215031094109510956954795379575
:101B20002795EC85FD853083EE85FF852083188E13
:101B3000EC89FD89B082EA89FB898081806180839C
:101B4000EA89FB89808188608083EA89FB898081BA
:101B500080688083EA89FB8980818F7D8083DF9123
:101B6000CF91FF90EF90DF90CF90BF900895CF93EB
:101B7000DF93EC01E881F9810284F385E02D19956A
:101B8000EA89FB8980818F7E8083EA89FB89808155
:101B9000877F8083EA89FB8980818F778083EA89C8
:101BA000FB8980818F7D80838A8D898FDF91CF91A2
:101BB0000895FC01538D448D252F30E0842F90E053
:101BC000821B930B541710F0CF9608950197089538
:101BD0001F920F920FB60F9211240BB60F922F93F4
:101BE0008F939F93EF93FF93E0914B0FF0914C0FE6
:101BF0008081E091510FF091520F82FD12C09081CF
:101C00008091540F8F5F8F732091550F821751F081
